:101000006F00801F6F00400073001000130181F813
:1010100023201100232231002324410023265100E4
:1010200023286100232A7100232CC101232ED10122
:101030002320E1032322F1032324A1022326B1026A
:101040002328C102232AD102232CE102232EF102FC
:101050002320010523221105232481042326910442
:1010600023282105232A3105232C4105232E510550
:101070002320610723227107232481072326910758
:101080002328A107232AB1076F00400073252034CD
:101090003703008013033300631865001703000053
:1010A000E700633E6F00400473252034370300805F
:1010B0001303B3006318650017030000E700233B28
:1010C0006F0080023703008013037300631865000C
:1010D00017030000E70083356F000001138600004E
:1010E00017030000E700233B832D4107032D010771
:1010F000832CC106032C8106832B4106032B01069A
:10110000832AC105032A8105832941050329010595
:101110008324C10403248104832841040328010497
:101120008327C10303278103832641030326010389
:101130008325C10203258102832F4102032F01026F
:10114000832EC101032E8101832341010323010169
:101150008322C10023244100232231008320010087
:101160001301810773002030F32240303713000051
:1011700013030380B3E26200739042306780000083
:10118000F32240303703000013030308B3E2620088
:101190007390423067800000F32240303703000034
:1011A00013038300B3E26200739042306780000053
:1011B000F322403037F3FFFF1303F37FB3F26200F3
:1011C0007390423067800000F322403037030010F4
:1011D000130373FFB3F26200739042306780000024
:1011E000F3224030370300001303F3F7B3F2620039
:1011F00073904230678000001721F87F130181420D
:10120000970200009382C2E073905230F3220030C4
:1012100093E282007390023017F5F77F130585DEA5
:1012200097F5F77F938505DE17F6F77F1306862E71
:101230003306B64097350100938585F817230100E2
:10124000E700434E17F5F77F1305C52C1726F87FE7
:101250001306463D3306A640B705000093850500FA
:1012600017230100E700035417030000E7004304BD
:101270001300000013000000130000001300000022
:1012800013000000130000006FF09FFE6FF05FD7A7
:10129000B7020000938232089382F2FFE39E02FEBF
:1012A0006780000067800000678000007D7106C6CF
:1012B00022C2EF00401BEF00801C0544930530055F
:1012C0002285EF00E0381375F5FBB705058023A6EE
:1012D000A514EF00A0083705F87F23080550EF009C
:1012E000D051EF00A043EF10E054EF00E03B630764
:1012F0008500EF00603B89456316B500EF00C036FE
:10130000EF70E07DEF00403A89456314B500EFC00F
:10131000400BEF30604BEF000055EF005113375595
:101320000100930585FF032585FF37060680CC4124
:101330002324A63E232EB63EEFF01FE3EF40302ECF
:10134000EF20000AEF408034EF207073EFB0B061FF
:10135000EF10316FEF806012D5B7000061113715C3
:101360000048B705F87F13064500B706F87F130756
:101370008500B707F87F1308C500B708F87F06C2D5
:1013800023AAA55023ACC65023AEE75023A0085390
:10139000EFF01FE50545A545EF00802B137585038C
:1013A000C1456316B50019651305C52021A019654F
:1013B000130505DC8145EF00C000924021016FF06C
:1013C0003FDC3706F87F03268651B706F87F1842C0
:1013D00083A64651944210426303C7008146369566
:1013E000B2953706F87FB336D50003260652B69578
:1013F0000CC2B705F87F83A5C55188C18280370527
:1014000000802308050082803705F87F0326855178
:101410003705F87F0C428326455188421842638481
:10142000E50088420C428280611106C2EFF05FDB6A
:10143000EF00E01BEFE060450545A545EF004021CA
:1014400013758503C1456316B50019651305C520DD
:1014500021A01965130505DC8145EFF09FF6924048
:1014600021016FF0FFD16FF0BFD4611106C2EFF020
:101470003FD4EF009034924021016FF0FFCE6FF027
:10148000BFD4611106C2EFF03FD4924021016FF04A
:10149000BFD06FF0FFDD00009305400A3305B502B1
:1014A000B725F87F938585802E9523260500232870
:1014B0000500232A0500232C0500232E05002320E8
:1014C00005022322050223240502232605022328E0
:1014D0000502232A0502232C0502232E05022320C0
:1014E0000504232205042324050482809305400A71
:1014F0003305B502B725F87F938585802E954C4539
:1015000091C59305C50090417D1690C10C4991C5C8
:101510009305050190417D1690C14C4991C59305F5
:10152000450190417D1690C10C4D91C593058501F3
:1015300090417D1690C14C4D91C59305C5019041D8
:101540007D1690C10C5191C59305050290417D1601
:1015500090C14C5191C59305450290417D1690C1B3
:101560000C5591C59305850290417D1690C14C554F
:1015700091C59305C50290417D1690C10C5991C546
:101580009305050390417D1690C14C5991C5930573
:10159000450390417D1690C10C5D91C5930585036F
:1015A00090417D1690C14C5D91C59305C503904156
:1015B0007D1690C12C4191C59305050490417D167F
:1015C00090C16C4191C59305450490417D1690C131
:1015D0002C4591C59305850490417D1690C16C45BD
:1015E00091C51305C5040C41FD150CC18280611124
:1015F000014506C2EFF09FEFEF00000B8945631530
:10160000B5000545EFF09FEE3715F87F8325857C03
:1016100091C58325857CFD152324B57CEF20102DF5
:101620003705F87F8325C56791C58325C567FD15F7
:10163000232EB5669240210182808280B725F87FF3
:1016400093858580C8D1C8517DFD23A20502828083
:1016500042058A052E95B70504802E950841B705E9
:10166000F87F23A0A5548280B7050680B0553705C2
:10167000F87F937606FB93E6A6002320C554B4D5E5
:10168000B705F87F83C545540946639EC500B70575
:101690000980AC55B706098013F605FB1366A60052
:1016A0002320B554B0D682803705F87F03454554D2
:1016B0008280370506809305F00F37060980B7064C
:1016C0000F8023240504232605042CC16CC1232884
:1016D0000504232A0504232005322322053223246E
:1016E000B5322326B532232E0504232406042326EF
:1016F00006042CC22CC223280604232A0604232015
:101700000632232206322324B6322326B632232E73
:10171000060423A6061823A806188280611106C2B3
:10172000EFF03FF937050F8005469305F002930669
:10173000F00F2320C5182326B518232805182322C7
:10174000D5182324D5183705F87F834545541385CC
:10175000F5FF1375F50F6365A610B70606803146D1
:1017600013050008B0C6E8C623A8060423AA060489
:1017700023A0063223A2063223AE06043705F87FE3
:10178000B8462320E554094893670708BCC603A759
:1017900086332320E5549367270023ACF63203A752
:1017A00086332320E5549377D7FF23ACF63203A783
:1017B000063F2320E5549367170023A8F63E03A7AE
:1017C00086332320E5549367470023ACF63203A702
:1017D00086332320E5549377B7FF23ACF632639129
:1017E0000509B7050980B0C523A6050423A805048B
:1017F00023AA050423A0053223A2053223AE050443
:10180000B0452320C55493660608B4C503A68533A6
:101810002320C5549366260023ACD53203A6853316
:101820002320C5549376D6FF23ACD53203A6053FBB
:101830002320C5549366160023A8D53E03A68533FE
:101840002320C5549366460023ACD532B7060980E1
:1018500083A585332320B55413F6B5FF23ACC632D8
:10186000924021018280611106C2EF000001EF1059
:101870007065924021016F00A0267D7106C626C2C8
:1018800022C0370606808325463C3705F87F93F64D
:10189000F5F72320B5542322D63CDD488325463E68
:1018A0002320B554294393F6F5F72322D63EB705F6
:1018B00009808326463E2320D554094413F7D6FFDA
:1018C0002322E63E370E058083A6053C2320D5540F
:1018D00013F7F6F723A0E53C232C063E3707F87FE5
:1018E0008326463C1308475293F7B6FF2320D5546E
:1018F0002322F63C1307000A83067800F14793E69B
:101900001600A303D8008326463C2320D55493F227
:10191000F6FB2322563CA302E8001307F00F8306D0
:10192000280093E6F6002301D800230A0800A3014B
:1019300018012324F62023026800232CE61C130838
:10194000D0028326C61D2320D55493E83600232ECB
:10195000161D2320061E9308A0058326461E23205D
:10196000D55493F2C6FF2322561EB9420323863371
:1019700023206554B7060F809373F3FD232C763232
:10198000930310030323461C232065542322661C63
:10199000232EE62613031004832E46332320D55529
:1019A00013EF1E00232AE633232C0631232A163197
:1019B00023248626232A562823AA76162324662C37
:1019C000C14E83234E022320755413FF8303630506
:1019D000DF01130FF00419A0130F30059303400A21
:1019E000232CE621232E7622B704F87F03C6445425
:1019F0006313860823A4F52023ACE51C83A7C51D2B
:101A00002320F55413EF370023AEE51D83A785335C
:101A10002320F55413FFF7FD23ACE53383A7451CC2
:101A20002320F55423A2F51C23AEE52603A7453356
:101A30002320E5549367170023AAF53223AC053120
:101A400023AA153123A4852623AA552823A4652C6F
:101A500003274E022320E554937787036385D7013C
:101A60001307F00419A013073005B707098023AC4A
:101A7000E52023AE772283A5C6162320B5547D1614
:101A800013F795FF23A6E6161376F60F83A5061720
:101A9000854713F795FF2320B55423A8E61663EA7C
:101AA000C700EF70207303C5445463148500EFB082
:101AB000502DEFD0700B03C5445411C537051400E9
:101AC0001306353029A037051400130635002945C3
:101AD000A145EF00403102449244B240416182800E
:101AE0007D7106C622C2EF00404F0944631B850C7E
:101AF000370505809305900F1306F00F2324B56E6C
:101B00002326C56E3706F87F8325C56E2320B6547D
:101B1000B707A48093F6F5FE2326D56EB705098096
:101B200083A685302320D6543708348013F776FCFB
:101B300023A4E530232E0560A14283A607112320AC
:101B4000D65413F7E6FF23A8E7108326080A2320BC
:101B5000D65413F736FF136747002320E80A1548C9
:101B600083A685302320D65413F7B6FF23A4E5308F
:101B7000370706808325C56E2320B65493F675FF7C
:101B80002326D56E9146832587302320B65493F7BC
:101B900075FC93E787012324F73099478325873025
:101BA0002320B65493F8B5FF23241731232A8560E8
:101BB0002326D562232A05632322F5622324556256
:101BC00039ACEF008041B70505809306F00F0D4654
:101BD00023A4D56E23A6D56E631BC5161305000B73
:101BE0009306F00323A4A55623A6D5563705F87F00
:101BF00083A6C56EB707098013F7F6FE2320D554D8
:101C000023A6E56E83A687302320D55413F776FCF0
:101C10001367870023A4E73083A687302320D55499
:101C200013F7B6FF23A4E73023AAC56003A6473005
:101C30002320C554937676FC93E6860023A2D73002
:101C4000854603A647302320C5541377B6FF23A249
:101C5000E73023ACD5603707068003A6C56E232086
:101C6000C554937676FF23A6D56E032687302320AE
:101C7000C554937676FC93E686002324D7309546A8
:101C8000032687302320C5541378B6FF2324073159
:101C900023AED560194803A6C7302320C5549376D8
:101CA00076FC23A6D73003A6C7302320C5549376ED
:101CB000B6FF23A6D73003A685562320C5549376B6
:101CC000D6FF23A4D55623A0056203264730232040
:101CD000C554937676FC93E686002322D73091464E
:101CE000032647302320C5549377B6FF2322F730CD
:101CF00023A2D562A1460326C7302320C55493777B
:101D000076FC93E787012326F73023A4856223A678
:101D1000056323A8D5621D4703A685562320C55415
:101D20009376F6FD23A4D55603A6856C2320C554CF
:101D3000937676FF23A4D56C03A6056C2320C554A7
:101D4000937676FF23A0D56C23AAE56249A81305F4
:101D5000E00F1306F00B23A4A55623A6C55637069D
:101D6000F87F03A5C56E370709809376F5FE23201B
:101D7000A65423A6D56E032587302320A654937638
:101D800075FC93E606032324D730032587302320F0
:101D9000A6549376B5FF2324D73023AE05603707CA
:101DA000068003A5C56E2320A654937675FF23A64F
:101DB000D56EB7060580032587302320A65493757A
:101DC00075FC93E585012324B73003258730232054
:101DD000A6549375B5FF2324B73023AA8660124416
:101DE000B2404161828042058A052E95B705048084
:101DF0002E9581459306000239A03357B600A10500
:101E00002300E5001105E39AD5FE8280611181452A
:101E100006C26305B500B705050019A0B7050200A5
:101E2000B7060480138686332E9618423706F87F4D
:101E3000937707022320E654A1C71387863D2E9788
:101E40001C431388063F93E817002E982320F6546E
:101E5000232017019386063E03270800AE9693675A
:101E600027002320E6542320F800856598429385B7
:101E70000580936717002320E6549CC2EF70706BB7
:101E80009240210182803706F87F231F06520DC53C
:101E90001305B00D6369B5041305E00BB7050680A3
:101EA000231FA65223A0A51E03A5451EB705F87F34
:101EB00023A0A5547199D9A8370506806C4537062B
:101EC000F87F93F6E5FF2320B65474C52320051E42
:101ED0008325451E2320B65493F6C5FF2322D51E25
:101EE00013054504D1A03705F87F130545528346F5
:101EF000C5001307C017B387E60213074006B3D720
:101F0000E70241689308C8FE7D18C697B3F707013A
:101F100063FAF5029946B3D6D50203454501958D7E
:101F20003385A540B7050680231FA6521376F50F0B
:101F300023A0C51EB706F87F83A5451E218123A0D7
:101F4000B65491A09307401AB386F60233D7E6023F
:101F50009946B3D6D5020345450151076373B700CF
:101F6000E115958D3385A5409375F50FB70606806D
:101F7000231FA65223A0B61E3706F87F83A5461E50
:101F80002320B6542181F1990D894D8DB705068026
:101F900023A2A51E3706F87FE8412320A6549366A6
:101FA0001500F4C11385C5040C413706F87F93E68C
:101FB00015002320B65414C18280611106C2EF407F
:101FC00010683705F87F0345455489456314B5000B
:101FD000EF50004A92402101828037050580832519
:101FE000856C3706F87F13D545000D89814623207F
:101FF000B6546313D50005458280611106C2EFF027
:10200000DFFD8D456314B500094525A0EFF0FFFC09
:102010008945631DB5003705058003250556B705BD
:10202000F87F1376150023A0A55419E2014511A0ED
:102030000545B705F87F2382A5549240210182808F
:102040007D7106C622C22A84EFF03FF98D456315E3
:10205000B5023705058003250557B705F87F01460A
:1020600023A0A5546305C4001365250011A075992C
:10207000B705058023A8A5561244B240416182806D
:102080007D7106C622C22A84EFF03FF58D456316A6
:10209000B5023705058003250557B705F87F0146CA
:1020A00023A0A5546305C4001365050419A0137586
:1020B000F5FBB705058023A8A5561244B24041613F
:1020C00082800D47638FE60005476384E602094777
:1020D0006389E602A1C281A094417D1614C19105D5
:1020E00011057DFA0DA883C605007D1614C185056E
:1020F000110575FA0DA094417D162300D5009105B8
:10210000050575FA09A8838605007D162300D5000C
:10211000850505056DFA828005476387E60099CA43
:1021200019A80CC17D1611056DFE31A02300B50064
:102130007D16050565FE8280211106CA26C64AC4A1
:1021400022C23284AA841389450011A88355C9FF8D
:10215000032609002685EFF01FC97D1421097DF4AF
:1021600012442249B244D2406101828042058A056C
:102170002E95B70504802E958145930600022E8783
:102180002320060009A8834705001105B397B7006F
:102190003E9718C2A105E398D5FE82803706F87FE6
:1021A000190513064652B70604803707F87F8347A0
:1021B000A5FF85CB0358C5FFC2070A08C297B6978B
:1021C00003A807008358E5FF8352050093C8F8FF72
:1021D000B3781801B3E858002320075523A017014E
:1021E00081A08357E5FF95C70358C5FF93C7F7FF45
:1021F000329883080800B3F7F8002300F8008357EB
:10220000C5FFB297038807008308050033681801EB
:1022100031A08357C5FF03080500B297238007014B
:10222000FD1593F7F50F2105D9F38280014601A82A
:1022300083060500FD1536961376F60F0505EDF9B4
:102240003305C0401375F50F8280211106CA26C6DA
:1022500022C209449304E00C2285A6854AC4EFF00B
:102260002FBF1365850037090680232CA9322285EC
:10227000A685EFF0EFBD5D99232CA93212442249C7
:10228000B244D240610182803D712D4593053004F6
:1022900006CE26CA4AC84EC652C422C2EFF04FBB71
:1022A0001375050825E93705F87F834585548DE5C5
:1022B0000149930900022D4493041004130A855424
:1022C00011A82285A685EFF0AFB8B3052A012380B7
:1022D000A5000509E31739FF2D4593053004EFF0FC
:1022E0002FB71375050405E137060F8001459305E7
:1022F00000081306060831A0B306C50023A0060097
:102300001105E31BB5FE3705F87F83058556850566
:102310002304B5561244224AB2494249D244F240FB
:102320000561828021112D459305400406CA26C609
:102330004AC44EC222C0EFF0AFB193050002636FF2
:10234000B5062D4593051006EFF08FB021893DE5C8
:102350003709F87F8345995605456381A5062D44C5
:1023600093042004A304A9562285A685EFF04FAE5E
:1023700013651500B7090F8023A4A9102285A6852F
:10238000EFF00FAD799923A4A9107D55930500278F
:10239000094605059356350063E8D50083469956EE
:1023A000E399C6FEA30409563705F87F8345A55671
:1023B00081C5FD152305B556EFF03FE9024492496A
:1023C0002249B244D24061018280211106CA26C648
:1023D0004AC4AE842A892D45930510064EC222C0F8
:1023E0003684B289EFF0CFA6218901E93705F87F5D
:1023F0000345955685456311B5024E85CA852686E7
:10240000A286EF00C004EFF05FE402449249224943
:10241000B244D240610182802D4593054004EFF023
:102420002FA393050002636BB500EFF0BFEF4E855D
:10243000CA852686A286EF008001C1BF4E85CA8567
:102440002686A286EF00A000EFF0DFED7DBF13012E
:1024500081FD06D252C85AC42E8A2A8B2D45930577
:10246000300426CE4ACC4ECA56C65EC222C0B68AB8
:10247000B289EFF0EF9D118941E1B70BF87F13842A
:10248000EB569304000201492285CA852686CA8636
:10249000EFF09FC81385190093956A004D8D23872F
:1024A000AB56A30064016309300113052400814683
:1024B000D2854E86EFF0FFC0890993F5F90F22858A
:1024C000EFF0DFD6B30534012380A50037050F8078
:1024D00001A8B305240183C505002320B510050913
:1024E000E31999FE3705F87F8345A55605466365D0
:1024F000B60085052305B5560244924B224BB24ADD
:10250000424AD2496249F2449250130181028280C8
:102510007D7106C6B2862303A100A303B100130593
:10252000610089451306000FEFF03FEAB2404161B8
:102530008280930545FE7D460145636BB6043746B0
:1025400001008A051306C681B2958C418285154526
:102550008280194582801D458280414582804545A3
:102560008280494582804D4582805545828059450B
:10257000828005458280094582800D458280114513
:10258000828035458280394582803D45828029455B
:1025900082800DC1FD1539460145636BB60837468B
:1025A00001008A051306C689B2958C418285130500
:1025B00000038280ED1545460145636BB60637463C
:1025C00001008A051306868DB2958C41828513051C
:1025D000400282801305100382801305200382804D
:1025E00013053003828013054003828013055003D6
:1025F00082801305600382801305C0038280130567
:10260000800382801305900382801305A0038280DB
:10261000130550028280130560028280714582801A
:1026200075458280794582807D4582801305200230
:102630008280130530028280130181FC06DA22C0F9
:102640002A8426D64AD44ED252D056CE5ACC5ECA0E
:1026500062C866C66AC46EC201C4EFA0305019A039
:10266000EF60A03EF5456305B50201C4EFA0104F31
:1026700019A0EF60803DA145630CB50001C4EFA037
:10268000F04D19A0EF60603C9305F0026310B516A1
:10269000B70CF87F938BBC5603C52B0005896307E5
:1026A000A014370CF87F93048C540385340003CDB9
:1026B0002400814522056314B400094911A015497D
:1026C000937D051093091008130AE008AD4A130B17
:1026D000C00C4A85CE85EFE0BFF71375050475F988
:1026E0004A85D285EFE0DFF6137505087DF1568542
:1026F000DA85EFE0FFF51375050261FD03C51400EF
:10270000D1456319B5041305400AB725F87F330591
:10271000A402938585802E952C51E9E903468C54BB
:10272000930505067D8A7D161357F64179833A96FF
:1027300085461357260094C1A302E5063725F87F86
:102740001376C63F1305C59D938524008146EFF09F
:102750005F9769A083C92B0033E9AD016D456360C4
:10276000A90413F5290005CD09459305000FEFE0F5
:102770003FEE83C5BC56937905022E85EFF07FDBD3
:10278000AA8603458C549357650063613005938591
:10279000440022854A863E87EFC0905681A003C53B
:1027A000BC56EFF01FD9AA8503851B0083468C54C5
:1027B0007D1513D619001377160093D7660093760C
:1027C000F50F22852686EF70E03B09A813864400AA
:1027D00005472285B685CA86EF70801403C52B0095
:1027E0001375E50F2381AB00EF0040020244924DC8
:1027F000224DB24C424CD24B624BF24A025A925991
:102800002259B254D250130181038280B705F87F58
:1028100037060F80014523840554930500081306ED
:10282000060831A0B306C50023A006001105E31B6E
:10283000B5FE82803D7106CE26CA22C009449304AB
:10284000E00C4EC652C4B7090680130AF00F228569
:10285000A6854AC856C223AA493FEFE07FDF6D999B
:102860001309800C23ACA9322285CA85EFE05FDE14
:102870001365450023A0A9322285A685EFE05FDD20
:102880005D9923ACA9322285CA85EFE07FDC136510
:10289000850023A0A9329305D00F2285EFE05FDBEE
:1028A0006D9923AAA93EEFE03FE063118506154428
:1028B0009304E00CB70A09802285A68523AA4A3F23
:1028C000EFE01FD96D991309800C23ACAA32228541
:1028D000CA85EFE0FFD71365450023A0AA32228501
:1028E000A685EFE0FFD65D9923ACAA322285CA8582
:1028F000EFE01FD61365850023A0AA329305D00F01
:102900002285EFE0FFD46D9923AAAA3E09449304DF
:10291000800C2285A685EFE0BFD3136505089305DB
:1029200000083706F87F23A0A93223A4B9322285F4
:10293000A685A3040656EFE0BFD1136505049305F1
:1029400000042D44930420043706F87F23A0A93205
:1029500023A4B9322285A68523040656EFE05FCF73
:102960001365450037090F802324A9102285A68509
:10297000EFE01FCE136585002324A9102285A685CC
:10298000EFE01FCD6D992324A9102285A685EFE0E5
:102990003FCC5D992324A9103705F87F1305B55660
:1029A000834525003706F87F93F5E50F2305065686
:1029B0002301B5000244924A224AB2494249D24414
:1029C000F24005618280130181FC06DA22D2930570
:1029D000B0032A8426D64AD463EE8504B7450100A5
:1029E00013152400938505922E950841028537051D
:1029F000F87F9305B55603862500B706F87F83C692
:102A000086541366360039A83705F87F9305B55606
:102A100003C62500B706F87F1376C60F83C6865413
:102A200013661600FD8A2381C500A3058556A38081
:102A3000D50095AD1305100F6302A4461305200FB2
:102A40006307A4461305C00F630EA4461305D00FF9
:102A5000631BA46481451305D00F2E86EFF05FAB96
:102A60003705F87F13068554034526008945631111
:102A7000B55C83467600514563E3A600AA8603054C
:102A800036008345460022054D8D834556002205BC
:102A90004D8D834566002205C98D2106094575A324
:102AA00081442685A6852686EFF09FA63709F87F04
:102AB00003458954930589547D891306F5FF37052D
:102AC000F87F890513059522A686EFF08FDF034571
:102AD00089547D897D159355F541F9812E9509819C
:102AE000B705F87F2384A522EF503076636D805AB6
:102AF000F545631AB55A0145EF6050346DA30144A2
:102B00000545A2852286EFF0BFA0B704F87F03C574
:102B10008454938584547D891306F5FF3705F87F27
:102B2000890513056524A286EFF0AFD903C5845447
:102B30007D897D159355F541F9812E950981B7055C
:102B4000F87FA382A52485A301440945A285228696
:102B5000EFF01F9CB704F87F03C584549385845419
:102B60007D891306F5FF3705F87F8905130585274D
:102B7000A286EFF00FD503C584547D897D1593554A
:102B8000F541F9812E950981B705F87F2384A528A1
:102B900019AB01440D45A2852286EFF07F973705DA
:102BA000F87F9305A5543705F87F13059528BDA830
:102BB0001145F5A13704F87F83448454EF50F06841
:102BC0009305F00363E0953693057002631DB54CE1
:102BD0006945EF503064154521A901441945A28586
:102BE0002286EFF0FF9291452285EF60500E7545E9
:102BF000F9A401441D45A2852286EFF07F91370597
:102C0000F87F9305A5543705F87F1305452739A8A4
:102C100001442145A2852286EFF09F8F3705F87F7A
:102C20009305A5543705F87F130505271146A2869D
:102C3000EFF02FC98DA93705F87F1305352691458B
:102C40005946EDA60145EF70601EB1A90145EF7030
:102C5000E01F91A93704F87F83448454EF50F05E5D
:102C60009305F00363E09530F5456307B500EF5039
:102C7000D05DA1456318B5443705F87F1305B556F7
:102C80008305250093E515002301B50029A95545C5
:102C900039A1EF50905B930580026316B53037057C
:102CA000F87F9305A5543705F87F014413053526B1
:102CB0001146A286EFF0EFC013059002EF50905539
:102CC000594529A201446545A2852286EFF05F841B
:102CD0003705F87F9304710011499305A5542685A3
:102CE0004A86A286EFF0EFBDB727F87F93878780EB
:102CF00003C85705034791001348280013381800EC
:102D00009312870003057100360893F2027083C5A1
:102D1000140033E80201A1621316850033685800DD
:102D2000B722F87F4D8EB706F87FB708F87F9382F9
:102D3000A29D1358880005432396C6262397E826AC
:102D400023812201A382A2002382B200A381020177
:102D5000A382670623A06706B9A6EF50104FF5457A
:102D6000631BB52801442285EF7040066D45B9A864
:102D70000145EF70403205AE130580020DA6EF50FD
:102D8000D04CA145631BB52601442285EF70000697
:102D900025452DA80145EF70600731A6EF50F04A98
:102DA000F545631EB52401458945EF6040726353C4
:102DB000A03005442285EFE07F882285EFE01F8860
:102DC000014499452285EF6080704945A28522869D
:102DD000C9AC01446945A2852286EFF06FF337053F
:102DE000F87F930471009305A55411462685A286A9
:102DF000EFF02FADB727F87F9387878003C857057B
:102E000003479100134828001338180093128700D5
:102E100003057100360893F2027083C5140033E88D
:102E20000201A1621316850033685800B722F87FAB
:102E30004D8EB706F87FB708F87F9382A29D1543A1
:102E40001358880085432396C6262397E8262381B6
:102E50006200A382A2002382B200A3810201A382A6
:102E6000770623A0770681A4130590020DACEF50DE
:102E7000D03DF5456317B5183705F87F0345A554D0
:102E80008945630FB52485456308B526636DA02089
:102E9000014593050008EF60706F31A4814513056B
:102EA000100F2E86EFF0CFE61305500209A88145DA
:102EB0001305200F2E86EFF0AFE513056002EF50EB
:102EC0007035D5A23705F87F9304855403C52400D7
:102ED0008945631FB51603C4740051456363A4009C
:102EE0002A840385340083C5440022054D8D83C5A3
:102EF000540022054D8D83C564002205C98D13063B
:102F0000D1000945A286EF00202093852400930478
:102F10007100014919462685CA86EFF08F9A13057C
:102F20006400A5A2F5456307B500EF501032A14536
:102F3000631DB51803458454130684549375F50135
:102F4000FD1593576500014593F6F50F8D452A87CA
:102F5000EF6050438345845413D66500630FA0147B
:102F6000154581A0F5456307B500EF50102EA1452A
:102F70006311B51603458454130684549375F50103
:102F8000FD1593576500014593F6F50FBD452A875A
:102F9000EF60503F8345845413D665006301A0124F
:102FA00051458145FDA8EF50502AA1456318B50E43
:102FB0003705F87F9305A5543705F87F13043526A8
:102FC000814411462285A686EFF0AF8F2685EF60FB
:102FD000700A635EA0003715F87F1305057F114660
:102FE0008146A285EFF0EF8D1945EF50B02259458B
:102FF00081452E867DA06D455DA025454DA04945A6
:1030000079A8EF509024A145631FB5083705F87FD4
:103010000345A55489456318B508EF600029A3034B
:10302000A1001305710085451306B0028146A5A0D5
:1030300083465600E54563E3B600AE868345360019
:1030400003474600A205D98D1906EF00001CA1A870
:1030500003C45400E5456363B4002E8483C5340083
:1030600003C64400A205D18D1306B100A286EF006D
:10307000A009938524009304710001491146268517
:10308000CA86EFF00F84130544009375F50F1306FD
:10309000C00F2685CA86EFF04FB331A0594585454C
:1030A0000146EFF0EFC612542259B254D250130128
:1030B0008103828049458945E5B7154511A05145F1
:1030C0008945C5B751458D45E1BF834584541545B4
:1030D00021A083458454514513D665008D45D1B751
:1030E000EF600018A303A10011CD1375F50F8545FE
:1030F000E319B5F2014525B7014593050008EF60D6
:10310000104755B7054521BF797106D626D222C48E
:103110003284AE8489454AD04ECE52CC56CA5AC863
:103120005EC6636FB500630BB502C1456314B50C91
:103130003705F87F13054552B3059500014775A083
:1031400013958400B705FF006D8DB70504802E959B
:103150009395240093F5C53FC98D79A013D58401BB
:10316000A9456318B506416513DA2600814A130B99
:10317000F5FF29499309410081A813952A00937B03
:10318000C53F33859B00B37565014A854E86EFE0E8
:10319000FFFD124593E61B0093E72B0093E83B00ED
:1031A000B305740113568500A29613570501A29723
:1031B00013588501A2982380A5002380C600238090
:1031C000E70023800801850A13F5FA0FE36745FB42
:1031D00015A0370600049395240071164205F18D61
:1031E0002E95B7050480AA95094722853686BA86AA
:1031F000EFE03FED2244B24B424BD24A624AF249E1
:1032000002599254B250456182803D7106CE26CA61
:1032100022C03284AE8489454AC84EC652C456C2C2
:10322000636EB500630AB502C1456310B50C37057E
:10323000F87F13054552269501475DA0139584003C
:10324000B705FF006D8DB70504802E95939524007A
:1032500093F5C53F4D8D61A013D58401A945631534
:10326000B506416593D92600014A930AF5FF29491D
:10327000B9A013152A001375C53F136615002296D1
:1032800093662500B305A40003460600A29683C5F5
:10329000050083C606002206D18D139606019366AB
:1032A0003500A29683860600D18D13968601269559
:1032B0004D8EB37555014A85EFE0FFB2050A1375CF
:1032C000FA0FE36835FB15A0370600049395240038
:1032D00071164205F18D2E95B70504802E95054790
:1032E000A2853686BA86EFE0DFDD0244924A224AA2
:1032F000B2494249D244F240056182807D7106C6DE
:103300003705F87F8345855422C213F6F50131C68F
:10331000B705F87F1384B5568345240093F615004E
:103320008DEE9306260001461307855401A88307F6
:103330000700FD163E961376F60F0507EDFA09EA2B
:103340001305855403451500EFF0EFE7834524008E
:1033500013F5150019E1EFF06FCB1244B240416153
:1033600082803D7106CE22C23704F87F0345845621
:1033700026CA4AC84EC652C421CDEFF03FF8030515
:1033800084567D159375F50F2304A456B1C12D45C0
:1033900093053004EFE0CFAB1375050805E9370559
:1033A000F87F0149930900022D4493041004130A85
:1033B000855411A82285A685EFE08FA9B3052A01BF
:1033C0002380A5000509E31739FF19A0230404563B
:1033D0001244224AB2494249D244F24005618280F5
:1033E000611106C2EFF0FFF7924021016FE09FF3F9
:1033F000130181FB86C23716F87F0346667C26DE02
:10340000AA844ADC4EDA52D856D65AD45ED262D05A
:1034100066CE6ACC6ECA22C8630BC0164165930C97
:10342000F5FF3705F87F130C157A3705F87F13057C
:1034300085542AC637052000814B9309F518374576
:1034400001000544130DF00F930D9003130A05A11D
:103450005E852EC435A2330B5C0103490B00834506
:103460001B0033F625016305A61333E6250163012E
:10347000C0121386A5FC63E1CD020A0652961042E3
:103480000286639C95049305F9FF13052B0093F5C1
:10349000F50FEF00303991A055456365B50233153E
:1034A000B4003375350119CD8DE83245DA85130640
:1034B0000002DE86EFE0FFC0EFF05FE439A8639E14
:1034C0009500C5A8130500036387A5001305D00F59
:1034D000E38CA5FC19A06385951213850A024DA003
:1034E00003053B00DE861316850003452B0013768B
:1034F0000610B36BA600639D950413058003639DBE
:10350000A40A83451B023725F87F03460B020355A7
:10351000A58AA205D18D6381A50A33857A0181A888
:1035200083053B0003462B00A20593F50510D18DC2
:10353000930610046386D40E5E85ED4663EFD502D4
:103540001375F6010DC9138505021375053E35A0E7
:10355000B6856D4663EBCB007D8911C513850B02E3
:103560009375053E19A093F50B1E3385BA0013051C
:103570000502B68B31A013F5051E569513050502FD
:10358000B37A950193D5CA00E307B0EC11A00544C6
:1035900022854244D24D624DF24C025C925B225B2A
:1035A000B25A425AD2596259F254964013018104D8
:1035B0008280A245090569A86D4563E3AB049305C4
:1035C000AB0313866BFE37050780854613840A021A
:1035D000EFE03FAF09459305000FEFE06F871375EC
:1035E000050231E5268533098C00EFE09FF40144A4
:1035F000AA862285CA855E862287EFB0707049BF91
:103600002685EFE01FF3AA851305F9FF01449376A1
:10361000F50F054722855A86A287EF60A0568DBF19
:10362000714663E4C502A245130600020DA026857B
:10363000EFE03FF033068C000144AA850547228560
:10364000DE86A287EF60C02DA1B7A2451146329554
:103650002390A50001442DBF3716F87F8346667C72
:103660000546639EC604C166B717F87F0143FD1681
:103670007D479387177A1308F00F930830049A82D6
:1036800033F3D200636D6702B3836700038E0300D8
:1036900083C31300B3FEC30163830E0333EEC30180
:1036A000137EFE0F630DC00113030302E31915FD22
:1036B000E39713FD1385220001462390A500328570
:1036C00082800000211106CA22C237050C80054401
:1036D00026C64AC42324852E9305201B2285EFD0BD
:1036E0003FF76D99B704058023A4A46C9305D0150A
:1036F0002285EFD0FFF53D999305F00A23AAA45641
:10370000056523A4B45621449304C5C02285A6852B
:10371000EFD01FF41365150037390C802328A90258
:103720002285A685EFD0DFF279992328A9021244D9
:103730002249B244D240610182803D7106CE4EC61C
:10374000AA89056552C422C02144130AC5C04AC8CB
:103750002E892285D28526CA56C2B284EFD05FEF69
:1037600013651500B73A0C8023A8AA022285D285DA
:10377000EFD01FEE799913D6890093F5F90F1376E0
:10378000F60F854637870C809307F00F23A8AA020F
:1037900005653728F87F23A4BA0023A6CA0023A80A
:1037A0002A0123A0DA0223A20A0223AEDA0023228E
:1037B000D73E232EF73A232C973C9304F5C005659A
:1037C0009309888029481309E5C02322D73E23AAFC
:1037D00009032285A685EFD0BFE711E52285CA85BA
:1037E000EFD01FE701C503A5490365F50244924ADE
:1037F000224AB2494249D244F24005618280130113
:1038000081FD06D24ECAAA89056552C856C6214A0C
:10381000930AC5C04ACC2E895285D68526CE5AC475
:1038200022C23684B284EFD0BFE213651500373B65
:103830000C802328AB025285D685EFD07FE113762A
:10384000E5FF13D5890093F6F90F1377F50F9377FA
:10385000F40F135884000545B7850C809308F00FCA
:103860002328CB022324DB002326EB0023282B0173
:103870002320FB0223220B03232EAB0023A2A53E11
:1038800023AE153B23A2A53E39A003C604007D1438
:1038900023ACC53C850475F823A2A53E05653726F3
:1038A000F87F9304F5C00565930986802946214475
:1038B0001309E5C023AAC9022285A685EFD05FD9E6
:1038C00011E52285CA85EFD0BFD801C503A54903FC
:1038D00065F51244224BB24A424AD2496249F24447
:1038E00092501301810282803D7106CE4EC6AA8994
:1038F000056526CA52C4A144130AC5C04AC82E8908
:103900002685D28556C222C03284EFD07FD413657B
:103910001500B73A0C8023A8AA022685D285EFD0DD
:103920003FD3799923A8AA020565B726F87F23A477
:103930003A0123A60A0023A82A01130905C1056537
:10394000854537860C80138A8680A9469309E5C091
:1039500023A0BA0223A20A0223AE0A002322B63E03
:10396000232EB63A232ADA022685CA85EFD05FCE07
:1039700011E52685CE85EFD0BFCD01C503254A03CD
:1039800065F509659305650F2145EFD07FCC2300D0
:10399000A4000244924A224AB2494249D244F24027
:1039A00005618280130181FD06D252C82A8A05650D
:1039B0004ACC56C62149930AC5C04ECAAE894A852B
:1039C000D68526CE5AC422C23684B284EFD05FC8D0
:1039D00013651500373B0C802328AB024A85D6853A
:1039E000EFD01FC779992328AB020565B727F87F69
:1039F00023244B0123260B0023283B01930905C1F7
:103A0000056593F5F40F13D68400B7860C8005473F
:103A1000938A8780A947130AE5C02320BB0223228B
:103A2000CB02232E0B0023A2E63E23AEE63A23AAC6
:103A3000FA024A85CE85EFD0BFC111E54A85D2850D
:103A4000EFD01FC101C503A54A0365F50965130938
:103A5000650FA14909A84E85CA85EFD07FBF230015
:103A6000A400FD140504E5F81244224BB24A424A70
:103A7000D2496249F24492501301810282800000CF
:103A8000611106C2EFF07FCB924001452101828097
:103A90007D7106C626C222C02E84AA8403C50400F6
:103AA00083C5140003C62400EFF09FFD7D14137539
:103AB000F40F8D0465F502449244B2400145416122
:103AC00082807D7106C626C222C03284AE84EFD0C9
:103AD000FFB62685A28502449244B24041616FF050
:103AE0003FFB7D7106C626C2894422C02A84930505
:103AF000000F2685EFD0DFB513750504630CA01009
:103B000011656302A4106306940611456309A406B7
:103B100021456308A4084145630BA408130500026E
:103B20006300A40A130500046303A40A1305000834
:103B30006304A40A130500106307A40A13050020F8
:103B4000630AA40A13050040630BA40C0565130562
:103B50000580630CA40C0565630EA40C0965630461
:103B6000A40A05456312A40EB705F87F2388A5585B
:103B700051A83705F87F23089558268469A0B70512
:103B8000F87F3706F87FB706F87F0547B707F87F55
:103B900023880558A308065823890658A389E7589F
:103BA00095A085453706F87FA308B658A1A8B705A4
:103BB000F87F03C625591376E60E1366160089A012
:103BC000B705F87F038625591366160115A8B705B2
:103BD000F87F238905583DA0B705F87F038625594E
:103BE0001366260031A8B705F87F03C6255913765A
:103BF000D60F39A0B705F87F03862559136646000E
:103C00002389C5582A843705F87F83156559C18DE6
:103C1000231BB55802449244B240416182808545DD
:103C20003706F87F230AB658F1BFB705F87F238A15
:103C30009558C9BFB705F87F0546B706F87F238AB0
:103C40000558A38AC6587DBF014475BF130181FD85
:103C50001306F5FF06D252C822C2137AF60F254684
:103C60002E8426CE4ACC4ECA56C65AC4636746290D
:103C7000A14A6366550161159304B01B19A0930412
:103C8000A01B85453399A5002E85A6859379240030
:103C9000EFD01F9C014B9375F90F638469014D8D23
:103CA00021A093C5F5FF6D8D93952400B70905807C
:103CB000B3E53501854488C119A813095B18268529
:103CC000CA85EFD0FF9863074501130BC9E7E3F6F8
:103CD0006AFF25A41375FB0F63E1AA22B745010013
:103CE0000A05938585AF2E95084102858544930585
:103CF000B01B2685EFD0DF953D9923A6A96E15450B
:103D00009305200CEFD0DF94137575FCB70509807F
:103D100023A4A5309305B01526850588EFD05F93C1
:103D20006364801A136505046DA215459305100C94
:103D3000EFD01F92137575FCB705098023A2A5303B
:103D400005459305B0150588EFD09F9063618018F5
:103D500013650508BDAA85449305B01B2685EFD0E1
:103D60003F8F5D9923A6A96E09459305200CEFD0DE
:103D70003F8E137575FCB705068023A4A530930507
:103D8000A01526850588EFD0BF8C63678014136566
:103D9000150095A215459305300CEFD07F8B137558
:103DA00075FCB705098023A6A53005459305A01528
:103DB0000588EFD0FF89636380121365250025AA6B
:103DC00009459305100CEFD0BF88137575FCB70536
:103DD000068023A2A53005459305A0150588EFD0E0
:103DE0003F87636F800E1365450031A20945930537
:103DF000300CEFD0FF85137575FCB705068023A640
:103E0000A53005459305A0150588EFD07F8479E896
:103E100013658500CDA037050C8085442324052E2D
:103E20009305201B2685EFD0BF826D9923A4A96C32
:103E30009305001B2685EFD0BF815D9923A0A96C57
:103E40009305A01526850588EFD09F8051EC13655A
:103E5000050155A085441309201B2685CA85EFD08E
:103E60002FFF6D9923A4A96C2685CA85EFD04FFE3C
:103E70005D9923A4A96C9305001B2685EFD04FFD07
:103E80005D9923A0A96C9305A01526850588EFD020
:103E90002FFC29EC13650502B9A837050C80854471
:103EA0002324052E9305D0152685EFD06FFA3D9972
:103EB00023AAA9569305A01526850588EFD04FF9AA
:103EC0000DE81365050405A81375F5FB19A0137516
:103ED000F5F723A6A95615A0799931A8759921A8B7
:103EE0006D9911A85D9901A83D9931A01375F5FD53
:103EF00019A01375F5FB23A4A9561244224BB24A0C
:103F0000424AD2496249F2449250130181028280AE
:103F10003D717D1506CE4AC822C01379F50F25459F
:103F20002E8426CA4EC652C456C263652507F95967
:103F3000214A854409A8938579182685EFD04FF149
:103F4000630825018509938A2900E3765AFF99A021
:103F500013F5FA0F89456367B500B3993401130966
:103F6000C01539A013050004B31955011309D01564
:103F70002685CA85EFD0CFED93F5F90F19C04D8D89
:103F800021A093C5F5FF6D8D931529003706058097
:103F9000D18D88C10244924A224AB2494249D24450
:103FA000F240056182807D7106C626C222C032843D
:103FB000AE84EFD0AFE803C6040003C5140083C588
:103FC000240001C6EFF0DFF419A0EFF03FC87D1424
:103FD0001375F40F8D0465F102449244B2404161BF
:103FE00082807D7106C626C222C03284AE84EFD0A4
:103FF000EFE413851400B70504800346F5FF03477B
:10400000050042062E960A0783461500598E7D1438
:1040100014C21376F40F0D056DF202449244B240BF
:1040200041618280611106C283461500BDC2370717
:10403000F87F835787590148BD4885421376F80FAA
:1040400063E4C8023393C200B373F3000508E36767
:1040500070FE3708F87F1308A8593298B3E7670055
:104060002300D800231CF758F9158D46B3C5D50297
:104070003707F87F0E061307C75A830605003A96DE
:1040800009052300D60048C2A300B60092402101D2
:1040900082800346050089466302D6028546630B8B
:1040A000D6026DF6F9150D4633C6C50293052500F7
:1040B00001451376F60FEFF01FEFC9BFF9150D4656
:1040C00033C6C5029305250001451376F60FEFF0C0
:1040D0005FF16DBFF9150D4633C6C5029305250086
:1040E00001451376F60FEFF0DF9D4DB73705F87FEA
:1040F0008325C56291C58325C562FD152326B5625A
:104100003705F87F035585591DC93707F87F814565
:10411000414685461307A7590DA0B397B600E98F0E
:1041200081CFB307B70003C8070063070001038806
:1041300007007D18238007018505E390C5FE828076
:10414000130181FD06D226CEB704F87F03D584592A
:104150004ACC4ECA52C856C65AC45EC222C049C5CD
:104160003705F87F1309055B01443705F87FC1491E
:10417000054A930AA559094BA28B63873B0703D5D0
:104180008459B3157A0133F6A50011C633867A0136
:104190000346060011C6850B2109E3923BFFA9A047
:1041A00013C6F5FF8345C9FF718D239CA458638D09
:1041B000650163834503E5F1832509000346D9FFC3
:1041C0002285EFF05FDEC1BF832509000346D9FFDA
:1041D0002285EFF01FE1C1B7832509000346D9FF0F
:1041E0002285EFF01F8E45BF0244924B224BB24A0C
:1041F000424AD2496249F2449250130181028280BC
:104200001305000681456FF0AF9E611106C23705A8
:10421000F87F0345055989456308B5008545631A4C
:10422000B5001305100619A0130520068145EFF00F
:104230002F9C9240210182808280130530068145A7
:104240006FF00F9B1305400681456FF06F9A611167
:1042500006C23705F87F03452559418901E5130555
:10426000500619A0130560068145EFF06F98924043
:10427000210182801305700681456FF06F9721112F
:1042800006CA26C6B704F87F03C5345922C22144A2
:104290004AC4636CA418B74501000A059385C5B1EB
:1042A0002E950841028509459305000FEFD04FBABE
:1042B00013750504630BA0163715F87F0345657C5D
:1042C0006305A016EFF0DFF36DA03709F87F034513
:1042D0006959118911C9EFF05FF603556959C16534
:1042E000ED156D8D231BA958EF402076C14563075E
:1042F000B500EF4080758D456319B5003725F87F0F
:1043000003258581E54563F6A506EF4000749545D4
:104310006367B500EF406073A545636CB504EF407B
:10432000C072E1456363B510EF402072F54563F25A
:10433000A504E5A87945B705F87F0D4623A6A56233
:10434000A389C458DDA03705F87F0325C56271ED48
:1043500011451DA03705F87F0345055979C5EFF0D4
:10436000DFEA01A83705F87F034515595DCDEFF069
:104370007FED038534590505A389A4587DA0370531
:10438000F87F0345255905894DC11D45F5B7EFF067
:104390001FEC038534590505A389A4583709F87F14
:1043A0000355695959C19375050485C5B705F87F4B
:1043B00083C52559858981E9EFF0DFEB03556959FC
:1043C0009945A389B458C1659385F5FB6D8D231B71
:1043D000A95893750538A1C5B704F87F03C52459BA
:1043E0009375450091E5098905E11305900639A803
:1043F0001305A0068145EFE0BFFF03C524591375DF
:10440000B50F2389A45831A0130580068145EFE03C
:104410003FFE031569591375F5C7231BA958C165DC
:10442000938505FC6D8D231BA958B704F87F83C5C0
:104430005459638B850205456388A5041146638042
:10444000C50A6367B00E09459305000FEFD04FA072
:104450001375050471CD3715F87F0345657C69C96F
:104460000385545905058DA83705F87F835565598F
:104470000966130606C06D8E45CE39661306F63FF3
:10448000F18D231BB5586DA03709F87F13056959C5
:1044900003451500418909CD1305D0068145EFE09C
:1044A0003FF503556959BD65FD156D8D231BA95851
:1044B000EF80D06AC1456300B502EF80306A8D4558
:1044C000630BB500EF809069F5456306B500EF809A
:1044D000F068631F85041145A38AA45891A8B70505
:1044E000F87F83C54559A9C509466387C500639A06
:1044F000A5001305B00619A01305C0068145EFE01D
:104500003FEF3709F87F1305695903451500137507
:10451000050409CD1305F0068145EFE07FED035555
:104520006959B165FD156D8D231BA958A38A84585F
:104530003704F87F13056459034515001375050208
:1045400009CD1305E0068145EFE09FEA0355645964
:10455000B965FD156D8D231BA45812442249B24440
:10456000D24061016FF0DFBD3705F87F0345356349
:104570009375250195C1B705F87F03864568937645
:1045800025001365160001462382A568138545683A
:10459000638CC602894515A8B705F87F03C6456830
:1045A0009376C500B9C609811345F5FF1366160059
:1045B0009386456805892382C568C8C63705F87F94
:1045C000032545638D6501A88D454CC53705F87FEA
:1045D00003254563856585056365B5021305F00F01
:1045E000B705F87F3706F87F238CA562232E066275
:1045F00082801375E60F1386456891462382A5686D
:1046000054C682803D7106CE22C22544E9452285EA
:1046100026CA4AC84EC652C4EFD08F830149937947
:10462000F50FCA8421A893058A002285EFD04F8216
:1046300093153A003315B500AA940509137AF90FBA
:10464000E3633AFF99C83705F87FB705F87F232A57
:10465000956223A40568EFF03FF1EF10E0173705EE
:10466000F87F232E05621244224AB2494249D244BD
:10467000F240056182803D7106CE26CA4AC84EC608
:1046800052C422C23704F87FB704F87F835504640C
:1046900003D52464A5C51DE9035504648945631E3B
:1046A000B500B705F87F3705F87F03A645630355C6
:1046B00045646376A600014631A0014501A803A622
:1046C0004563098E23AAC5622391A464B705F87FC8
:1046D00093854568D04183560464A1471387F6FF4C
:1046E000AA8663E3A700BE863387E6026308E60076
:1046F000035604647D163306D602D0C101E9835502
:10470000046405466394C500014529A0A14563E3FF
:10471000A5002E85370AF87F83454A6813094A6841
:1047200085892304A90099ED3705F87F0345356392
:10473000058909E93705F87F8345456993B5150073
:10474000230AB5688549EF10E00FE30E35FF0345F6
:104750004A68058919ED3705F87F034535630589F2
:1047600009E93705F87F8345456993B51500230AA4
:10477000B56803D5246409E5035504646302350371
:104780003705F87F03264563834589006374B600C7
:10479000814529A003264563B305B640232AB562A7
:1047A0003705F87F0325456301E9EF10C01E094571
:1047B000B705F87F2383A5641244224AB2494249CF
:1047C000D244F240056182807D7106C622C237055F
:1047D0000D80414460DD0545A545EFC07FE71375B9
:1047E0008503631785004545B7050D8023A4A508FB
:1047F0001244B2404161828037050D809305000963
:104800006CDD828037050D80C1456CDD8280370507
:10481000F87FB705F87F3706F87FB706F87F3707C8
:10482000F87FB707F87F3708F87FB708F87FB70237
:10483000F87F3703F87FB703F87F2314056423AEAE
:10484000056223260664238806642319076423AAC5
:104850000764231C08642390086423AA0262230CC3
:1048600003622383036482803706F87F8305050093
:104870001306E6152305B60083051500A305B6004B
:10488000830525002306B60003053500A306A60010
:104890008280611109459305A00F06C2EFC05FDB5E
:1048A000B705F87F238DA5649240210182806111B4
:1048B00009459305F00F06C2EFC09FD9B705F87FF1
:1048C000A38DA5649240210182807D7113050003B0
:1048D0009305001406C626C222C0EFC07FD7137509
:1048E000050209ED1305000393050014EFC05FD620
:1048F00013650502B705348023A0A55013040003F7
:10490000930540142285EFC0BFD4B705F87F238EEE
:10491000A5649384C5659305C0142285EFC05FD359
:10492000A380A40002449244B240416182807D7120
:1049300021459305006006C626C222C0EFC05FD1A4
:104940001375050201ED214593050060EFC05FD0AE
:1049500013650502B7250C8023A0A580214493058B
:1049600010602285EFC0DFCEB705F87F238FA564E6
:104970009384E565930530602285EFC07FCDA380E9
:10498000A40002449244B24041618280211106CACF
:1049900022C64000B7050D80214689462285EFD00A
:1049A0004FF203085400834844002208336818017A
:1049B00083087400830734008342A1000347240066
:1049C000A208B705F87FB3E8580093928700030563
:1049D00041001386056683061400B3E2E2002380DB
:1049E000A566A300D6002301E600A301F60023126A
:1049F000560023130601231416013244D2406101EC
:104A0000828021113705F87F06CA26C69304056601
:104A100083C5340022C03D444AC44EC2638285042B
:104A20000945638AA5060D456386A5080549639671
:104A30002527B709F87F1384A96613053004A285DA
:104A4000EFE09FC151CD13053004A285EFE05F9ADE
:104A50004DE103D5A966B705F87F9385157A79A04E
:104A600003D58400930510056363B5002E85B72632
:104A7000F87F83C616873706F87F8D453707F87F9E
:104A8000898A2316A6663705F87F232EB762B1E61A
:104A9000230A056619A483D58400494663E3C5004B
:104AA000B2853706F87FB706F87F2316B66623AEC1
:104AB000A662E5A203C524001D49636BA904B7459E
:104AC00001000A05938505B42E950841028583D51A
:104AD00084001145E3E7A5FCA9A0230AB56675AAE1
:104AE00003D5A966B715F87F9385157A2E95EFF053
:104AF000BFD703D58400C9456363B5002E85B705CC
:104B0000F87F3706F87F2396A566232E266371A2C9
:104B10009305E00E6313B51883D584004945E3E29D
:104B2000A5F8AA85BDBF3705F87F1305157A3709A3
:104B3000F87FB709F87F2328A9669385A96613052E
:104B40000004EFE0FF8A71C903D58400C94563639F
:104B5000B5002E85B705F87F154615AA3705F87FED
:104B60001305157A3704F87F3709F87F2328A466E0
:104B70009305A96613051004EFE09F8771C503D55F
:104B800084009305C0036363B5002E85B705F87FE5
:104B90001946F5A83705F87F1305157A3704F87F0D
:104BA000B709F87F2328A4669385A9661305200416
:104BB000EFE01F8445CD03D58400E945E370B5F4EB
:104BC0003DBF03D58400930500036363B5002E85C4
:104BD000B705F87F214665A803D5840093058004B6
:104BE0006363B5002E85B705F87F25464DA003D534
:104BF0008400930580046363B5002E85B705F87FB4
:104C0000294671A003D58400930500036363B500B2
:104C10002E85B705F87F2D469DA80325096783D506
:104C2000A966AA952328B96603D5840083C5050023
:104C30006363B5002E85B705F87F3706F87F2396A6
:104C4000A566232E866291A8032504678355A9666D
:104C5000AA952328B46603D5840083C50500636341
:104C6000B5002E85B705F87F414615A003250467DA
:104C700083D5A966AA952328B46603D5840083C585
:104C800005006363B5002E85B705F87F4546B70676
:104C9000F87F2396A56623AEC66202449249224954
:104CA000B244D240610182803145B705F87F23AE1E
:104CB000A56282803545B705F87F23AEA562828064
:104CC0003945B705F87F23AEA56282803705F87FA6
:104CD00003454566B7050D8013060008A8D9F0D135
:104CE0008280611106C23705F87F03060566130549
:104CF000056683451500634406022D466382C5049C
:104D00002546638CC50415466399C50603454500D1
:104D1000B7050D8013060008A8D9F0D1B9A813D59E
:104D20001500FE054D8D29C195456301B5049145DA
:104D30006300B5048D456312B504EFF09FCC35A830
:104D4000830545003706F87F03056500B706F87F41
:104D5000A308B6622389A6620DA003054500B70526
:104D6000F87F2388A56211A8314521A0394511A0FB
:104D70003545B705F87F23AEA562924021018280B8
:104D80007D7106C63705F87F834505661306000466
:104D900022C2638BC5041306100C6381C50C130675
:104DA000000C639BC5241305056683451500694403
:104DB000F9156363B424374601008A05130686B8E3
:104DC000B2958C418285834525001146E9156365BE
:104DD000B62203156500B705F87F2390A564EFF0B0
:104DE0009F8913052002E9A29305056603966500D5
:104DF0003705F87F2310C564094683C6150063870D
:104E0000C6080546639AC61E8356056495E2B70632
:104E1000F87F7947B707F87F3708F87FB708F87F3A
:104E200023AEE762A3890662230CC862239108645B
:104E30000355056411C57D453706F87F232EA6620C
:104E400003C525009145691563E0A50AB745010032
:104E50000A05938545B72E95084102851305056619
:104E60008355650015466399C5180355850093055C
:104E7000E0086363B5002E85B705F87F5146B70695
:104E8000F87F2396A56623AEC662BDA203560564CD
:104E90001DE23706F87F8346366313071002858AC2
:104EA000B707F87F0548B708F87FA309D66223AE95
:104EB000E762238C086383C525001146E915636505
:104EC000B602374601008A05130606B6B2958C4134
:104ED0008285035505646361A0123705F87F830559
:104EE000356393E5250039A23705F87FB705F87FCC
:104EF000232E0562238C056201A2130500024DA832
:104F00003705F87F03059553B705F87F5946B7066F
:104F1000F87F238BA56685BFEFF07FA1754549A873
:104F20003705F87F0305A553B705F87F5D46B7063B
:104F3000F87FA38BA56681BF835565001146639DED
:104F4000C50A03558500930580026363B5002E856D
:104F5000B705F87F4D4625B73705F87FD5453706A5
:104F6000F87FA30A0566232EB66279A0EFF07F9240
:104F70003705F87F232E856241A013051004B7057D
:104F8000F87F6146B706F87F238CA566EDBD130553
:104F90000003B705F87F6546B706F87FA38CA566C2
:104FA000DDB5EFF0DF906D4521A0EFF01F92714568
:104FB000B705F87F23AEA56281A0035505640DED0A
:104FC0003705F87F8305356393E5450025A0035534
:104FD00005641DE13705F87F8305356393E585009A
:104FE00011A80355056409E93705F87F8305356382
:104FF00093E50501A309B5621244B2404161828084
:10500000611106C2EFF09F983705F87F03450566EA
:1050100093050004137505066306B50011E5EFF06E
:105020005FCC19A0EFF0DFD59240210182803D7165
:1050300006CE22C22544E945228526CA4AC84EC664
:1050400052C4EFC0EFE001499379F50FCA8421A85B
:1050500093058A002285EFC0AFDF93153A00331520
:10506000B500AA940509137AF90FE3633AFF99CCC6
:105070003705F87F232A9562EFF00FCF3705F87FC9
:105080008305456893E525002302B5680544EF10C4
:10509000600BE30E85FE3705F87F232E0562124470
:1050A000224AB2494249D244F2400561828021112C
:1050B0002545E94506CA26C64AC44EC222C0EFC0ED
:1050C0002FD93709F87F835529653706F87F1306EE
:1050D00086692E961374F50F37050D80930505022A
:1050E000894632852286EFC0DFFD3705F87F0355FC
:1050F00005648544631995003705F87F8315256499
:10510000A2952311B56403152965B709F87F83A516
:1051100049652295A2951376F5032319A96423AA5C
:10512000B96439E63704F87F03558465B705F87F1D
:105130001A059385456813060004C8C12384C50079
:10514000EF10C00BE30E95FE9375F50F1305F00FEE
:105150006396A500B705F87F238CA56203158465C7
:1051600083A549650505231CA46401452319096429
:105170003704F87F032644636391C50A1375F5036A
:105180000DCDB705F87F83D585653706F87F9A057D
:10519000130646684CC22304A600EF102006E30E57
:1051A00095FE9375F50F1305F00F6396A500B705EF
:1051B000F87F238CA56223190964EF104039E30EB0
:1051C00095FE9375F50F1305F00F6396A500B705CF
:1051D000F87F238CA562EF10803AE30E95FE370529
:1051E000F87FB705F87F231C05642383956423AA01
:1051F0000964232A04623705F87F03454568B7052B
:10520000F87F058923AE056209E93705F87F830534
:10521000356393E51500A309B5620244924922491A
:10522000B244D24061018280611106C23705F87F25
:105230000325C56393051002630BB500FD45630BA1
:10524000B500F945631AB500EFF07FDE31A0EFF04D
:105250006FBB19A0EFF0BFE59240210182807D7104
:1052600006C626C222C02E84B7040D80AA851385E7
:10527000040485462286EFC0DFE4E0D40244924471
:10528000B240416182807D7106C622C23704F87F38
:105290000325C463930510027D1563EEA5223746EE
:1052A00001000A05130646BF32951041B705F87F85
:1052B0001385452289450286B705F87F3705F87FB3
:1052C00083D58564032505678E05E9AA3705F87F30
:1052D00003558564B705F87F0E059385E515D9A2BA
:1052E0003705F87F03558564B705F87F0E0593856C
:1052F00005174DAA3705F87F834545673705F87FC1
:10530000035585640E05630BB018B705F87F9385C8
:10531000351D49AA3705F87F03558564B705F87F21
:105320000E0593850500BDAA3705F87F03558564F2
:10533000B705F87F0E0593854500ADA23705F87FC8
:1053400003558564B705F87F0E059385850199AAF5
:105350003705F87F03558564B705F87F0E059385FB
:10536000450589A23705F87F03558564B705F87FA1
:105370000E059385E5063DA23705F87F0355856444
:10538000B705F87F0E059385E50929AA3705F87F4B
:1053900003558564B705F87F0E059385650E19A240
:1053A0003705F87F03558564B705F87F0E059385AB
:1053B000E512CDA83705F87F1305056355A8370515
:1053C000F87F130515636DA03705F87F03558564D5
:1053D000B74501000E059385C5C7E9A03705F87FDD
:1053E00003558564B74501000E059385E5C85DA8A2
:1053F0003705F87F03558564B74501000E05938591
:1054000065CB4DA03705F87F1305556795A0370587
:10541000F87F13056567A9A83705F87F1305756739
:1054200081A83705F87F1305856799A03705F87FB0
:105430001305956735A83705F87F1305A5650DA8F1
:105440003705F87F1305B56525A03705F87F1305E7
:10545000C565B9A83705F87F1305E56591A8EF0084
:1054600000764DCD3705F87F230C05621305856363
:1054700085453DA83705F87F035585643706F87FD5
:10548000B705F87F0E0583D5256413068669329526
:10549000F1C12146636EB600B28519A8B705F87F41
:1054A000938525182E95B705F87F83D5C56685C5E4
:1054B0003706F87F83568664139736009307870074
:1054C00063FFF500998D23140664232E046293F57F
:1054D000F50FEFF0DFD81244B2404161828093852E
:1054E00016008326C4632314B66413062002A14564
:1054F000E39FC6FC3706F87F0356266469FA370631
:10550000F87F035606648546E313D6FC3706F87F1A
:1055100083164664A1062312D66455BF3706F87F6A
:10552000834586639306F00F13058663E382D5F403
:10553000B706F87F03C7666485456307B70003C7EE
:10554000666489476314F7020947230CE6622383E4
:105550000664B9BFB705F87F83D505640546638443
:10556000C500A145B1B79305001099B7230CB662E9
:1055700081B77D7106C622C23704F87F03450465F2
:105580009375150089C9EFF0BFA737050D808545D4
:105590006CD1034504659375250089C9EFF0DFC818
:1055A00037050D8089456CD1034504659375450029
:1055B00089C9EFF05FCD37050D8091456CD103456A
:1055C0000465218909C937050D80A1453706F87F93
:1055D0006CD1231406641244B240416182807D7113
:1055E00006C622C23704F87F0325C46493751500EC
:1055F00095E11375050415C52545E145EFC04F85B7
:10560000B705F87F1376F5002388A56419CEEFF06F
:105610005FF601A8EFF0AF9F0325C46479992326B4
:10562000A4641244B240416182800325C4641375AE
:10563000F5FBF5B761112545F94506C2EFC04F816D
:105640009375F50F37060D80937615002CDE89CA09
:10565000B705F87F03A6C5641366160023A6C564C4
:105660001375050409C93705F87F8325C56493E5DB
:1056700005042326B564924021018280611106C28F
:10568000EFF05FFB924021016FF07FF5611106C2E0
:105690003725F87F8345858085C11305858083453F
:1056A0009506898999E1684501E937050D809305DB
:1056B00000096CDDEFF09FFC924021018280000028
:1056C0003D7106CE4EC6B709F87F26CAAA8403C527
:1056D000196852C48945014A4AC856C222C0630BA0
:1056E000B50605446300850659E105499305300573
:1056F0004A85EFB0FFF513650502B70A058023A6BA
:10570000AA14EF10A007930540034A85EFB05FF499
:1057100081456385B4001365C50919A0137535F675
:1057200023A8AA0C930530034A85EFB07FF21365D6
:10573000450023A6AA0CEF0090750385196805059E
:10574000A380A968EF10000B05E50385196805051E
:10575000A380A968054593053005EFB07FEF137569
:10576000F5FDB705058023A6A514A380096852841A
:1057700022850244924A224AB2494249D244F24026
:1057800005618280211106CA26C6B704F87F83C549
:10579000246822C22A844AC4638A850215E4370930
:1057A00005801305B00A232CA90C05459305300389
:1057B000EFB01FEA136505042326A90CEF00B074AF
:1057C000EF001077EF00507923818468124422495A
:1057D000B244D240610182807D7106C622C201447A
:1057E0002285EFF03FFA22851244B2404161828067
:1057F0003705F87F130545684C4591CD0546638014
:10580000C5020D466381C50209466392C50248413F
:10581000B785030035A04841B715030015A04841DE
:10582000B745030031A84841B795030011A8B70553
:10583000F87F83C54569484199C1856511A0E56533
:105840002E958280211106CA26C6B704F87F03C5AB
:1058500004684AC401494EC222C019CD8545630A75
:10586000B50289456305B5088D45631DB51037053B
:10587000F87F0345C568D5A813050002EF00705BEB
:1058800003850468B705F87F0505A38A05682380AA
:10589000A468EFF0FFF53707F87F0347C7689375F3
:1058A000F5013706F87F930600028D8EA30BB668CC
:1058B0003A866363D700368681476313F7003686DE
:1058C000B706F87F0D8D238BC668EF00B0500545F5
:1058D00093053003EFB0DFD713652500B7050580CA
:1058E00023A6A50C0385046805052380A468054448
:1058F00095452285EFB0DFD51375050849C53704F6
:10590000F87F3706F87F03455469B705F87F0346EB
:105910007669938585692E9593152600370605804F
:1059200013060618B709F87FB29503C66969894658
:10593000EFC02FF93705F87F1306456883C56969FD
:105940004842830686003307B5003385B640830698
:10595000546983870468B6959386170058C2230458
:10596000A600A30AB4682380D4681375F50F09C58F
:1059700005442380846801A83705F87FA30A0568D9
:10598000238004684A842285024492492249B24411
:10599000D240610182803705F87F0346256885453E
:1059A0006304B6002301B56801458280211106CA4F
:1059B00026C6B704F87F03C504684AC4894501496F
:1059C0004EC222C06306B50685456300B50279E97B
:1059D000B705F87F1305000223AE0578EF00704588
:1059E0000385046805052380A4683705F87F03450F
:1059F000057A81456305B5003795030019A0378501
:105A00000300B705F87F83A5C5792E95EF00903C7C
:105A1000054593053003EFB0BFC313652500B705F7
:105A2000058023A6A50C0385046805052380A468CA
:105A3000054495452285EFB0BFC11375050825C5FE
:105A40003704F87F0325C479B705F87F9389157A61
:105A5000B70505804E959385051813060002894603
:105A6000EFC02FE60325C479B385A90003C605005E
:105A700011CA9306F00F631AD60083C5150063960A
:105A8000D50039A883C5150081CD130505029355AE
:105A9000C500232EA47889E505442380846821A0CD
:105AA000238004684A842285024492492249B244F0
:105AB000D24061018280211106CA26C6B704F87F50
:105AC00003C504684AC4894501494EC222C0630621
:105AD000B50685456300B50271E9B705F87F130582
:105AE000000223AE0578EF00D03403850468050575
:105AF0002380A4683705F87F0345057A814563054F
:105B0000B5003795030019A037850300B705F87F66
:105B100083A5C5792E95EF00F02B0545930530033D
:105B2000EFB01FB313652500B705058023A6A50CAC
:105B30000385046805052380A468054495452285EE
:105B4000EFB01FB1137505083DC1B719F87F138475
:105B5000197A370505809305051813060002894652
:105B60002285EFC00FD68385197A0345140093066A
:105B7000F00F3376B5006309D602C98D93F5F50FA2
:105B800085C5930530046301B5023705F87F832589
:105B9000C5799385050213D6C500232EB57809E68D
:105BA00005442380846821A0238004684A842285D8
:105BB000024492492249B244D240610182803715A1
:105BC000F87F0345157C134585003335A00082809E
:105BD0003715F87F8345257C37060680BD8923016C
:105BE000B57C232EB63C82803715F87F8345257C13
:105BF0003706068093F5F50B2301B57C232EB63CC2
:105C00008280797106D626D222C2AE842A8431459A
:105C1000B74501003305A402938545DA2E954AD095
:105C200052CC56CA5EC662C403290500834A4500A9
:105C3000035C6500835B8500034AA5004ECE5AC80D
:105C4000EF00903191C81305805F335585000589B9
:105C500081456303B5009D4A0544930900042285EC
:105C6000CE85EFB0FF9E1375F5FC93F504034D8DC3
:105C7000370B05802320AB104A85EF00B015139534
:105C80004B00EF00101B13558C009375FC0F232263
:105C9000AB002324BB008D452285EFB07F9B93D5BD
:105CA0008B004199BD894D8D2326AB002285CE8581
:105CB000EFB01F9A93D59B005D99A1894D8D93F507
:105CC000FB0F2320AB102328BB0081452285EFB0BA
:105CD0003F9893954A001375F5F093F5050F4D8D98
:105CE0002320AB00930530032285EFB07F96136528
:105CF000250095442326AB0C2285A685EFB05F9541
:105D000093151A00759989894D8D232AAB00228538
:105D1000A685EFB0FF9313651500232AAB0012444C
:105D2000224CB24B424BD24A624AF2490259925437
:105D3000B25045618280211106CA22C285452A845B
:105D400026C64AC463EB850005459545EFB05F90D4
:105D50001375050439E5894465A805459545EFB0F7
:105D60003F8F13750508894445C5054995454A8502
:105D7000EFB01F8E418949CD1305F4FF1374F50F61
:105D800095454A85EFB0DF8C3716F87F8306367C61
:105D9000137505020147B31589006300E504CD8E34
:105DA00081A03715F87F3716F87F8345357C830649
:105DB000267C93E5150093E6160037070980A301BA
:105DC000B57C2301D67C232EB73CB705068003455E
:105DD000267C23AEA53C814425A813C7F5FFF98E88
:105DE000A301D67C3716F87F0307267C93F6F60FBF
:105DF000D98D3707098015812301B67C232ED73C26
:105E0000934415008345267C37060680232EB63C36
:105E1000268512442249B244D240610182803D71FC
:105E200006CE26CAB714F87F83C5147C4AC821451C
:105E300001494EC652C422C2636CB52E37460100DA
:105E40008A05130646D4B2958C418285B709058030
:105E50001145054423ACA90C930530032285EFB00E
:105E60002FFF1365050423A6A90CEF00D009EF004E
:105E7000300CEF00700E930500042285EFB04FFD4B
:105E80001365050823A0A910EF00100D93058003EA
:105E90002285EFB0EFFB23A8A90C1305F00F838533
:105EA000147C3716F87F85052302A67CA380B47C7A
:105EB00005449305F0032285EFB08FF90D89631C2B
:105EC000850E0145F5A8EFF07FAE636CA022054575
:105ED000B715F87F01442383A57C2285A285EFD0E6
:105EE0002FD13705F87F954523050556A380B47C4F
:105EF00089A4370AF87F03450A7A8549630A350180
:105F0000636CA01225458145EFF0BFCF23003A7B9B
:105F1000054495452285EFB0AFF313750508630A74
:105F2000A020054495452285EFB08FF24189630298
:105F3000A02005459545EFB0AFF113750502636BE1
:105F4000A00E23000A7AC5A205442285EFF04FF780
:105F50006361A01E13050002EF00A06D0385147C91
:105F6000930515000905A380B47CB705F87F83C6A7
:105F7000256805466384C6002381C568A380A47C88
:105F80003715F87FB715F87F0345457C83C5257C19
:105F90006300B51A93C5F5FF6D8DB715F87F4A8478
:105FA000A382A57C6307A0180145EFF0AFFD09456A
:105FB000A380A47CB9A23705F87F230A85682285CF
:105FC000EFF07FD70385147C0505A380A47CB7156B
:105FD000F87F3715F87F8385257C0305457C93C5BD
:105FE000F5FF6D8DB715F87F13762500A382A57C8C
:105FF00005EA1375F50F937545008DE593758500DA
:1060000085E5937505019DE19375050295E193750D
:106010000504B5E5137505086309A01021458DA099
:106020000945B9A80D45A9A8114599A8154589A8FC
:106030001945B9A003450A7A6307A00E6315350117
:1060400009452300AA7A371AF87F03456A7C63184A
:106050003501EFF05FA64E84636DA00CE9A0EFF070
:10606000FF944E8479E5894501452303BA7CAA85CE
:10607000EFD00FB83705F87F230505566DA01D45F5
:106080008145EFF01FB80385147C0505A380A47C2F
:106090003714F87F0345547C937525008DE593757F
:1060A0004500A1E1937585009DED93750501A1E182
:1060B000937505029DED9375050495ED137505081F
:1060C00039C1214515A809442285EFF0DFC6630ACE
:1060D00085023715F87F0345357C098919E5154593
:1060E000B1A00D4511A8114501A8114581A0154584
:1060F00021A0194511A01D45EFF0FFC38945631488
:10610000B50005443DA0B715F87F3715F87F8385A6
:10611000257C0305457C93C5F5FF6D8D9375F50FC3
:10612000A302A47C99C1094511A01945A380A47CB0
:106130004A8422851244224AB2494249D244F2405A
:1061400005618280211106CA26C6B704F87F03C5FF
:1061500004684AC44EC21149814922C06360A9083B
:10616000B74501000A05938585D62E95084102851D
:1061700001442285EFF00FE12285EFF06FD439E979
:106180000385046805052380A468EF00A066054424
:1061900039E53705F87F03454568058929E937055D
:1061A000F87F0345456939C50385046805052380E3
:1061B000A46801442285EF00006809ED238004688B
:1061C00039A805442285EF00006711E931A0EF00EE
:1061D000A07519C1054421A0238004684E8422853E
:1061E000024492492249B244D24061018280238014
:1061F0002469F5B70D452380A468D5B7797106D613
:1062000056CAB70AF87F03C50A6852CC5AC8114B60
:10621000014A26D24AD04ECE5EC662C422C2636212
:10622000AB16B74501000A059385C5D72E950841E1
:1062300002853715F87F8545A303057C2380BA685E
:10624000EFF00FDB3706F87F930B46689375F50187
:106250009304000203C68B00B387B44081462687AF
:106260006383D7003E8732846363F6003A84631306
:10627000D6003A840D8DEF00E0352685EF00603BB7
:10628000370C058013094C0485499305F00F4A85A6
:106290002686CE86EFB05FE8B714F87F03C5747C1E
:1062A000B705F87F93858569AA954A852286CE86AB
:1062B000EFB03FE103A54B0083858B000386747C20
:1062C0002295818D229623A2AB002384BB00A38359
:1062D000C47CEF00A04A930530034E85EFB04FB762
:1062E000136515002326AC0CEF00603A03850A689D
:1062F00005052380AA68EF00E04F19C1054A51A0A7
:106300003705F87F03454568098901E523806A69F7
:106310008DA803850A6805052380AA6805459305AD
:106320003003EFB0EFB21365250037040580232654
:10633000A40CEF00604213054404930504181306EF
:106340000008EFD0E03811C93715F87F23800A68BC
:10635000A303057C130AF00F2DA003850A68050529
:106360002380AA683705F87F0345C56809C5054A33
:1063700023804A6939A03715F87FA303057C238061
:106380000A6813158A011244224CB24B424BD24A7E
:10639000624AF24902599254B25061854561828045
:1063A0003D7106CE4AC83709F87F034509684EC6D5
:1063B0009145814926CA52C422C263E7A50EB7455A
:1063C00001000A05938505D92E95084102853705F8
:1063D000F87F0345456919C1014511A0054593059D
:1063E0000002EFF01F820305096805052300A96874
:1063F000054495452285EFB0AFA541895DC50545AA
:106400009545EFB0EFA41375050201E51304F00FF5
:1064100069A80305096805052300A968EF00004C79
:106420000544630485083705F87F034545693DE960
:106430000305096805052300A9683705040001154F
:10644000EF00401913050002EF00A01E370A058077
:106450001304F00F854413054A044146A285A6861D
:10646000EFB09FCB13058A083D46A285A68623225E
:106470000A08EFB07FCAEF0060309305300326852D
:10648000EFB00F9D136515002326AA0CEF00202006
:106490000305096805052300A968EF00A03519C1A7
:1064A000054421A0230009684E8413158401124479
:1064B000224AB2494249D244F24061850561828054
:1064C000211106CA4EC2B709F87F83C509684AC4BC
:1064D0000545014926C622C0638DA502B9EDB70561
:1064E000F87F83A505690D466387C5006387A5000E
:1064F00099E5194531A0254521A0214511A009455F
:1065000093050002EFF0EFEF03850968050523808E
:10651000A968054495442285A685EFB06F9341890B
:106520007DD905459545EFB0AF921375050201E59C
:106530001309F00F19A0238009681315890102447B
:1065400092492249B244D240618561018280611141
:1065500006C23705F87F83454568858981E5EFF0F8
:106560003FE419A81305456848458D4563E5A50036
:10657000EFF01FF511A00145924021018280211109
:1065800006CA26C6B704F87F03C504684AC422C2F7
:1065900005440149630C85000DE52285EFF04F921B
:1065A00015E10385046805052380A4683705F87F95
:1065B0000346256885456304B6002301B56823803A
:1065C00004684A84228512442249B244D2406101BF
:1065D00082800000211106CA26C64AC485440D499E
:1065E00022C02A842685CA854EC2EFB06F861375F5
:1065F000F5F9B709058023A6A9002685CA85EFB05D
:106600002F859355B40093F505064D8D9355840061
:1066100093F5F50F1376F40F23A6A90023AEB90264
:1066200023A0C904024492492249B244D2406101E4
:106630008280211106CA26C622C005448D444AC460
:106640001309F5FF2285A6854EC2EFB06F803D99F4
:10665000B709058023A6A9002285A685EFA05FFFC4
:106660009355C900C1894D8D9355890093F5F50F58
:106670001376F90F23A6A90023A2B90C23A4C90CF1
:10668000024492492249B244D240610182806111A0
:1066900006C2EF008001058911E50D45B715F87FA9
:1066A00023A4A57C9240210182807D7106C626C26A
:1066B00022C08144294421A0EFA09FBD850413F589
:1066C000F40FE36B85FE054593050004EFA05FF82A
:1066D00013650508B7050580814423A0A51021A0F6
:1066E000EFA01FBB850413F5F40FE36B85FE054592
:1066F00093058003EFA0DFF502449244B240137586
:10670000F50F416182807D7106C622C2EFF03FF82D
:106710003714F87F39A0EFF05FF9058919C12324F8
:10672000047C0325847C65F91244B2404161828077
:10673000611106C2EFF07FF793751500E5FD9240F9
:1067400021018280611106C2EFF03FF693752500AA
:10675000E5DD9240210182807D7106C626C222C0FD
:10676000054495442285A685EFA09FEE1375050884
:1067700075D902449244B240416182807D7106C65F
:1067800022C2EFF07FFD370405801945232CA40CAD
:10679000054593053003EFA0BFEB136505042326E1
:1067A000A40CEFF05FF6EFF0BFF8EFF0BFF9124482
:1067B000B24041616FF05FFA7D7106C626C222C009
:1067C0002E84AA84EFF09FFB2685EFF0BFE0B7048C
:1067D000058005459305300323AE840CEFA05FE7E9
:1067E0001365050223A6A40C02449244B240416101
:1067F0006FF0FFE97D7106C622C23714F87F0325CA
:10680000847C09C9EFF07FEA058919E1054439A8BC
:106810002324047C054495452285EFA07FE313756E
:10682000050809C5EFF07FE81374150022851244AE
:10683000B240416182807D7106C626C2B714F87FDE
:1068400083C5C47C22C001449DC10946638BC50435
:106850000546639FC506B715F87F83C5D57C0DC176
:1068600013953500B7450100938585E205A0B7155E
:10687000F87F0546A386057C81452386C47C6DF19F
:1068800013953500B7450100938585E7AA958841A2
:1068900083C54500EFF05FF20385C47C05052386C0
:1068A000A47CEFF03FF519C105441DA03715F87F12
:1068B0008305D57CA546850513F6F50FA306B57CA3
:1068C00063E6C60005442386847C19A02386047CE5
:1068D000228502449244B24041618280211106CA5D
:1068E00026C6B714F87F03C5C47C4AC422C2054437
:1068F0000149630E85000DE137F5030093050002A1
:10690000EFF09FEB0385C47C05052386A47CEFF0A4
:106910007FEE01E52386047C4A84228512442249C5
:10692000B244D240610182807D7106C626C2B7148E
:10693000F87F03C5C47C22C0014401CD8945630DA5
:10694000B50685456317B50A3715F87F0325057D1C
:1069500099A83705F87F032505698545630BB500C0
:106960000DE10D453716F87FA306A67C3715030009
:106970002DA00D453716F87FA306A67C37450300EA
:1069800029A83716F87F8D46A306B67C6305D50087
:106990003785030019A0379503003716F87F2328A1
:1069A000A67C2386B47C93050002EFF0FFE003850C
:1069B000C47C05052386A47CEFF0DFE319C1054400
:1069C0000DA83715F87F8305D57CFD1513F6F50F57
:1069D000A306B57C09CE3715F87F8325057D0566AE
:1069E000B29505442328B57C2386847C19A0238690
:1069F000047C228502449244B240416182800000BE
:106A0000130181FC06DA4AD44ED252D03689B289BB
:106A100001462A8A26D656CE5ACC5ECA62C866C6B7
:106A20006AC46EC222C06304CA00154411A009449E
:106A3000B70B0480131B040113854B145A952320B4
:106A4000350113858B14F9465A954E8663E3D900B8
:106A500036868544A686EFB0CFE61305400AB725F3
:106A6000F87F3305AA0293858580B38DA500130DA9
:106A7000800C138C4D02130A100823A2AD0322854B
:106A8000D285EFA0FFBC1375050401C503250C00DA
:106A90007DF513850B04330AAB00930A0007930CB2
:106AA000F00F23200C0023205A01638E990103C5A7
:106AB0005D0589456305B5001305000319A013059D
:106AC00000023369250113850B145A9523202501F3
:106AD00041492320AC012285CA85EFA07FB71375F9
:106AE000050709E903250C007DF523200C0093041C
:106AF000B00F15A8C145228523200C00EFA05FB57B
:106B0000137505040DE1C1452285EFA07FB413750F
:106B10000502E68409E9C1452285EFA07FB36E0531
:106B20007D859374E5FF23205A0113958401024467
:106B3000924D224DB24C424CD24B624BF24A025A19
:106B400092592259B254D250618513018103828037
:106B50007D7106C63725F87F0345A58022C009440C
:106B600026C293741500F5452285EFA07FAE0D89EE
:106B700085E0914485452684630AB5060944F545B8
:106B80002285EFA0FFAC0D89631785042144B9A8C5
:106B90008545630BB5000945F545EFA07FAB0D8931
:106BA00013452500133415000945F545EFA05FAAEC
:106BB000318991456315B50013640402BDA00945F0
:106BC000F545EFA0FFA83189A1456314B500136412
:106BD00004012285A9A80945F545EFA07FA70D89E5
:106BE0008D456304B500014411A031440945F545C4
:106BF000EFA01FA63189631595001364040435A026
:106C00000945F545EFA0DFA43189A1456315B5001D
:106C1000136404F819A80945F545EFA07FA331894D
:106C2000B1456314B500136404FC1375F40F0244FA
:106C30009244B240416182807D7106C63725F87F5B
:106C40000345458622C20544630285020945930532
:106C5000E008EFA0FF9F1375050809E92D4593058E
:106C6000C00CEFA0FF9E15811374150022851244FD
:106C7000B24041618280211106CA22C209449305B3
:106C8000C00F228526C64AC4EFA09F9C13658500CD
:106C9000370906802328A93EEFF09FEB2326A93E63
:106CA0009305D00F2285EFA0BF9A21891DE10944E9
:106CB0009304E00C2285A685EFA09F9913654500FB
:106CC000232CA9322285A685EFA09F986D99232CAD
:106CD000A93212442249B244D2406101828021117A
:106CE00009459305800F06CA26C64AC422C2EFA0F2
:106CF0003F96B704F87F83C544520581058985898D
:106D00006309B50609449305C00F2285EFA05F947F
:106D100013654500370906802328A93E9305800F97
:106D200003C54452937415002285EFA07F928145DC
:106D30006385B4001365250011A075992320A93E31
:106D40009305D00F2285EFA0BF9011891DE1094462
:106D50009304E00C2285A685EFA09F8F1365450064
:106D6000232CA9322285A685EFA09F8E6D99232C16
:106D7000A93212442249B244D24061018280611199
:106D800009459305100F06C2EFA09F8C9375B5FFC0
:106D9000370606802322B63C0145924021016F3020
:106DA00080312111370506809305000706CA26C6E3
:106DB0004AC44EC222C02CC1B725F87F83C5D585F1
:106DC00009466385C5009305500319A09305500239
:106DD0009309800C0944C14405492320B514228538
:106DE000A685EFA0FF861375050701E94A85EFA088
:106DF000FF8413F5F90FFD197DF1024492492249F0
:106E0000B244D2400545610182807D7106C622C22E
:106E10002A840945E945EFA0BF838145137505FB29
:106E20006304B400954511A0A945C98D37060680B5
:106E30002CD605451244B24041616FA03F803D71A0
:106E40000945C14506CE26CA4AC84EC652C422C20A
:106E5000EFA01F801375050819CD0144930500406C
:106E60002285EF20106D2285EFA05FFA1305000840
:106E7000B7050680A8C10945C545EFA06FFD058986
:106E80006360A0260945C145EFA08FFC318915C17B
:106E90000945C145EFA0CFFBB725F87F3726F87F1E
:106EA000854637070680B147238DA59E2302D686E7
:106EB0003CC30945C545EFA0AFF913750508630646
:106EC000A01EB70906809304000809459305800CAD
:106ED00023A29904EFA0CFF71375050815C1094443
:106EE0009305A00C2285EFA0AFF61375050809C91C
:106EF0003705F87FB7050680A304855623A495328D
:106F000009459305800CEFA0AFF4137505040DC17E
:106F100009459305A00CEFA0AFF31375050409C94B
:106F2000EFB08FB613050004B705068023A4A53281
:106F300009459305800CEFA0AFF11375050231C12F
:106F400009459305A00CEFA0AFF01375050215C914
:106F50002D44930450062285A685EFA06FEF13659C
:106F6000050237090F80232AA9182285A685EFA0DC
:106F70002FEE1375F5FD93050002232AA91823A40B
:106F8000B93209459305800CEFA08FEC21891DCD06
:106F900009459305A00CEFA0AFEB218905C92D444D
:106FA000930450062285A685EFA08FEA136585001D
:106FB00037090F80232AA9182285A685EFA04FE95B
:106FC0005D99A145232AA91823A4B932094593053F
:106FD000800CEFA0EFE711891DCD09459305A00CAA
:106FE000EFA00FE7118905C92D44930450062285AF
:106FF000A685EFA0EFE51365450037090F80232A2A
:10700000A9182285A685EFA0AFE46D999145232AA2
:10701000A91823A4B93209459305800CEFA04FE3CA
:1070200009891DCD09449305A00C2285EFA04FE2EC
:1070300009891DC5AD44130950062685CA85EFA0F0
:107040002FE113652500370A0F80232AAA18268509
:10705000CA85EFA0EFDF7599232AAA1823A48932E5
:1070600009459305800CEFA0AFDE05891DCD0945CC
:107070009305A00CEFA0CFDD058905C92D4493042D
:1070800050062285A685EFA0AFDC136515003709F1
:107090000F80232AA9182285A685EFA06FDB799996
:1070A0008545232AA91823A4B9321305000A93059C
:1070B0004004EFA0EFD9058901CD1305000A93051F
:1070C0004004EFA0EFD87999B705A48023A8A510B4
:1070D0001244224AB2494249D244F24005618280B8
:1070E000EF10C06B2A843705F87F0319E55301457B
:1070F000AA85EFA05FD93725F87F9304858003C563
:1071000044090589E300A0D803C5C409E36CA0D6EF
:10711000EF10B013A9456367B500EF101013BD451C
:10712000E362B5D6EF107012930500026368B500F4
:10713000EF10B01193054002E366B5D46545330402
:10714000A4023309A902EF105010E945636FB5009E
:10715000EF10B00FC165FD153376B900E18DE3F393
:10716000C5D2F14563EAA50031BB41657D15B37514
:10717000A900618DE378B5D00545238EA408EF40C2
:10718000606A09B37D7106C63725F87F0345E58A35
:1071900026C222C0058909C915459305000FEFA035
:1071A0002FCB137505080DE51545F545EFA04FCA22
:1071B00091440D89854526846301B5081545F5453B
:1071C000EFA00FC90D898945631EB5002144B5A004
:1071D0001545F545EFA0CFC70D898545631EB50060
:1071E000094425A01545F545EFA08FC60D898D45AD
:1071F0006304B504014491A01545F545EFA04FC5C2
:107200000D8913452500133415001545F545EFA0EC
:107210002FC4318991456315B50013640402A9A8F0
:107220001545F545EFA0CFC23189A1456314B500DE
:1072300013640401228599A031441545F545EFA05A
:107240002FC13189631595001364040435A01545D9
:10725000F545EFA0EFBF3189A1456315B500136473
:1072600004F819A81545F545EFA08FBE3189B14541
:107270006314B500136404FC1375F40F02449244C4
:10728000B240416182807D7106C63725F87F034593
:10729000859022C205446302850215459305E008E6
:1072A000EFA00FBB1375050809E92D459305C00C28
:1072B000EFA00FBA15811374150022851244B24055
:1072C00041618280211106CA22C215449305C00F74
:1072D000228526C64AC4EFA0AFB7136585003709DB
:1072E00009802328A93EEFF0FFE92326A93E930554
:1072F000D00F2285EFA0CFB521891DE1154493045D
:10730000E00C2285A685EFA0AFB413654500232CC1
:10731000A9322285A685EFA0AFB36D99232CA9329F
:1073200012442249B244D2406101828021111545A4
:107330009305800F06CA26C64AC422C2EFA04FB1E9
:10734000B705F87F9384455283C56400058105899C
:1073500085896309B50615449305C00F2285EFA002
:107360002FAF13654500370909802328A93E9305EF
:10737000800F03C56400937415002285EFA04FAD04
:1073800081456385B4001365250011A075992320FC
:10739000A93E9305D00F2285EFA08FAB11891DE187
:1073A00015449304E00C2285A685EFA06FAA13650F
:1073B0004500232CA9322285A685EFA06FA96D99DF
:1073C000232CA93212442249B244D2406101828066
:1073D0002111370509809305000706CA26C64AC44D
:1073E0004EC222C02CC1B725F87F83C5159009462F
:1073F0006385C5009305500319A0930550029309B6
:10740000800C1544C14405492320B5142285A68566
:10741000EFA00FA41375050701E94A85EFA00FA29D
:1074200013F5F90FFD197DF1024492492249B24446
:10743000D2400545610182807D7106C622C0154497
:1074400026C2AA84E9452285EFA08FA08145137545
:1074500005FB6393B4002944B365850037060980B2
:107460002CD6054502449244B24041616FA00F9D65
:107470007D711545C14506C622C2EFA06F9D1375EB
:10748000050819CD0544930500402285EF20700AB8
:107490002285EFA0BF9713050008B7050980A8C192
:1074A0001545C145EFA0CF9A318915C11545C14594
:1074B000EFA00F9AB725F87F3726F87F8546370764
:1074C0000980B147A38DA59E2304D6903CC31545E2
:1074D000C145EFA0EF9705891DC137050980854596
:1074E0002CC13725F87F130485800345440905899D
:1074F00019C50345C40901E5EFF0DFC809C5124409
:10750000B24041618280EF50704A75D9EF10E0536C
:10751000A9456367B500EF104053BD45E361B5FE73
:10752000EF10A052930500026368B500EF10E05120
:1075300093054002E365B5FC0945230EA408EF401E
:10754000602E75BF7D7106C622C2EFA0EF958945FA
:107550006318B506EF509045B705F87F138465248E
:107560008345340005C513E58502B725F87F03C6BA
:10757000D585834524008546A301A4006319D6025E
:10758000BD891375E50F2301B4000DA893F5750FA0
:107590000945A301B4009305100FEFA06F8B9375FD
:1075A00005080345340089E91375F50D01A813E5B5
:1075B00005082301A40029A013650502A301A40066
:1075C0001244B240416182803705F87FB706F87FE8
:1075D00093057526030675261385362683472500F1
:1075E0000388250093F70708B3E707013708F87FFA
:1075F000034898240387150083C535001378480095
:10760000A381C626A300E5002301F500A301B50070
:107610006306000193E52500A301B5003715F87F47
:1076200081451305057F1146AE866FA0FFAEB705F5
:10763000F87F014593869528C16541770D46FD1574
:107640001307071089472A881DA0B3880601838283
:10765000180083C80800A202B3E81201B3F2B80010
:107660003383E2006364F300636850000908137811
:10767000F80FE37C06FDAA8833F5B800828061111B
:107680003725F87F06C2130585808345A506416628
:10769000A20513060680F18D13D68500A304B50656
:1076A0002305C506EFF0BFF8B715F87F239BA57E2D
:1076B000924021018280211106CA22C62A840345F4
:1076C0001400F945791563E2A50285453395A500B7
:1076D000B7050040938515046D8D01C91305200C75
:1076E000EF8060131305000231A01305400CEF80FA
:1076F00080124145EFC0EFBE03451400C14563123F
:10770000B5021305E014930580082AC42EC229454A
:107710004C000546EFA05FA2370534809305F003C7
:1077200005A01305401E930580082AC42EC22945D2
:107730004C000546EFA05FA037053480930500029A
:107740002328B5183244D240610182803D7106CEB3
:1077500022C22A840345040026CA85449356650044
:107760004AC84EC652C46381960289456382B602F6
:107770008D491376F501639F36019305F6FF8D461B
:1077800063F0D508054951A01375F503014979AB9C
:10779000014979AB7D1641450149636DC554B74632
:1077A00001000A06938686EC36961042028603454F
:1077B000140005491375050EB725F87F2300240131
:1077C000A300A4009389858003C5590523002401E3
:1077D0001345250013351500160513650508A3008C
:1077E000A40003C529009375250003C5590581C56B
:1077F0008945631EB53E854463079540914529A19F
:1078000095456303B600914501491375F50339ABFE
:107810000345140089441375050EB725F87F23002E
:107820009400A300A400138585808345550523009B
:107830009400054993C5250093B51500960593E579
:107840000508A300B400B705F87F83C5B527918963
:107850006302B04A83452500898991C503455505D2
:1078600089456319B5483709F87F930499281305AA
:10787000440011468146A685EFA0BF8403C51400CD
:107880008345992822054D8D8544630FA02A8145A3
:10789000130584001146AE86EFA01F884E8999A972
:1078A000034514008345040022054D8D83453400B3
:1078B00003462400A205D18DC205B3E6A5003965B3
:1078C00033F6A600218213D5860193D50601A300C5
:1078D000C4003726F87F23003401A301A40023014C
:1078E000B4001306868003475605B707FF00134709
:1078F0002700133717003607F58F370800FFB3F658
:1079000006015D8FD98E21670D07D98EA182A30153
:10791000A4002301B40023003401A300D400B7065F
:10792000F87F83C6B6278944918A05496304D03C11
:1079300083462600898A91C6034656058946631BFD
:10794000D63A220593F5F50F4D8DC165138605F0E6
:107950006302C53A938515F06312B532B705F87F17
:10796000130544009385052711468146EFA06FF566
:107970008544D9AA034514000549937975008944C3
:10798000639E29333705F87F0345B52711896307BF
:10799000A0323725F87F130A858003452A0009891C
:1079A00011C503455A058945631AB53003453400AE
:1079B0008345240022054D8DC165138605F06308BB
:1079C000C52C938515F06316B52C370514001306E6
:1079D00035302945A145EFA00FC103459A068544DE
:1079E00013652500A304AA06C1AC3725F87F9309C7
:1079F000858003C59906894409890549630CA02E31
:107A0000834514000345040013968500518D0346F9
:107A10003400834624002206558E4206518D396675
:107A2000698E9546418121822300D4002301A40060
:107A3000A300C4009D8903C65905A205134626006C
:107A4000133616003606D18D2166D18D416AA1818B
:107A500013061AF02300D4002301A400A300B400ED
:107A60006319C51E37051400130635302945A14595
:107A7000EFA06FB79145694681462285EFA0FF943C
:107A800003C5A90683C5990622054D8D93058ABFB6
:107A90006D8D93558500A384A906130500042385E5
:107AA000B906EFC00F840549C1AA834534000346D7
:107AB0002400A2054169D18D130619F06391C51206
:107AC000834514003726F87F93F5050E2300A400A4
:107AD00093098680A300B4003706F87F83C5590553
:107AE0002300A40093C5250093B51500960593E6E1
:107AF000050893054627A300D4000345462783C6FF
:107B000015001375F50793F6E60F230AA626A38042
:107B1000D5001305440011468146EFA08FDA0345D6
:107B200014009305098022056D8D136505102181D0
:107B3000A300A4009305A00F03C599061365450093
:107B4000A384A90623A4B90209496DA20345340000
:107B5000034624002205518D4166130616F0631A70
:107B6000C50813054400EFF01FB5370514001306D0
:107B700035002945A145EFA00FA703451400C545D1
:107B80001375050EA300A4003725F87F2300B40069
:107B90009304858003C554052300B4009145134523
:107BA000250013351500160513651508A300A4005C
:107BB000654603C59406814613651500A384A40693
:107BC0002285EFA09F80885405495DC523A4040247
:107BD0000385A406136545002385A40671A83715FF
:107BE000F87F0355657F0549CA846385A5108944DC
:107BF00011A23716F87F0356667F0549CA84630BC6
:107C0000C50EAE84C5A88D453709F87F2304B92871
:107C100013962500B705F87F130544009385852743
:107C20008146EFA00FCA03C55905631D95000345A2
:107C30006400834574007D8993F5C50F2303A40078
:107C4000A303B4000305892813091500EFF03FA32F
:107C500055A0B715F87F83D5657F631DB50891459D
:107C6000694681462285EFA04FF603C5A90605495E
:107C70001375D50F2385A906CA84ADA8B715F87F5B
:107C800083D5657F8544E301B5EC2689A5A08944A9
:107C900025A0B715F87F83D5657F8544631EB500A1
:107CA0000305AA0691451365250065462305AA0626
:107CB00081462285EFA06FF123260A0403451400B4
:107CC00091451375050EA300A4003725F87F230006
:107CD000B400139689000345D5852300B4001345ED
:107CE0002500133515003605518D2166518D2181F2
:107CF000A300A400034534008345240022054D8DD4
:107D0000C1651386E5FF698E938505F06309B600AA
:107D1000B715F87F83D5657F6303B50089440345B4
:107D20000400939564001375F5034D8D2300A400A2
:107D30001375F90F1244224AB2494249D244F24023
:107D400005618280130181FC3725F87F1303A59913
:107D50000305130085654ED2814F118193898538C3
:107D6000B705F87FC16726D64AD452D056CE5ACC32
:107D700022C013747500B70400C0370900801305D2
:107D80002003A942130F10271306803E9385455206
:107D9000930640061307401F130AF00BFD17B70A9E
:107DA00000409303A00F7E8B7E8EFE887E885ECA85
:107DB00062C866C66AC46EC209AA8A0E9A9E83CB3E
:107DC0005E0003CC4E0003CD3E00939C8B01420C21
:107DD000336C9C01220DB36DAC0103CD2E00B3FEBC
:107DE0009C0033EDAD01638A2E03638C5E057E8CAF
:107DF000FE8C6367D00793DEAD0013FCFE3F937EDD
:107E0000FD3FB38E5E0293DC3E00330CAC0263E5B3
:107E1000EC03856E938E8E3805A0935E4C0113FCA7
:107E2000FE3F937EFD3FB38E5E0293DC3E00330C3B
:107E3000AC0263E3EC01CE8EB38E8E03B3DCCE02D4
:107E400005A0935E4C0193FEFE3F137CFD3FB30CF7
:107E50007C02338C7E0263E38C01E28C338CAE02B5
:107E600083CE9500B38EDE0263E08E0783CEA5003D
:107E7000B38EEE0263E6DC0183CEA500B38CEE0286
:107E800063629803B3EE0C01630ED00183CE7500DC
:107E900033FDF800637B8D0163990C0193FE8E0026
:107EA0006305D001637F7A0105A083CE7500636D01
:107EB0007A01637BAC0163990C0193FE8E006365CC
:107EC000D0015A8EE2886688050B937EFB0FE3E6AD
:107ED0008EEE937EFE0F994F63E2DF1B3704F87F2F
:107EE000930F3426838E3F0083C42F00E20EC2041A
:107EF000B3EED40183C4B5003709800BB389E40223
:107F0000B3F42E016375380583CE7500370900047C
:107F100093FE2E00B3E42401630BD0030348330027
:107F20008348230013783800220833681801B30807
:107F3000580293D8380063E6E80119681308881AD4
:107F400019A03308A8028568014E93888838937E6B
:107F5000FE0F8A0E93EE3E00769303432300B70E86
:107F60000004137F030C1309000433F3D401631AD4
:107F70002F03B352780293031E0093F37300139EF2
:107F8000C30193F3F23F9392A300B3E2C2016305EE
:107F9000600603C3A500B3E292000603B3E26200E9
:107FA00069A8630E600413031E0013737300720349
:107FB000630F0007B303C80233FEF80083CEA500A9
:107FC00037AF0700B3D3C303130F0F12B38EEE0303
:107FD00033DECE0333639300B3D35302B3525E0256
:107FE000370E1000130E0EC0AA03B3F3C3013363A0
:107FF000730093F2F23F81A0B3E2920035A0330305
:10800000C802B3F3F80033537302B352530213039D
:108010001E001373730072033363930093F2F23FF5
:108020009393A200B3625300B3E2720039A0B70287
:10803000800FB3F25400B3625300B3F8F800330674
:10804000C80233561603B3D6D8023357E80213D802
:108050008201A30154267D8E3355A60213D68200D9
:1080600093D70201A380CF002381FF00A3810F01DA
:108070002386D500A386E5002387A5000244924D00
:10808000224DB24C424CD24B624BF24A025A9259A8
:108090002259B2541301810382803D713725F87F44
:1080A00006CE1305A59926CA834455004AC852C472
:1080B00056C2030A4500834A35000349250013D5FB
:1080C00044004EC622C093797500EF50200E11CDAA
:1080D000EF50800E19C9EF902FDD89456317B50069
:1080E0003705F87F1305052929A03705F87F130503
:1080F000852205446300300D03450500636C350B94
:1081000013150A01A20A33E5AA002981137AF53F63
:10811000EF50C00905C1EF50200A09CDEF90CFD82C
:1081200089456319B500B705F87F13952900938534
:10813000552E39A0B705F87F139529009385952210
:108140002E959305C5FF03C5150003C6050022053E
:1081500093760530D18E63EF46053717F87F33E805
:108160002A0103C625008347477F93F8840093754F
:10817000F83F636D100193F7E70F13F84400230AEB
:10818000F77E636B000163E7B60239A093E6170040
:10819000230AD77E6360BA024206518D2D813706CD
:1081A000F87F2308A6522945B385A5020545EF00AF
:1081B000B07A014422850244924A224AB249424995
:1081C000D244F240056182803705F87F9305F5338C
:1081D0008306F53303C535003707F87F038815009C
:1081E000838825009372D50F3715F87F8145930753
:1081F000B7331305957F1146A30DD732AE86A38002
:10820000070123811701A38157006F90FFF07D7153
:1082100009459305100F06C626C222C0EF904FC332
:108220003714F87F8345F47F937405086382B404A0
:1082300009459305100FEF90AFC11375050811E9BB
:108240003715F87F0305E57FB705F87F2388A52854
:1082500021A83705F87F830505293716F87F85465D
:10826000230FB67E2308D528EF002001A30F947EAC
:1082700002449244B24041618280130181FB86C274
:108280004EDAB709F87F03C50929B705F87F131639
:1082900025003705F87F52D85AD422C8138A552EA4
:1082A0001304D52A014B5285A285DA8626DE4ADCE4
:1082B00056D65ED262D066CE6ACC6ECA02C6EF9047
:1082C0005FE089449305100F2685EF906FB86D9994
:1082D000B705068023A2A53C9305E00F2685EF9005
:1082E0002FB79305401F330CB50265651305A5052F
:1082F0001309C1002AC2370500C1930C3A00914A04
:10830000136D3900936D2900936B19007D15DA8484
:108310002AC4DDA04A85A28556868146EF907FDA81
:1083200083450D0003C50D0083C60B001396850120
:108330004205518D139686008346C100498E13F77E
:10834000050CB365D60041EB29821376F63FD14682
:10835000B356D60293F5F53F2947568ACE8AB385A0
:10836000D5023387E502E28563638701BA85B38965
:108370008541930540061307803E63E4E900B3D5C9
:10838000D902A946B3D5D502B706F0FF758D2A06E6
:10839000518D63633B01DA89336BB5000945930561
:1083A000100FEF90EFAA1375050881456309B5001A
:1083B0003705F0C092453375AB00336BB5002245ED
:1083C000B375AB0001456395A4003705002FC98D37
:1083D0004E8BD689D28A13D5850013D6050193D644
:1083E0008501A38EBCFE238FACFEA38FCCFE238021
:1083F000DC008504910C110403C50929E3ECA4F009
:108400001305803E636D6501854509452388B928BC
:108410009305100FEF90CFA31365450039A00945D0
:108420009305100FEF90CFA26D99B705068023A298
:10843000A53C4244D24D624DF24C025C925B225B01
:10844000B25A425AD2596259F254964013018104E9
:10845000828061113705F87FB705F87F1305952CE9
:108460009385D52A714606C2EFB0802692403335F7
:10847000A000210182803705F87F81451305952CE6
:108480007146AE866F905FC921110545B705F87F2B
:1084900006CA2388A528B705F87F26C64AC422C283
:1084A0003705F87F13841529914401491305D52A0E
:1084B000A2852686CA86EF90DFC03705F87F1305B0
:1084C000552EA2852686CA86EF90BFBF3705F87F56
:1084D000CA85CA8612442249B244D2401305952C5B
:1084E000714661016F905FC3611106C2EFE09FC9E1
:1084F0001376C5001375050C9345C6001345050C8E
:1085000093B5150013351500C98D21456306A600E6
:108510001305A00589E531A0130560F999C113057C
:10852000C00281E5930500F919A0930510F93706FB
:10853000F87F9306D62A0547A306A62AA380B6008D
:108540002381E6009240210182803705F87F1306DF
:108550003526830636001D4793D546009D896382E4
:10856000E518834726000346160013978601939665
:108570000701D98E220633E8C6003706F87F834606
:108580003526139525001306D62A32950346D5FFC6
:108590008348E5FF22060345C5FF937706305D8DCE
:1085A000A9473305F5029352350013031027C2087B
:1085B00063E5620005651305853833661601854855
:1085C000B366D800639615099358A60093F8F83F50
:1085D000B388A80293022003B3885802B702F87F39
:1085E0009382425203C312011358A8009373F83FB9
:1085F0003303F3021308803E63F66302B356F502B9
:1086000083C212010D6313030380B3826202370336
:10861000100013030380B3F2620093F6F63FD98E85
:10862000B3E6560033D8080313D7A6001377F73FF5
:108630003307F7026374E5043357F502B70700FF09
:10864000FD8E1377F73F9317A7005D8FD98E3DA05E
:108650003708F87F034858539308401F93F2F63FBA
:10866000B382F20233081803637A5500B356F50259
:1086700093F6F63F9397A600D98EDD8E9397C501AA
:10868000B705F87F37078080938545527D1783C8EB
:108690001501758F9302401FB3885802D98F636507
:1086A00018013708000119A03708000593082003B6
:1086B00033551503B3E707013708F87F9308B8333C
:1086C00093D286004183E1832D82A30DD832A3800B
:1086D00058002381E800A381F8002389C500A389FD
:1086E000A50082803725F87F9306A59983C5560299
:1086F0003705F87F13D645001D8A0347153013054B
:10870000F6FF9377F50F054563F8E70883C7360250
:108710000387460213988700B707F87F0A069387F6
:1087200027304207B388C7003367E80003C6D8FF85
:1087300029839377F73F220603C7C8FF9372063059
:1087400033E7E200636AF70483C2260283C6E8FFC8
:10875000B718F87F3368580083C2887F13F3850009
:108760001378F83F636B600093F7E20F9189238CD5
:10877000F87E91E96362070339A093E51200238C28
:10878000B87E63EB070113950601518D2D81B70566
:10879000F87F238BA552014582800000211106CA73
:1087A0004AC44EC20949930900074A85CE8526C6A8
:1087B00022C0EF80FFE92A84930510074A85EF80E5
:1087C0003FE9AA844A85CE851374F40FEF805FE8F1
:1087D000630FA4008944930500072685EF805FE7B7
:1087E0002A84930510072685EF809FE6AA841395B7
:1087F000840013750530C165418DFD150244924911
:108800002249B244D2406D8D610182809305400AB5
:108810003305B502B725F87F938585802E95230310
:108820000506130575068145094631A0B306B50056
:10883000238006008505E39BC5FE82809306400ADF
:108840003305D502B726F87F938686803695834612
:108850006506094763E8E60085890606D18D23048D
:10886000B506828085890606130765063695D18D83
:1088700013861600A303B5062300C7008280930663
:10888000400A3305D502B726F87F93868680AA96DC
:1088900003C7660605451DC381473E889378F80FD8
:1088A00063FFE800B69883C87806050893F21800BD
:1088B000E396B2FE93D81800E392C8FE82803E850C
:1088C0008280ADCD9305400A3726F87FB305B50207
:1088D00013068680B2953726F87F130606952A96EA
:1088E00023A605002300060023A0050623AA0500F1
:1088F0003726F87F83C6A50603C79506A206D98E3C
:108900004167130707DC13062695F98E3295130687
:10891000F00F13D7860023000500A389C504238A1E
:10892000C504238E0504238D0504A38B0504A384AD
:10893000D5062385E5062389050882809305400A2C
:108940003305B502B725F87F938585802E9583057D
:108950004509094693E515009546230AB508A30A7B
:10896000C504231C0504A30D0504A300050023165C
:10897000050623070506A30A0508232C0508230E70
:1089800005082310050A2312D50682807D71B725BC
:10899000F87F06C622C2138485808345240006051D
:1089A000098993F5D50F4D8D2301A4000945930541
:1089B000E002EF80FFC9834524005D998A05A18903
:1089C0004D8DB705068023ACA50A1244B240416123
:1089D00082807D71B725F87F06C622C21384858008
:1089E00083452400058993F5E50FC98D09452301C9
:1089F000B4009305E002EF80BFC583452400799958
:108A000085894D8DB705068023ACA50A1244B24076
:108A100041618280B725F87F93858580D041C8C1A8
:108A20006304A6022145631DA60003C5550509463A
:108A30006318C500A38A050823AC0508238E050822
:108A40003725F87F2308059482803725F87F034572
:108A5000C58082807D7106C622C201442285EFF066
:108A6000FFDAEFE07FB685452285EFF09FE5370519
:108A7000F87F1305B55683452500124493F5E50F9D
:108A80002301B500B240416182807D7106C622C2D9
:108A900001442285EF805FA0EFF0DFFBEFE03FBEF7
:108AA0002285A285EFF0FFE10945E945EF805FBA35
:108AB0001375F5FCB7050680A8D51244B240416194
:108AC0006F60305B9305400A3305B502B725F87F28
:108AD000938585802E95B70500FF2CC98280611192
:108AE0003725F87F93058580370600FF06C22304EB
:108AF0000580238B0504B0C9EFF03FF93725F87FD7
:108B0000834545951306459593F5E50F230AB594DE
:108B1000A3000600924021018280211106CA26C6C8
:108B20008545AA844AC422C2639AB40015459305B8
:108B3000000FEF80FFB11375050815E5EF400067E2
:108B400011CDEF40606719C9EF801FB689456317E3
:108B5000B5003705F87F1305552E11A83705F87FA6
:108B60001305952229A03705F87F130525309305B5
:108B700015008385050003450500A20593F5053022
:108B8000C98D1305400AB726F87F3385A402938662
:108B90008680369529468346550509443389C502A2
:108BA000639086024841D545631BB50205651305F0
:108BB00085BB636BA90201456387A4041544A9A082
:108BC00001456383A4001544E9452285EF805FA831
:108BD0009305C05D1375F5FC63F4250325A80145D5
:108BE0006389A400154439A001456385A404154494
:108BF00099A00944E9452285EF809FA51375F5FCEE
:108C00001365050111A80944E9452285EF805FA499
:108C10001375F5FC136505023706048093150401EE
:108C200013068606B29588C112442249B244D24046
:108C3000610182800944E9452285EF807FA1930587
:108C4000B05D1375F5FCE3ED25FBF9B721119145F6
:108C500006CA26C64AC44EC222C0630EB504894560
:108C60006307B50A8D456307B50E85456314B514D2
:108C70003705F87F9305455203C66500B70609809E
:108C80001376E60F13076006930740042383C5009D
:108C900023A6E60823A6F608370606808305455274
:108CA0009306700793E515002302B5522326F608B4
:108CB0002326D60891A23704F87F03454452B7040F
:108CC00006801375E50F930560061309400413062B
:108CD00044522302A45223A6B40823A62409B705AC
:108CE00009800305660093097007136515002303C7
:108CF000A600094523A6250923A63509EF801F9460
:108D000003054452136515002302A45279A83705C0
:108D1000F87F834545523706068093F5E50F9306A5
:108D200060062302B55293054004130545522326DD
:108D3000D6082326B608B706098003066500130780
:108D40007007136616002303C50023A6B60823A6E2
:108D5000E6085DA03705F87F13044552834564009B
:108D6000B704098093F5E50F130660061309400464
:108D70002303B40023A6C40823A6240937060680CB
:108D8000830545529309700793E515002302B552F8
:108D900009452326260923263609EF803F8A030545
:108DA0006400136515002303A40023A6240923A649
:108DB000340999A03705F87F9305455203C665002D
:108DC000B70609801376E60F130760069307400481
:108DD0002383C50023A6E60823A6F60837060680E7
:108DE00083454552B706068093F5E50F2302B55239
:108DF0002326E60823A6F608024492492249B244F3
:108E0000D240610182807D7106C626C222C02A84BA
:108E1000EF809F898945631DB502B704F87F03C5BC
:108E200044346307850291456315B40085456301A9
:108E3000B5022285EFF09FE1154523828434630556
:108E4000A4002145EFA0FFC9EFD07FE9EFE00FCEEE
:108E500002449244B240416182806111814506C260
:108E60006303B50099453706F87F13064652B2955D
:108E700083C50500858985E1834536001306400AD0
:108E80003305C5023726F87F1306868093F5050F54
:108E900032950CCD31A8EF40603101C9EF80DF8001
:108EA00089456314B500094511A01545EFF0BFF5DC
:108EB000924021018280130181FD3705F87F06D29F
:108EC00026CE4ACC4ECA52C856C65AC45EC222C02A
:108ED0001309455203457900058901ED3D45894552
:108EE000130620032305A900A305B900A304C900A4
:108EF00025A00345990009E51305800CA304A900EA
:108F00000345A90001E53D452305A9000345B90036
:108F100001E50945A305A9003725F87FB705F87FC6
:108F2000B706F87F9304858093859522938636262D
:108F30000385440903863500038726000944136529
:108F400015001366160013670708A38A8404238A92
:108F5000A408A38A040823AC0408238E0408A38170
:108F6000C5002381E600EF802FF4631C85003705E0
:108F7000F87F1305552E8305350093E51500A301F1
:108F8000B500B725F87F03C54595138645959376BB
:108F9000E50F0945A3000600238AD5949305100F19
:108FA000EF800FEB1375050815E1B705F87F37055E
:108FB000F87F93858527130600069306400523094D
:108FC00005262381C500A381D50025A03705F87F9C
:108FD000130505273706F87F830515001306862736
:108FE000AD46130700062301B5002306D600230172
:108FF000E60009449305D00C2285EF806FE56D995A
:10900000B709068023AAA9329305F00C2285EF80C8
:109010002FE41365050123AEA93293056002228572
:10902000EF800FE3136505089305A00F23ACA90893
:1090300023A8B9349305000F2285EF806FE14189A1
:1090400055ED09449305E00C2285EF806FE0137520
:10905000F5FD23ACA932154A034599009305500F3D
:10906000B30A45032285EF80AFDE5695930AF03FA1
:1090700063F5AA001305F00F29A883059900094597
:10908000338445039305500FEF808FDC22951375D1
:10909000F50F094423ACA91C930570072285EF80C6
:1090A0002FDB83459900137BC5FFB38B45039305E5
:1090B000500F2285EF80CFD95E9563F4AA000D454D
:1090C00029A8834599000945338445039305500F2A
:1090D000EF800FD8229521810D89336565019305B5
:1090E000000823AEA91C23A0B90409459305E00C90
:1090F000EF800FD61365050223ACA93203D5840592
:10910000C1659385F5BF3376B5009306403D239C3A
:10911000C404F4C405650244924B224BB24A424A4D
:10912000D2496249F24492509305853801451301B2
:1091300081026F0060021306400A3305C50237261C
:10914000F87F1306868032950316850593C5F5FFD3
:10915000F18D231CB50482807D7106C626C222C013
:109160002E84AA8409459305900FEF806FCE137566
:10917000050821CD91C82285EF002019130540056F
:109180009305800C09460DA8130540069305E006DB
:1091900013060004EFA06FDA2285EF000017130416
:1091A00040059305800C09462285EFA00FD9930551
:1091B000F00B130610022285EFA02FD8B725F87FF9
:1091C0000145A3800580EF00A01B02449244B240F9
:1091D000416182807D7106C622C201442285EFF082
:1091E000EFFA2285EFF0EFFE0945EFF0BF8222850E
:1091F000EFD0BFC13725F87FB7050680232405824D
:1092000023A6053E1244B240416182807D7106C6AC
:1092100022C22A840945E945EF808FC309C8137526
:10922000F5FC13650502B7050680A8D535A01375B2
:109230000503C1456302B5020945E945EF804FC109
:109240001375F5FC13650501B70506803726F87F11
:10925000C946A8D52322D6841244B24041618280F7
:1092600061110945E94506C2EF808FBE13750503FC
:10927000930500026314B50005451DA00945E945A5
:10928000EF800FBD13750503C1456317B500372582
:10929000F87F0325458401C51305F00F11A0014592
:1092A000620592406185210182807D710945F54505
:1092B00006C626C222C0EF80AFB90D898D45054490
:1092C0006303B5028944F5452685EF806FB831897F
:1092D000B145630AB500F5452685EF806FB70D8966
:1092E000631995000144228502449244B2404161D1
:1092F00082800945F545EF80AFB53189A1456314FA
:10930000B5000145D5B77D55C5B77D71B145B305EC
:10931000B5022945B3D5A50241669306C6FF1307DA
:10932000804C06C626C222C0ED8E89826362D702B7
:109330007D16F18D3385A502AD453355B502B705D0
:109340000400E1150A056D8DE545B354B50219A079
:109350009304802C1304400513F6F40F9305D00DED
:109360002285EFA08FBD13D58400137635002285AA
:1093700002449244B2409305E00D41616FA0EFBBFF
:109380007D7106C622C22A8409459305900FEF809D
:109390002FAC1375050809C53725F87F2301858093
:1093A0001244B240416182807D7109459305900F5E
:1093B00006C6A3030100EF80AFA91375050819E1E4
:1093C000014529A8130540059305800C130671007B
:1093D000EFA08FD10305710005810589B24041617D
:1093E00082807D7106C622C209449305900F2285B2
:1093F000EF800FA6137505081DC1EF00C00205E13F
:10940000EF30D05A11C9EF802FAA63178500EF30D3
:10941000B05A19C1094511A01545EFF0DF9E12445D
:10942000B24041618280611109459305900F06C2E7
:10943000EF800FA2B725F87F83C515801345F5FF90
:109440001375050893B515001D8192404D8D2101BE
:109450008280611109459305900F06C2EF804F9FEE
:10946000B725F87F83C52580137505081D81B335A1
:10947000B00092406D8D21018280611109459305F4
:10948000900F06C2EF80CF9C1375050815C93725CC
:10949000F87F0345C580930500036305B500F545D6
:1094A0006310B502EFF0FFFA01CDEFF0FFEF3335B7
:1094B000A000B725F87FA380A580EFF09FF229A038
:1094C0003725F87FA3000580924021018280611139
:1094D0001306400AB726F87F3306C50293868680B6
:1094E00006C2369683460600B1CA3727F87F931620
:1094F00055001307679536978346260003085605DF
:1095000093974600FD8993F70702DD8D9317680056
:10951000858A0346060593F7070CA206DD8E1D8A91
:10952000D58D26064D8E21822300B700A300C700EB
:1095300009468146BA85EF00400119A01305C00F06
:10954000620592406185210182803D7106CE26CA66
:109550004AC83689AA841305400AB726F87F4EC642
:109560003385A4029389868052C4338AA9000345B7
:109570001A0A854622C26315D5001304C00F35A808
:10958000630E200103C5150083C605001375E50FA2
:1095900093F6F60DA380A5002380D5002685CA8604
:1095A000EFD00FC62A846355800233052A01830554
:1095B000050585059D892308B5041315840112440A
:1095C000224AB2494249D244F24061850561828013
:1095D00091C4EF30B05863072001C5B703A5490017
:1095E000E36D20FD1375F50FE145E308B5FC7955F2
:1095F0006318A4001305500289CCEF30505421A801
:1096000091CC03C5690A814505896301B502754599
:1096100039A8EFF02FC01304E00F45B703C52900A8
:10962000814505896308B500754531A02145EF30B6
:10963000105161B72145EFF0EFBD41B7211106CAC6
:109640004EC222C085492A8426C64AC4631A340100
:1096500015459305000FEF70BFFF1375050815E55D
:10966000EF30D03411CDEF30303519C9EF80CF83D2
:1096700089456317B5003705F87F9305052911A8BB
:109680003705F87F9305852229A03705F87F9305D4
:1096900015301305400A3726F87F3305A402130658
:1096A000868032950346050051CA03C90500630A46
:1096B00020093726F87F9315540013066695B304E6
:1096C000B6008345250003065505939645001A0606
:1096D0008589034505051376060CA205D18D1D89E4
:1096E0001376790093F6060226053206D58D518D44
:1096F0004D8D936515002181A380A4002380B400C3
:10970000631A340115459305000FEF707FF413754C
:10971000050831E5EF30902915C9EF30F0291DC556
:10972000EF709FF889456313B502B705F87F13857D
:109730002400131629009385552E15A81305C00F74
:10974000A9A091452285EFF09FD881A0B705F87FA9
:1097500013852400131629009385952209A8B705BF
:10976000F87F138524001316290093852530814640
:10977000EF803F9513152900136525001376E50F3B
:1097800081462285A685EFF05FDC6205024492499E
:109790002249B244D240618561018280211106CA0A
:1097A00022C22A841305400AB725F87F3305A40294
:1097B000938585802E958345050026C64AC4BDC97C
:1097C0003726F87F9315540013066695B304B60048
:1097D0008345250003065505939645001A0685899D
:1097E0001376060CA2050345050593F60602D18DF6
:1097F0003709F87F33E6D5001D89834559242605AE
:10980000518D13F675003206518D13664500218186
:10981000A380A400138524002380C40019CCB705BD
:10982000F87F83C5E531B706F87F13962500938549
:10983000F63111A81305C00F35A013962500B70502
:10984000F87F938565248146EF80BF8703055924FF
:1098500081460A05136525001376E50F2285A68546
:10986000EFF0BFCE620512442249B244D240618576
:10987000610182807D7106C622C02A841305400AD8
:10988000B725F87F3305A402938585802E958345FF
:10989000050026C2B1CD3726F87F93155400130674
:1098A0006695B304B60083452500030655059396D7
:1098B00045001A068589034505051376060CA205A1
:1098C00093F60602D18D1D89D58D26054D8D8565B2
:1098D00089054D8D935585002380A40013852400B0
:1098E000A380B40009C8B705F87F9385B53301A8F4
:1098F0001305C00F39A8B705F87F938535261146A3
:109900008146EF800FFC194681462285A685EFF03F
:10991000DFC3620502449244B240618541618280A6
:10992000211106CA26C622C23E84AA841305400A13
:10993000B727F87F3385A402938787803E958347B6
:1099400005004AC4D9CB3728F87F939754001308F1
:1099500068953309F8008347250083085505139857
:1099600047002295FD891378080203450505B3E5F4
:10997000050113986800858B1378080CA2071D89D0
:10998000B3E7070126053E07DD8D598D4D8D13F791
:10999000061021812183938746002300B900A3008C
:1099A000A900A301E90069473708078093D8870019
:1099B0002301D900130549008146B2853A86232444
:1099C000F83A2326183BEF80CFEF1306F00F2685D9
:1099D000CA85A286EFF07FB719A01305C00F6205F4
:1099E00012442249B244D240618561018280130150
:1099F00081FD06D226CE4ECAB289AA841305400A3A
:109A00003726F87F3385A402130686805EC2B30B27
:109A1000A60003C50B004ACC52C856C622C03E84DD
:109A20003A8A3689AE8A5AC44DC5630F4007094544
:109A30009305000FEF70DFC11375050235C503856F
:109A4000190063430506B725F87F139554009385E5
:109A500065952E9583C52B0003875B05939645007E
:109A600013F6FA0193F60602558E93166700858960
:109A700093F6060CA205D58DB3868B0083C606052A
:109A8000D18D13F6760026069316FA00558E4D8E6C
:109A900021822300B500A300C50009058146CE85BB
:109AA0004A86EF800FE255A01375390015C5914520
:109AB000338BA540B725F87F1395540093856595A2
:109AC0002E954A95814509055A86AE86EF80CFE4EA
:109AD00029A01305C00F49A8014BB725F87F13959E
:109AE0005400938565952E9583C52B0003875B05F0
:109AF0009396450013F6FA0193F60602558E9316D7
:109B00006700858993F6060CA205D58DB3868B0078
:109B100083C60605B30A2B01D18D13F67600939602
:109B2000AA009D671317FA00FD8E2606D98E558E62
:109B30004D8E21822300B500A300C5000905814692
:109B4000CE854A86EF80EFD75689B725F87F1395E3
:109B5000540093856595AA95130529001376F50F92
:109B60002685A286EFF07F9E62050244924B224B2F
:109B7000B24A424AD2496249F24492506185130185
:109B800081028280797106D626D252CC328AAA848A
:109B90001305400A3726F87F3385A4021306868012
:109BA0005EC6B30BA60003C50B004AD04ECE56CA04
:109BB00022C23E84BA893689AE8A5AC862C455C563
:109BC0006300300909459305000FEF707FA81375F6
:109BD00005023DC503053A0063440506B725F87F35
:109BE00013955400938565952E9583C52B000387A7
:109BF0005B059396450013F6FA0193F60602558E1F
:109C000093166700858993F6060CA205D58DB38659
:109C10008B0083C60605D18D13F676002606939633
:109C2000F900558E4D8E21822300B500A300C5009A
:109C3000090593052A0081464A86EF808FC86DA8E2
:109C40001375390015C59145338BA540B725F87FAD
:109C500013955400938565952E954A958145090580
:109C60005A86AE86EF804FCB29A01305C00F65A0A2
:109C7000014BB725F87F1395540093856595338C78
:109C8000A50003C52B0083865B051316450093F5DD
:109C9000FA0113760602D18D1396660005891376B4
:109CA000060C2205518D33868B0003460605B30A48
:109CB0002B014D8D937576001396AA001D67939620
:109CC000F900798EA605558ED18DC98DA18123000D
:109CD000AC00A300BC0013052C0093052A008146AC
:109CE0004A86EF800FBE6308300103053C00136510
:109CF0000508A301AC005689B725F87F13955400D9
:109D000093856595AA95130529001376F50F268589
:109D1000A286EFF09F8362051244224CB24B424B65
:109D2000D24A624AF24902599254B2506185456161
:109D300082801306400A3305C5023726F87F1306D2
:109D40008680329503168505D18D231CB50482804B
:109D50001306400A3305C5023726F87F13068680AE
:109D60003295035585056D8D3335A000828013062D
:109D7000400A3305C5023726F87F130686803295E0
:109D80000306A505D18D230DB50482801306400A74
:109D90003305C5023726F87F130686803295030601
:109DA000A50593C5F5FFF18D230DB504828013063B
:109DB000400A3305C5023726F87F130686803295A0
:109DC0000345A5056D8D3335A00082809305400ABB
:109DD0003305B502B725F87F938585802E958315C9
:109DE000850593E50502231CB50482809305400A8E
:109DF0003305B502B725F87F938585802E958315A9
:109E000085050566D18D231CB50482809305400A23
:109E10003305B502B725F87F938585802E95831588
:109E200085050966D18D231CB50482809305400AFF
:109E30003305B502B725F87F938585802E95831568
:109E400085051166D18D231CB50482809305400AD7
:109E50003305B502B725F87F938585802E95831548
:109E600085052166D18D231CB5048280034535000C
:109E70009375050C91C18280137685003725F87F94
:109E8000130585808355850581466305D60093E5D6
:109E9000150021A041667916F18D231CB50482803E
:109EA000211106CA22C209449305F002228526C662
:109EB0004AC4EF70EFF9137505F837090680232EB1
:109EC000A90AEFE09FBCEF30602E19C9EF30C02E19
:109ED00001C9EF706FFD631585000545EF30A02EB9
:109EE0003725F87F93048580C840D1451365050167
:109EF0006305B50AF1452285EF708FF5799923281E
:109F0000A9063705F87F3706F87F13059522130653
:109F10003626830535008306260093E5150093E673
:109F20000608A301B5002301D600EF70EFF7631C0C
:109F300085003705F87F1305552E8305350093E519
:109F40001500A301B500CC400D451386F5FD6367F0
:109F5000A60090449306F6FD6367D4040544228569
:109F6000EFC0BFEA03852400136515002381A40018
:109F70002285EF70AFEC03C52400B70500FF05890B
:109F8000ACC811E50145EFE07FA0114529A00545CA
:109F9000EFE0DF9F4D45EFE0FFA712442249B244B6
:109FA000D24061018280D515914663E6D5009305C4
:109FB00056FFE362B5FC03C524009375E50F014528
:109FC0002381B400EFC07FE4EF30401E19C5EF706D
:109FD000AFED63148500094511A01545EFE0BFE220
:109FE00059BF611106C2EFE0FFA63725F87F034590
:109FF000A580058919E1154511A06145EFE09FA1F4
:10A00000014592401306100FAA85AA8621016F8090
:10A01000CFBB7D7106C622C2EFC03FDF0944E945D0
:10A020002285EF70EFE23D8995456313B5003D440D
:10A0300022851244B24041616FE0DF9D7D7137257A
:10A04000F87F06C622C213048580034544090589AA
:10A050001DCD09459305100FEF708FDF058905C9E8
:10A0600009459305100FEF70AFDE09890DC1830517
:10A07000A405094513E625009305100F230DC4041C
:10A08000EF700FDD7599B705068023A2A53C124439
:10A09000B240416182809305400A3305B502B7257D
:10A0A000F87F938585802E958305A50593E525008A
:10A0B000230DB5048280B725F87F2380A580828098
:10A0C0003725F87F03450580828021113725F87FE9
:10A0D00006CA22C2130485800345440926C64AC421
:10A0E00005893DCD03455409A54563E2A5029D457B
:10A0F000636BB500EFE08FEA83258409AA950345D9
:10A100005409232CB4080505A30AA40891A89304B4
:10A11000F00F63079504032584098D453355B50277
:10A120003729F87F231BA998EFE04FE70356699979
:10A13000AA856365B6003305B64019A03385C540CE
:10A1400041667D16718D09466368A6000545EF706E
:10A150009FD3A30A940829A0A30A0408232C040867
:10A1600012442249B244D24061018280797106D6FC
:10A170004ECEB729F87F83C58999094526D24AD0A2
:10A1800052CC56CA5AC85EC662C422C2638DA508A4
:10A19000854A63895511636EB02CEFC05FB40944E2
:10A1A0009305D00F2285EF70AFCA9344F5FF930556
:10A1B000C00F2285EF70CFC9658D0DC58944130985
:10A1C000E00C2685CA85EF70AFC813654500370AD5
:10A1D0000680232CAA322685CA85EF706FC76D9939
:10A1E000232CAA32372AF87F13098A8003254900D5
:10A1F00029469375F50F63EBC5003D4663EBC52615
:10A200001376C50F930600026305D626034659054B
:10A210006316860C1306A00263EBC50A1306E00260
:10A2200063FEC50AB9A409449305F0022285EF70C4
:10A230002FC2137505F8B70506803726F87F23AEC1
:10A24000A50A23040680EF2070761DCDEF20D0767E
:10A2500005CDEF706FC5631985020545EF20B07617
:10A260000145AA85EF703FC21544C1452285EF70B4
:10A270002FBE13651500B7040980A8C0C945228503
:10A28000EF700FBD7999A8C405659305853805451C
:10A29000EFE09FECEFC0BFAE0145EFF09FD7238CFE
:10A2A0000998C1AAB725F87F138485800C4C6300F8
:10A2B000B01CEFE0AFCE9305700963ECA51A0385DF
:10A2C00089990505238CA998232C04005DA2754665
:10A2D0006396C500EFF09FD6032549001375F50F6F
:10A2E0006309551991456306B51893056002630229
:10A2F000B5183705F87F034545520989636BA016E9
:10A30000EFC09F9383452900AA84858981E9EFE006
:10A31000EFC893058007B3BAA5001DA803458A803E
:10A32000631B5501F5452285EF708FB20D896301DE
:10A33000850203458A80631C85000945F545EF7059
:10A340002FB1318913458500933A150011A0814A38
:10A350000345290093C51A0005898DE085E119EDB3
:10A3600009459305B00FEF70AFAE2A84EFC04FFEE2
:10A370006306A40203051900050515A013B6140011
:10A38000F18D95C9B725F87F03C6959915CEA38C95
:10A3900005981DE96145232EA900E1A801459375A3
:10A3A000F50F13065006A300A90063E6C500EFC031
:10A3B0009F8CA3000900394585453726F87F232E59
:10A3C000A900A30CB69875A00325C9015DE1954AC3
:10A3D000130B8009854BF544214C13F5FA0F29C561
:10A3E00003452900FD1A058911E5EFE02FBBE3764F
:10A3F000ABFE41A003458A80631B75012285A685BB
:10A40000EF700FA50D896306850603458A806319E1
:10A4100085002285A685EF70AFA33189630B850582
:10A42000EFC09F815DD9B1A00945F145EF704FA202
:10A430007999B7050680A8D90145EFE01FA2EFD0B2
:10A440000FA4EF706FA609C9370514001306353045
:10A450002945A145EF703F99EFA0CFBA1145EF9084
:10A460004FE80145EFE00FDB038589990505238C53
:10A47000A9981244224CB24B424BD24A624AF2494A
:10A4800002599254B25045618280211106CA26C6F3
:10A49000B724F87F22C21384A49903051400B725BA
:10A4A000F87F09814AC47189138985801366250064
:10A4B000130529078146A285EF70BFC0034529090E
:10A4C00089456314B500230909080345140083C5B1
:10A4D000A49911811306490712442249B244D2407B
:10A4E00093767500FD89014561016F50000B611184
:10A4F00009459305000F06C2EF708F95137505028D
:10A5000019C53725F87F0305D59963550500EFF088
:10A51000DFF709E50145C145EFE07FFB92402101EE
:10A520008280130181FD06D25EC2B72BF87F22C064
:10A530001384AB990305140026CE4ACC4ECA52C8E8
:10A5400056C65AC4635005028345340013F6050805
:10A5500011EA139585008345240013750510336BAC
:10A56000B50021A01181137B75003725F87F930A70
:10A57000858003C56A0619CD03C5AB99B335600163
:10A580001376F5010145EFE08FAF630EA020014582
:10A59000EFE0CFA703A54A0063636003F5456310AE
:10A5A000B50283C5AB990546FD89F51593F5F50F01
:10A5B0006367B60013055002EFE0CFC521AC030678
:10A5C000140083C63A05935516009D896398B6001A
:10A5D00083C6AB993547FD8A639EE61EA389BA04FC
:10A5E000634B061C83C5AB9993F6F50163006021AC
:10A5F0003D476380E6228944638A96260D49638637
:10A60000263B1146638BC63C0546639DC642A54664
:10A6100063EAA6443315A6001375053B6304A04402
:10A6200013D565006314C50C83C55A056370B50C5A
:10A630009305E0022685A38ACA04EF706F8103C6E2
:10A640005A056599A68563049600931516004D8DED
:10A6500037090680232CA90A9305400F2685EF6051
:10A660003FFF83C55A051375F5FC92054D8D2328D0
:10A67000A93C3705F87F3707F87F3708F87F1305BF
:10A6800065241307972213083826834525000346BF
:10A69000350083C64A098347370083482800BD89AF
:10A6A0001376E60F93F6E60F93F7E70F93F8F807A4
:10A6B0002301B500A301C500238ADA08A38A0A088A
:10A6C00023AC0A08238E0A08A301F700230118010E
:10A6D000EF609FFD631C95003705F87F1305552E2D
:10A6E0008345350093F5E50FA301B500EF60DFFB6F
:10A6F000631995023705F87F93152B003716F87FFD
:10A700002301652713F5C53F930524001306467DF5
:10A7100001A8838605007D152300D6000506850562
:10A720006DF9034554009375050C8DE983C95A05ED
:10A73000137915009305000F2685EF607FF193755F
:10A74000F5FD2E86639499001366050201456303A7
:10A75000A900B285370506802320B53C0345540087
:10A760009375250003D58A0589C513654500239C8B
:10A77000AA0483C5AB991365051093F50502239CC4
:10A78000AA0481E50545EFE06FA013052400EFF072
:10A79000EFED3705F87F0345B5520589636EA02AB2
:10A7A0001305800275AC03A54A009D45631DB500E5
:10A7B0001305600219A803C55A058945631CB50035
:10A7C000EFF0FFD201A813055002EFE0AFA401455E
:10A7D000EFE0CF830244924B224BB24A424AD24925
:10A7E0006249F24492501301810282801386F6FF7F
:10A7F000C94663E7C63EB74601000A069386C6F01F
:10A8000036961042028603C52A00058961F549463D
:10A8100065A303C5AA0593758500636AB02203A5E5
:10A820000A0605497D156364A90023A00A0613558D
:10A8300026007189136625003725F87F9304A59DAE
:10A8400081462685A285EF70DF8703053400634DBE
:10A85000054009449305000F2285EF607FDF0589DD
:10A8600035F903C55A05630C854CADB7930924002F
:10A87000114A814459464E85D285A686EF70FFB4B1
:10A880003705F87F130935264A85CE855286A68678
:10A89000EF703F8305456319AB1E83C52A00858988
:10A8A0006304B01E83C5AB9903C65A05998163FF43
:10A8B000C50A639DA50A8949A38AAA049305E002F3
:10A8C0004E85EF60FFD803C65A056599CE856304AF
:10A8D0003601931516004D8D370A0680232CAA0ADF
:10A8E0009305400F4E85EF60BFD683C55A0513759B
:10A8F000F5FC92054D8D2328AA3C3705F87F3707D4
:10A90000F87F130565241307972283452500034626
:10A91000350083C64A098347370003482900BD89AB
:10A920001376E60F93F6E60F93F7E70F1378F80721
:10A930002301B500A301C500238ADA08A38A0A0807
:10A9400023AC0A08238E0A08A301F700230109019A
:10A95000EF609FD5631C35013705F87F1305552E31
:10A960008345350093F5E50FA301B5008309440045
:10A97000094403C95A059305000F2285EF605FCD96
:10A980009375F5FD63C9990E2E85630389002E85A5
:10A99000B705068023A0A53C3705F87F0345B552CF
:10A9A000058979ED1305700201B9EFD03FDF9305FA
:10A9B000B00DE3E1A5E203455400930500081375CB
:10A9C000050F6304B52E93050005E315B5E03705C3
:10A9D00006809D452320B514F5BB03958A05930495
:10A9E000240013650501239CAA042685EFF00FC8F7
:10A9F00003455400098919C503958A051365450067
:10AA0000239CAA0403C52A000D8963182501039518
:10AA10008A0591654D8D239CAA0413152B000144D2
:10AA20009375C50F05462685A286EF701F9A03A56C
:10AA30004A00F945E310B5DA03C52A000589631910
:10AA400085045DAE03C55A05630B952EA1AE137543
:10AA5000750F238DAA04BDBBEFD0CFAE13059002B6
:10AA6000EFD05FFB93152B0001461305240093F5EF
:10AA7000C50FB286A9A613650502E30B89F001BFD5
:10AA8000EFD0AFE1630AA02E01459145EFE03FA46E
:10AA900075451DB699456300B53EA945630BB542A2
:10AAA000FD456303B54493050002630DB54493056A
:10AAB0005002E311B5D2A5A299456308B530A94566
:10AAC000630CB53093050002630BB532FD45E3130B
:10AAD000B5D0454585450146EF709FA303C52A00C3
:10AAE00005895DF511AE95456301B5529305D00218
:10AAF0006306B542B545630DB5509305300263005A
:10AB0000B544930540026302B548B1456316B54AA2
:10AB10003545EDA903C52A00058901E93705F87F08
:10AB2000034595241375050245CD0145EFE01FB19E
:10AB3000E34205CA03C52A000589E30DA0C865459F
:10AB4000A5BC03C52A00058909C93705F87F034557
:10AB5000C522137505026307A0240145EFE01FC459
:10AB600095B93725F87F9305459583C5150085442C
:10AB7000639895008345459593F5E50F230AB594B1
:10AB800003C52A0005896360A0143705F87F0345D3
:10AB9000952435AAB725F87F1385459503461500FA
:10ABA00009456318A60003C645951376E60F238A68
:10ABB000C59483C52A00014685896385C516B705F6
:10ABC000F87F938595229DA203C52A00058909C9AE
:10ABD0003705F87F0345C52213750502636DA01A7A
:10ABE00003C55A058945630CB5146DAA9945630ED2
:10ABF000B520A9456308B516930500026304B51690
:10AC0000FD456310B5223725F87F8545B9AAB705FC
:10AC100000FF014523A8BA048D45EFE05F8BEFF0FC
:10AC20004FBC4DBE1306A002631BC50E03C52A0010
:10AC3000058909CD01458D45EFE07F896351A00E5F
:10AC40001305B002EFD01FDD83C5AB998144FD89A8
:10AC5000268513192B00EF70DF932A861305240035
:10AC60009375C90FA686A1AA034514001181937597
:10AC7000750013852400EFC07FADE30DA0B48345BC
:10AC800024001306000C63EFC51283C54A06630354
:10AC9000B03E8D453726F87F93060005230926959B
:10ACA00023A0BA0623AADA00C1AE83C52A0005454F
:10ACB0003726F87F85898146A380AA0A230806944F
:10ACC000E398D5DC15AA3705F87F0345C522098925
:10ACD00015CD09449305100F2285EF607F971375FA
:10ACE00005040DE5EF20804C09E5EF60FF9B630F45
:10ACF0008500EF20A04B631F9512EF60FF9A631B46
:10AD0000851203C52A0009896366A01203C5AA0635
:10AD100083C59A0622054D8D1375252041C513055F
:10AD2000600259B8B705F87F9385652483C535005F
:10AD300093F5050281E983C55A056395A50601458A
:10AD4000C1459DA001458D45EFE06FF803C52A0080
:10AD5000058931ED03958A05936585002D45239C72
:10AD6000BA0481A83725F87F89451306C012A30AC3
:10AD7000B59423A8CA0275A0EF20404319C9EF205B
:10AD8000A04301C9EF605F92631585000545EF2080
:10AD90008043694515B00945F145EF607F8B058912
:10ADA000636EA02A01459145EFE06FF225B41305CB
:10ADB0001002EFD03FC641460145AA85AA86EF7032
:10ADC000CFE009BC23A02A0745AC01451946AA8556
:10ADD000AA86EF708FDF0DA009459305100FEF6075
:10ADE0003F8713654500B705068023A2A53C414572
:10ADF00085450146EF70CFF121456FF0EFFB4145EE
:10AE000085450146EF70CFF061B13725F87F8D455C
:10AE10001306C012A30AB594214523A8CA02EFD095
:10AE20007FBF3725F87F8305459593E51500230AF5
:10AE3000B5944DB203C5AA0683C59A0622054D8D69
:10AE400013752520E36DA0EC01458D45EFE02FE85B
:10AE5000E342059883958A0503C52A0093E585009A
:10AE600013762500239CBA046361C0261365250070
:10AE70002381AA00A5A401451546AA85AA86EF70DC
:10AE8000CFD409459305200FEF608FFC15C9094405
:10AE90009305200F2285EF60AFFBB705F87F938401
:10AEA00045522386A4009305300F2285EF604FFAA8
:10AEB000B70506802387A40023A4053C238604004D
:10AEC00003958A05936505041D45239CBA046FF01C
:10AED000AFEE03D58A05C1659385F5FB6D8D239C87
:10AEE000AA042D456FF04FED0545EF602FF503C522
:10AEF0002A0093752500636DB01813652500238122
:10AF0000AA0045A203D58A05C1659385F5FB6D8D21
:10AF1000239CAA04130510026FF00FEA03C59A06DA
:10AF2000B70500FF1375150223A8BA0419E50395A8
:10AF30008A0513658500239CAA047D4589A003C565
:10AF40009A06B70500FF1375150223A8BA0419E580
:10AF500003958A0513658500239CAA043725F87F8D
:10AF60000345058001CD09459305100FEF604FEEB5
:10AF700013654500B705068023A2A53C41458145E0
:10AF80002E86EF70EFD8154551A00945F145EF60C9
:10AF90002FEC05896305A0120945F145EF604FEBE1
:10AFA0007999B7050680A8D9814503C52A00058986
:10AFB0006304B510754511A203C52A00058929E966
:10AFC00009449305C00F2285EF608FE813650501E2
:10AFD000370906802328A93E9305D00F2285EF600C
:10AFE0002FE741891DE109449304E00C2285A685E1
:10AFF000EF600FE613654500232CA9322285A68554
:10B00000EF600FE56D99232CA9322145EFD09FA069
:10B010003705F87F130445520345C4009304000527
:10B02000330595026549B3552503B70906800945DF
:10B0300013F6F50F9305300723A4C91CEF604FE109
:10B040008345C4007199B3859502B3D52503A181C9
:10B050008D894D8D23A6A91C6FF0CFF701458D4535
:10B06000EFE0EFC66358A0F613054002EFD09F9AB9
:10B070004D4699B323A00A0683C55A050946A38203
:10B08000AA066399C5F40385AA0513650504D1B220
:10B090009375D50F09652381BA00EF809FA403C57E
:10B0A0002A0005810589EFD07F8E01444545A285A0
:10B0B0002286EF70EFC549B22145EFD0BF9581459B
:10B0C0004D452E86EF70CFC4A1B79375D50F096596
:10B0D0002381BA00EF80FFA003C52A0005810589FE
:10B0E000EFD0DF8A014445462285A285A286EF7013
:10B0F000CFAD03C52A009375250099E583A50A06FF
:10B100006394950023A00A0683D58A0531667D16CF
:10B11000F18D0589239CBA04E31C8596F1B92111B0
:10B12000B725F87F06CA4AC41389A59903461900B2
:10B130003725F87F26C69304858003C544059356BA
:10B1400016009D8A22C2630BD51C131586016185EA
:10B15000238AD404634005141355460003C6A599F9
:10B16000937575001375F601630FB0143D466315B2
:10B17000C51683C6D4058A05130529005146EF700C
:10B18000CFA403053900635B051803452900930527
:10B1900010041375F50D6313B51803452901937554
:10B1A000050613050004638BA516B705F87F83C554
:10B1B00085223706F87F856785681306A6229306E1
:10B1C00000082947938797BB1308C00293888838E3
:10B1D0008D4215439303000C130E200355A8834E94
:10B1E000260013FF0E0C6306DF006308AF02636DD9
:10B1F000E007834E0600834FF6FF13FF3E00220F49
:10B20000336FFF01330FEF026362FF0893FECE0F2F
:10B2100093EE1E00A30F06FFA9A0920E034F160087
:10B2200093FF0E3F834E0600135F4F0033EFEF0195
:10B2300093FF3E008340F6FFA20FB3EF1F00B38FD2
:10B240001F03B3DFEF0363E3FF04330F5F02335FDA
:10B250006F0293FECE0F935F8F00B3EEFE01A30F3C
:10B26000E6FF2300D6011DA093FE0E0F63907E0221
:10B27000834EF6FF13FFFE07330FCF036368FF0013
:10B2800093FE0E0893EECE03A30FD6FF1106FD1515
:10B29000B9F569A003C6540589466311D60883C56C
:10B2A000A5992D46FD896385C5001D466396C50297
:10B2B00003063900FD561304290063C2C604098140
:10B2C0001379C50189A0C1456306B5028D45631593
:10B2D000B500014515460DA003C554058945631FFA
:10B2E000B5020145C14585472A86AA862A87EFE02F
:10B2F0000FF02DA0014571468546AA8531A80305AA
:10B300002900130925000545EF70AFA883C6D405B1
:10B310002A869375F90F2285EF702F8B12442249EC
:10B32000B244D2406101828021113725F87F06CADC
:10B330004AC4130985800345990626C64EC222C019
:10B340001189630FA020034529000989636AA020A1
:10B35000EF40604E29CD0545231609062307A906AF
:10B36000EF40404F09449305C00F2285EF604FAE78
:10B3700013650502B709068023A8A93E9305800F2F
:10B380002285EF60EFAC6D999304E00C23A0A93EF9
:10B390002285A685EF60CFAB1365450023ACA932AB
:10B3A0002285A685EF60CFAA6D9923ACA932EF4024
:10B3B00020490DC90345E90655C9131615008355E3
:10B3C000C9069306E6FF0947B316D700ED8EC5EA16
:10B3D0008D463396C600D18D11462316B906637D7E
:10B3E000A60871A8EF40604649CD0345E9068D45A2
:10B3F00013161500B395C5008316C90693C5F5FF4E
:10B40000F58D85463396C600D18D11462316B906B3
:10B410006365A60005052307A906EF40E04409443B
:10B420009305C00F2285EF60AFA213650502B7092F
:10B43000068023A8A93E9305800F2285EF604FA1C7
:10B44000136545009304E00C23A0A93E2285A68540
:10B45000EF600FA01365450023ACA9322285A685B5
:10B46000EF600F9F6D9923ACA93221A88315C906FF
:10B4700093E535002316B90605052307A906EF4015
:10B48000003E0325890219E50305A9061365450059
:10B490002305A9060325090661E50345E90669C1F7
:10B4A0000345A90611894DCD3706F87F0345590597
:10B4B000834646278357C9061304462713452500AC
:10B4C00093F6F60703471400139877001335150019
:10B4D000B366D80013D81700B725F87F1605137781
:10B4E000E70F137818009389A59D9305F00F854405
:10B4F0003367E800194813651508858BA382B900E6
:10B500002381090123829900A381A900230AD62659
:10B51000A300E40081E71305001019A0130500083B
:10B52000EF802FDC0345C906098909C513050020F2
:10B53000EF802FDB1385690011468146A285EF60FD
:10B540005FB80355C9068305E9060981FD1509465B
:10B550002316A9062307B906A302C90623209906C4
:10B56000024492492249B244D24061018280372587
:10B57000F87F8345A59F3726F87F93F5750F230243
:10B580000686230DB59E8280211106CA26C68944EF
:10B59000F54526854AC44EC222C0EF606F8B0D89E7
:10B5A00063149500854409A8F5452685EF604F8A08
:10B5B0003189A145631AB50A05443729F87F2285E8
:10B5C00023049980EFD0EFC02285EFD02FBC8944AF
:10B5D000F1452685EF60CF877999B709068023A8C2
:10B5E000A906EF10B03C19C5EF600F8C63149500ED
:10B5F000094511A01545EFD01F8183448980094575
:10B60000E545EF60EF84639C84009375E5FF094591
:10B6100023A2B906E545EF60AF83799919A8936530
:10B620001500094523A2B906E545EF606F82136551
:10B63000150023A2A9063725F87F8345A59F130689
:10B64000898093F5750FB946230DB59E230E060428
:10B6500054CE0345898063148500054511A0094532
:10B66000EF802FC8014531A03725F87F23040580DE
:10B670000545024492492249B244D2406101828088
:10B68000211106CA26C64AC44EC222C0EFD00F916D
:10B69000930590096361B5060944F5452285EF508D
:10B6A0003FFB0549937535004A8589E9F5452285B3
:10B6B000EF501FFA9375C500228595CDB724F87F0A
:10B6C00001442384A4802285EFD0AFB02285EFD03F
:10B6D000EFAB83C984800945E545EF507FF7639E52
:10B6E00029017999B7050680E8D10945E545EF506C
:10B6F0003FF6799931A805448DA813651500B70563
:10B700000680E8D10945E545EF509FF41365150023
:10B71000B70506803726F87FE8D113898480034572
:10B72000A69F230E09041375750F230DA69EEF50D7
:10B73000BFF709C937051400130635302945A1455F
:10B74000EF606FEA03158905B94513658500231C71
:10B75000A904232EB900854503C584806314B50070
:10B76000054511A00945EF80CFB7228502449249D3
:10B770002249B244D24061018280211106CA22C00E
:10B780002A840945F54526C64AC44EC2EF505FECEF
:10B790003D8911C53725F87FB9452322B582372564
:10B7A000F87F130985800325C9013DC10945F54589
:10B7B000EF501FEA3D891DE9D1490944F54413F5CD
:10B7C000F90F19C92285A685FD19EF507FE83D893B
:10B7D0007DD513F5F90F19E93705F87F03055552A3
:10B7E000130585071375F50F2328A9000325090103
:10B7F0001DE1EFC0BFFA93059009636EB500EFD06D
:10B800008FEBEFF0FFE701E91545EFD0AFA021A0E6
:10B810002285EFE01F80024492492249B244D2407F
:10B8200061018280211106CA22C209449305B00A2F
:10B83000228526C64AC4EF50BFE113652500B70430
:10B84000068023A6A42A3725F87F1309858003558F
:10B850008905C1659385F5FD6D8DB725F87F231C9E
:10B86000A904232C0902A3810580EF50FFE3631A8A
:10B8700085001545F145EF50BFDD3D99B7050980BD
:10B88000A8D90945F145EF50BFDC3D99A8D803057B
:10B89000A905124413652500230DA9042249B244C9
:10B8A000D24061018280797106D652CC372AF87F66
:10B8B00026D24AD04ECE56CA5AC822C693098A808A
:10B8C00003A5090211C909459305000FEF505FD880
:10B8D000098961C123A0090203458A8045C1EFE0BF
:10B8E000FF8803852909F9556308B5088944630D64
:10B8F000950685456314B50803A54900F54563051C
:10B90000B500A145631CB506EFB00FB325E903A54B
:10B91000090619C93725F87F0345C59D930500041D
:10B920001375050C630CB50403C5390983C50909F2
:10B930001376F501158105449306260093771500CB
:10B940001386290701452287EFE06F8A03853909AD
:10B95000634405023725F87FF94523098594238937
:10B96000990823AAB90019A83725F87F034525951A
:10B9700011C503A5490119E12389090803A5890116
:10B980001DC103C5C9058545630FB5000145EF60BD
:10B99000BFCA3244424BD24A624AF24902599254D7
:10B9A000B2504561828003458A806308A02A83A53E
:10B9B00009067959638925030D456388A50409455E
:10B9C0006388A506854A6390552183C5590563950B
:10B9D000A50A0945F545EF50BFC7418949E5EFD0B4
:10B9E0003F8849E551A803C55905894523A00906A3
:10B9F000631BB51C03C5A905937505046305B01C3D
:10BA00001375F50B238DA9047DAA3725F87F03450F
:10BA10002595630AA01A03A549016366A01A038548
:10BA2000490685457D1523A0B9062382A90661AA8A
:10BA3000B725F87F83C525956307B01883A549010D
:10BA40006363B01883C5290023A00906898999C5B5
:10BA50008385A90593E58500238DB90483C5590520
:10BA6000E38AA5F88DA2EFD05F8419E503C5A90587
:10BA7000137505046309A01403A549009545630BDC
:10BA8000B500A145630DB500F545630AB500E14574
:10BA9000631BB512A14523A009066316B51209441C
:10BAA0009305E0082285EF50BFBA9375050803C5DA
:10BAB000C905636CB010630A5511038529097D150A
:10BAC0001375F50F6361851003C52900838559053A
:10BAD000131645009A05058993F5050C22054D8D31
:10BAE00083C5090513760602518D9D8903C6590643
:10BAF000A6054D8D93757600B2054D8D9365F500C5
:10BB0000B726F87F21819384A69D238DB69C83C59B
:10BB10009906A380A40013152600136525008D81C6
:10BB200093F635001376E50F0145A685EFD0FFA10A
:10BB30006346050203853400634C050203C55905BD
:10BB400023A00906631B850603C5A9059375050493
:10BB5000A9CD1375F50B238DA90481A8FD55631696
:10BB6000B50003C5290009891DED23A0290735A8C3
:10BB700003C52400B725F87F1376E5019146238994
:10BB8000559523A089066305D600F1453D4621A0C1
:10BB9000930540066546930600046363D500B285AD
:10BBA00023AAB90019A023A0590703C55905631694
:10BBB00085001305400623A0A90403C59906137543
:10BBC000750EA384A90603C5C90505496314250993
:10BBD000B724F87F03C5A49F238E090493758500BD
:10BBE000A9E9118925C93725F87FB70506800944D9
:10BBF0001305A5999385850C7946A286EF606FCCD5
:10BC0000930510032285EF50BFA41D895DC509442B
:10BC1000930510032285EF50BFA31D89631A250BDE
:10BC200003C5A49FA38E29051375B50F238DA49E6C
:10BC3000C1A089451375750FA305B100238DA49E7E
:10BC40001305B10085451306200F8146EF60EFF71D
:10BC5000EFE00FA50145EF603F9E83AA49009305E1
:10BC6000F0021385FAFF63F4A5006F1040493746D0
:10BC700001000A05130686F53295104103A58900D7
:10BC800002868544631495006F1060470944E945B6
:10BC90002285EF50FF9B1365F500B70506806546CA
:10BCA000B726F87F3727F87FA8D523A6C90023AE8B
:10BCB000869E230897946F10804403C5A49FA38E8B
:10BCC00009041375B50F238DA49EEFE09F8559B726
:10BCD000930510032285EF50BF9783C5A49F1D894C
:10BCE00093F5B50F238DB49EE31685F6A38E8904D4
:10BCF000EFF0EFC285B78945E30DB53CEFC03FDEFD
:10BD000001442285EFC0FFCC2285EFC03FC8238BC2
:10BD10000904EFC09FD70944F1452285EF505F9396
:10BD20007999B7040680A8D8EF104048E30FA034F3
:10BD3000EF509F97E31B853409456F0030358D45E3
:10BD4000630FB5003705F87F03055552B945130554
:10BD500085071375F50F23A8A90023AEB900054583
:10BD6000EFF0BFA16F10A0399145E305B5520395DF
:10BD700089059305A02813658500239CA904238FBA
:10BD8000090423A6B900894503C56905E369B54ED1
:10BD900015456F00104F95456314B5006F102036A0
:10BDA000EF10C040E308A034EF501F908945E31323
:10BDB000B53409456F0090341944631485006F1041
:10BDC00000340145238B0904EFC05FA403C5690655
:10BDD0008945E366B550238489066F0030529D453E
:10BDE0006314B5006F10A0310145EFC03FA203C539
:10BDF00069068945E368B55031452384A9066F007B
:10BE0000905183C5190A0544639485006F10202F53
:10BE1000A1456305B5002145EF70BFCCEF10003997
:10BE2000E302A01603A5C902E36EA014EF50DF875A
:10BE30008945E319B514EF1000419305E00BE36366
:10BE4000B51409456F001016A5456314B5006F10B1
:10BE5000002B03D58905BD65FD156D8D239CA904B7
:10BE600001459D45EFD0AFE67145A1456F00904C6F
:10BE7000A9456314B5006F1080280145A945EFD08E
:10BE80000FE5635405006F10802703D58905B96558
:10BE9000FD156D8DF1452146B5A30545EFC07FB376
:10BEA00031456F108025B1456314B5006F10202512
:10BEB000130500328DAFB545E316B506EF10E0353A
:10BEC00019E16F10C0230145EF100036EFC01F8D40
:10BED0009305900B6374B5006F10602239456F10A5
:10BEE000C021B9456314B5006F1060210145994523
:10BEF000EFD0EFDD2A8485443725F87F2300958035
:10BF0000E348044A814541452E86EF606FE003C552
:10BF10009906B70500FF058923A8B904A38B090476
:10BF200019E50395890513658500239CA90413056C
:10BF30002003E1453726F87FB726F87F23A6A9001E
:10BF4000232EB69E238896946F10601BBD45E30C8C
:10BF5000B526EFC0DFB80944F1452285EF504FEF19
:10BF60007999B7040680A8D8EF104024E303A020F5
:10BF7000EF508FF3E31F851E09456F00B01FC145C9
:10BF8000630FB500394523AEA9003705F87F0305D7
:10BF90005552130585071375F50F23A8A900094409
:10BFA0009305000A2285EF50AFEA418905E1F54586
:10BFB0002285EF50EFE90D89630A85000945F545B3
:10BFC000EF500FE93189A1456315B500394523AE1E
:10BFD000A90003A5C9016367A06A09459305000A82
:10BFE000EF500FE74189636FA06801458DAFC545EC
:10BFF000630CB5003705F87F030555521305850717
:10C000001375F50F23A8A9003725F87F034565951B
:10C0100009446316857209459305000AEF504FE302
:10C02000418919C93705F87F03055552130585075E
:10C030001375F50F23A8A90003A5090119C16F10F5
:10C04000000C29AFCD456314B5006F10400B3725A8
:10C05000F87FB705F87F2302058003C57552930565
:10C0600030023D893385A540D1456F00B02CD145C4
:10C07000E307B518EF108013E300A018EF50CFE2EC
:10C080008945E31BB51609456F003017D545631484
:10C09000B5006F10C0063725F87F094423020580DC
:10C0A0009305F0022285EF50AFDA137505F8B70457
:10C0B000068023AEA40A9305F00F03958905239803
:10C0C000090423890904A389B904A38B0904F14550
:10C0D00013658500239CA9042285EF506FD7136553
:10C0E0000501A8D8EFD02FB4E304A02E11456F00AE
:10C0F000502ED9456314B5006F1060008944930534
:10C10000900F2685EF50CFD4098955C503C5290066
:10C1100003C65905931525000544A189A28663032A
:10C120009600B2860589139616004D8D518D370BFA
:10C1300006801309F002232CAB0A2685CA85EF502E
:10C140002FD113651502232EAB0A2685CA85EF5021
:10C150002FD013652500232EAB0A3727F87F03C5A0
:10C16000590583C51905131665009D891376060CBC
:10C17000A605D18D0566134525003D06133515002E
:10C180004D8E1605935686009305A79D13650508E9
:10C190009307F00FA380D500230DC79CA381A500B2
:10C1A00001451946A286A382F500238185002382DA
:10C1B0000500EFD08FB913056009DD456F009017BA
:10C1C00009459305F002EF50AFC8137505F8B705A0
:10C1D00006801306F00F23AEA50A239809042389CD
:10C1E0000904A389C90461456F003071E145E30585
:10C1F000B52E03C599050589E300A02E0565130535
:10C20000853823A6A900894503C56905E36BB52ACE
:10C210003D456F00502BE545E303B56E0145EFC08A
:10C22000EFDE03C569068945E36AB50E154523842B
:10C23000A9066F00D00FE945E303B56C01458D45B4
:10C24000EFD0EFA8E34D056A0145EF00F07D0395BF
:10C250008905B705F87F13650504239CA90403C568
:10C26000855295451D893305B50293053002338506
:10C27000A540ED456F00100CED456316B54EEF007F
:10C28000D079E30EA0660145EF00107AEFC00FD120
:10C2900093059009E365B56671456F001066014529
:10C2A0009945EFD0CFA22A846341045C1305600452
:10C2B00085453726F87F23ACA902A301B680A38A5F
:10C2C000090823AC0908238E090861A603852909FA
:10C2D00089447D151375F50FE363956203C5190A4B
:10C2E0000549E30E256103C55905E31A953E03A5EB
:10C2F000890311ED3725F87F8345358089C98395FA
:10C300008905A301058093E50502239CB90403A5D3
:10C3100009067D15636E95000385A905634A05002E
:10C3200003D58905B965938505026D8DE30FA038A6
:10C330000145EFC0BFEDEFC0BFF2E362A05C6F004C
:10C34000103AF945E30DB55A0385290989457D154C
:10C350001375F50FE365B55A814421442685A285FE
:10C36000EFD0EF96E35DA05803D58905C1659385AD
:10C37000F5FD6D8DF145239CA90423A6B90003C5E5
:10C38000290005896303950075443725F87F8545A5
:10C390003726F87F232E859E2308B6946F003056EB
:10C3A000FD45E30EB55403C5C9050544630385DEA9
:10C3B0000145A545EFD0AF91E343055403D5890569
:10C3C000B16503C62900FD156D8D93751600714684
:10C3D000239CA90423A6C900E368B01E21456F0071
:10C3E000D01E93050002E30CB5500145A945EFD0DE
:10C3F0000F8EE346055003D58905B965FD156D8D92
:10C40000F1457546B726F87F0547B727F87F239C87
:10C41000A9046F00301A93051002E302B54E3705E8
:10C42000F87F0345855295451D893305B50293056F
:10C4300050023385A54093052002EDAD93052002FF
:10C440006317B532EFC08FB5E145E3EAA54A13059E
:10C4500030026F00904A93053002E302B54A01446E
:10C460002285EFA09F9A2285EFC0AFD699452285FD
:10C47000EFD0EF856357051AF955E31BB52071A777
:10C4800093054002E30DB5460945F145EF504F9C39
:10C490000589636DA06A03C5290081450589631A72
:10C4A000B51A21456F00704593055002E309B54464
:10C4B000B70500FF014523A8B904B545EFD02F818A
:10C4C00063570566B725F87F03C5A59F1376750FDB
:10C4D00013056002238DC59E6F00304293056002F4
:10C4E000E30FB540038569050505238BA904EFA07B
:10C4F0005F8B85451305A1001306200F8146230598
:10C50000B100EF509FECEFD0BF996F00503F930503
:10C510007002E306B53E5945E94529AD9305800211
:10C52000E30FB53C59459305900229A59305900268
:10C53000E307B53C0145EFD0EFB3E352A03C37151C
:10C54000F87FB705F87F1305057F938535261146DB
:10C550008146EF501FB719456F00303A9305A0028E
:10C56000E30FB53803C559058945E31AB538494580
:10C57000F5453726F87F85463727F87F23A6A9009B
:10C58000232EB69E2308D794EFC0FFE901C50545C9
:10C59000EFC07F873705F87F930520032308B55246
:10C5A0006F00F0359305B002E30BB53403C55905B0
:10C5B0008945E316B5341305C002B725F87F054653
:10C5C000B726F87F23A6090055A303C55905894559
:10C5D000E317B532EFC08F9C9305B00DE3E1A532B0
:10C5E0001545EFC05F821305D0026F00103193052F
:10C5F000D002E306B53003C559058945E311B530CE
:10C6000001442285EFC0EFBC2285EFA01F80994531
:10C610002285EFC0DFEB9305401F23A6B9026343D9
:10C62000055E1305801B85453726F87FB726F87F02
:10C6300023A6A900232EB69E2388B6946F00302C23
:10C640009305E002E30DB52A03C529000589E30A35
:10C65000A0E475456F00702AE303B52A03C52900DD
:10C66000F145058923A6B900636CA04E2145D5A9E3
:10C67000EF00D03349CDEF502F8389456319B508BA
:10C68000094551A83729F87F13046995834414009C
:10C690000945F545EF40DFFB3D896303950237050A
:10C6A000F87F8305555209459385850713F6F50FE5
:10C6B000F54523A8C900EF40BFF93D89A300A400B8
:10C6C00003A5090109C503C5B905E30AA022094567
:10C6D000F545EF40FFF70D8901E90945F545EF40C4
:10C6E0003FF731896309A0700944F5452285EF4081
:10C6F0003FF60D89854463139536F5452285EF4055
:10C700003FF531899145631BB534228BF5A5EFC008
:10C710009FD101C50545EFC00FEF0545EFC05FC6CE
:10C720006F00F01D0145EFC04FBF05442285EFA00B
:10C73000CFEDEFC05FCF630CA04C1145D1A9F545FB
:10C740002285EF40FFF00D89631A85000945F54504
:10C75000EF401FF03189A145E303B51A0545EFD03D
:10C760005F8B6F00D0191305201CF145E1A6EF0087
:10C77000F0236303A02CEF403FF38945631EB52AE5
:10C78000094565AC15459305000FEF407FEC137527
:10C79000050809C503C5690A058919E5EFC0BFC8C1
:10C7A00001C50545EFC02FE6EF00502039CDEF0061
:10C7B000B02021CD03A5C90229E9EF40FFEE89454C
:10C7C0006315B504EF0030289305E00B636FB502E5
:10C7D00003C52900058915E903C5990513750502E7
:10C7E0000DE53715F87F0345757D1375050211CDED
:10C7F00009459305100FEF40BFE5118919E5039531
:10C80000890589654D8D6F00100E03C55905094BCB
:10C8100063166501EFC07FA9E303A00E03A5090617
:10C82000E30F650D038529097D151375F50FE36881
:10C83000650DB724F87F03C5449593751500630211
:10C84000B07E83A50903636EB07C1389449583454C
:10C8500019000D466384C57A6389657B639D857A7B
:10C860008395890511666F00A07A1545EFC0AFD991
:10C870000945F145EF40DFDD7999B7050680795626
:10C88000A8D96317C4606F0090071545EFC0AFD7F4
:10C8900009459305F002EF40BFDB137505F823AEA1
:10C8A000A40A0145AA85EF500FDE1544C145228533
:10C8B000EF401FDA13651500B7040980A8C0C94509
:10C8C0002285EF40FFD8799993058002A8C423A858
:10C8D000B9000945F545EF40BFD73D8901C50D4574
:10C8E0006F00B00103A50901E36BA0000545EFA0AF
:10C8F000CFD179ABEFC03FB301C50545EFC0AFD095
:10C900000965EF700F9E03C5290003C659059315ED
:10C9100025000944A189631386000546058906069A
:10C920004D8D518DB704068023ACA40A9305F00207
:10C930002285EF40FFD11365150223AEA40AEFA0B4
:10C94000BFC80145EFB09FEC1305F00FA389A90400
:10C95000F1452285EF40DFCF13650501A8D803C557
:10C9600069056300A02E636BA42E05651305853849
:10C97000C1A21545EFC02FC909459305F002EF404C
:10C980003FCD137505F8054423AEA40A2285EFC0F8
:10C990004F842285EFB09FFF0145AA85EF50AFCEAF
:10C9A0001544C1452285EF40BFCA13651500B70481
:10C9B0000980A8C0C9452285EF409FC97999F945EA
:10C9C000A8C423A8B90009449305000A2285EF40B2
:10C9D0003FC8418905E1F5452285EF407FC70D89B4
:10C9E000630A85000945F545EF409FC63189A14599
:10C9F0006310B538414511A71545EFC0CFC0EFB062
:10CA0000FFD99305000263ECA56E3725F87F8345B7
:10CA100045806366B06E930560315546B726F87F52
:10CA20000547B727F87F23A6B90023AEC69E238803
:10CA3000E7942302E580E1A51545EFC0CFBC37059B
:10CA4000F87F034565529305800C09810D893305F4
:10CA5000B5021305250393053002E9A8F5452285A3
:10CA6000EF401FBF0D89631885100945F545EF405C
:10CA70003FBE3189A1456310B5100D4BB5AE13050E
:10CA80006002B725F87F0546B726F87F23AEA59E3E
:10CA90002388C694EFB09FD09305800963E5A50273
:10CAA00003C5E9050DE105459305B04F0946B726D5
:10CAB000F87F3727F87F238FA90423A6B90023AE78
:10CAC000C69E2308A794EFB07FCD930590096368B5
:10CAD000B56203C5E9056304A062154539AD9385C8
:10CAE000690613071500B386A5001376F70F85476F
:10CAF000A38086002383E90663FCC728214523849D
:10CB0000A90671AC93856906AA9531460505A380EF
:10CB1000C5002383A9061305401F19A8938569063C
:10CB2000AA9515460505A380C5002383A90671456E
:10CB3000930560023726F87F85463727F87F23A6BE
:10CB4000A900232EB69E2308D79455AB13054006A3
:10CB500023A6A900814503C529000589E308B5B0CE
:10CB60007545B725F87F0546B726F87F23AEA59E05
:10CB70002388C69469A3F5452285EF407FAD0D89D2
:10CB8000114B630B85260944F5452285EF405FACC8
:10CB90003189A1456302B5269305000A2285EF403D
:10CBA0003FAB418981456303B500A284268BA9A4CC
:10CBB000230005800145EFA04FA5EF00205F630A29
:10CBC000A00EEF407FAE89456315B50E0945DDA087
:10CBD0000945EFC04FA30945F145EF407FA7136515
:10CBE0001500A8D80145EFB05FF3EF40FFAB09C9CE
:10CBF00037051400130635302945A145EF50AF9E87
:10CC00005945E5A9F955631EB51A0545FDA1094524
:10CC1000EFC06F9F3705F87F0345655293052003EA
:10CC20000D893305B50213052503B9453726F87F6D
:10CC3000B726F87F23A6A900232EB69E23888694C4
:10CC40007DA93705F87F034585529305C0F90D810D
:10CC50000D893305B5021305251CD9BD03C59905FA
:10CC60000589636DA0160945F545EF407F9E0D8946
:10CC70008545130440386303B5348944F54526855A
:10CC8000EF401F9D31899145630AB532F5452685F0
:10CC9000EF401F9C0D89630195320945F545EF4032
:10CCA0003F9B3189A1456309B5300565130485BBF8
:10CCB00031A61545EFC02F9579556302A444094567
:10CCC0002DA913056002B725F87F0546B726F87F22
:10CCD00023AEA59E2388C69403C579059305500409
:10CCE00063EFA54003C5290003C659059315250028
:10CCF0000944A189631386000546058906064D8D02
:10CD0000518DB704068023ACA40A9305F002228556
:10CD1000EF401F941365150223AEA40A0145EFC02E
:10CD2000FF91634D0502654523AC0900EFB09FCE2E
:10CD30000395890583C5590513650510239CA9042E
:10CD4000239B0904639D853A0945E945EF405F90BF
:10CD50001375F5FC13650501A8D455A6038579055F
:10CD6000930560090505A38BA90423ACB90041AE66
:10CD700003A509016365A03809459305000AEF4042
:10CD80003F8D4189636DA0360145EFA00F8805BF37
:10CD9000B29521460905A380C5002383A9066145F4
:10CDA000F14513066002B726F87F0547B727F87FDD
:10CDB0002384A90623A6B90023AEC69E2388E79440
:10CDC0003DAE1305600215AE7545B725F87F3726D1
:10CDD000F87F23AEA59E2308869415A60565130546
:10CDE0008538B725F87F0546B726F87F23A6A90022
:10CDF00023AE859EB5BB014B09449305B00F228538
:10CE0000230B6995EF40DF84AA84EF907FD463847D
:10CE1000A400EF905FE6034569959305E5FF63FB8A
:10CE20008500EF00A0383DC5EF401F8863148506DC
:10CE3000094595A09145631DB504EFC0CF87EFB0BC
:10CE4000FF9583C5090A1386050283C5B90563707A
:10CE5000A6066363B018EFB07F9493051002636970
:10CE6000B516EFB0BF939305700963E3A5160945A6
:10CE7000F145EF40EFFD13654500B7050680054617
:10CE800093062003A8D9A38DC90423A8D900A9A279
:10CE90003D45A5A41545EFB01FF70945F145EF4005
:10CEA0002FFB7999B7050680A8D94545B9A4E1CDEE
:10CEB000A38D09043705F87F03055552130585072F
:10CEC0001375F50F23A8A9001DACEFC06FB9630857
:10CED000250103A5090401E50545EFC02FB303A50E
:10CEE0000906630E9520038529097D151375F50F35
:10CEF0006367952003C559056316950403C5A90505
:10CF000009893DE5038549009145130565FD1375C4
:10CF1000F50F6369B502238E0908EFD00F9B154406
:10CF2000C1452285EF40CFF213651500370B09800C
:10CF30002320AB04C9452285EF408FF1136515000E
:10CF40002324AB043725F87F8345459513F6150058
:10CF50006309C01203A609036365C0121306459551
:10CF60008346160063832611639796108966FDA891
:10CF70001305A002EFB01FAA03C5A9051375D50FAD
:10CF8000238DA904ADAA0944F1442285A685EF406A
:10CF90002FEC6D99370906802328A9062285A685DE
:10CFA000EF400FEB136505012328A906EFE0CFDD65
:10CFB0006367A014554591A21304C05D0545A28581
:10CFC000EFC08F992145EF60DFB11305000335A253
:10CFD00003C5B9056305A01203A509016361A01289
:10CFE00009459305000FEF40AFE609810D899305D0
:10CFF00080023305B5022380A90A11A2130590020D
:10D00000EFB05FA103C5449539A0839589050966F2
:10D01000D18D239CB9041375E50FA3000900238A61
:10D02000A49403D589058965E98D95E19165E98D1C
:10D03000CDE18565E98D91ED9375050289ED8565F5
:10D04000938505806D8D45E9EFE00FAE4DA829452C
:10D050006DA025455DA003C5990605894DC179459B
:10D06000EFB05F9B03D589059DA89166039789055D
:10D07000D98E239CD90493F5E50FA3000600230A5B
:10D08000B59403D58905937505029DED8965E98DF4
:10D09000B1ED9165E98D95ED8565938505806D8D83
:10D0A00039E90545EFC0CFADEFE00FA8EF00001064
:10D0B00039C5EF00601021C5EF00C01229C1EF4053
:10D0C000AFDE6302959225A89375050189E979453C
:10D0D0002DA09375450091EDB165FD1521A0C165A9
:10D0E0009385F5FD6D8D239CA90411A813050002FD
:10D0F00029A07D4519A01305E002EFB0BF910345BB
:10D100008A8023A459010DC5B725F87F03C605956C
:10D1100003A5C90021C219C16FE0BF873725F87F79
:10D120000325C59F23880594EFB0DF8E6FE07F86CF
:10D1300003A5C90009C53725F87F232E059E03A541
:10D14000C90019E16FE0FF843725F87F23080594B3
:10D150006FE03F8419E16FE0DF833725F87F232EEE
:10D16000059E6FE01F83611106C2EF40EFD3854536
:10D170006307B500EF404FD389456314B500EFE076
:10D180008FF2EF406FD289456314B500EF10003184
:10D1900092402101828000003725F87F834545A019
:10D1A00093F5150C2302B5A06FA0CFB93725F87FF2
:10D1B000034545A0058982803725F87F034545A0B2
:10D1C000058105898280B725F87F03C645A0814681
:10D1D0006305D5001365460019A01375B60F2382A9
:10D1E000A5A08280B725F87F03C645A01355360059
:10D1F00005891376760F2382C5A08280B725F87F34
:10D2000003C645A081466305D5001365060119A034
:10D210001375F60E2382A5A082803725F87F03457B
:10D2200045A0158105898280B725F87F03C645A0F2
:10D2300081466305D5001365060219A01375F60D26
:10D240002382A5A08280211106CA4AC44EC2154974
:10D25000930900074A85CE8526C622C0EF404FBFFE
:10D260002A84930510074A85EF408FBEAA844A8519
:10D27000CE851374F40FEF40AFBD630FA400954447
:10D28000930500072685EF40AFBC2A84930510075D
:10D290002685EF40EFBBAA841395840013750530F3
:10D2A000C165418DFD15024492492249B244D240E4
:10D2B0006D8D610182807D71B725F87F06C622C21F
:10D2C000138485808345640A0605098993F5D50F83
:10D2D0004D8D2303A40A15459305E002EF404FB797
:10D2E0008345640A5D998A05A1894D8DB70509803A
:10D2F00023ACA50A1244B240416182807D71B725FA
:10D30000F87F06C622C2138485808345640A058996
:10D3100093F5E50FC98D15452303B40A9305E00283
:10D32000EF400FB38345640A799985894D8DB70520
:10D33000098023ACA50A1244B24041618280B7251E
:10D34000F87F9385858003A6850A23A4A50A630632
:10D35000A6003725F87FA308059482803725F87F3B
:10D360000345058B82807D7106C622C20544228555
:10D37000EFB0CFC9EFA05FE52285A285EFB06FD4F3
:10D38000EFF09FE11244B24041616FB0EF8F7D71C9
:10D3900006C622C205442285EF400F90EFF0BFFC85
:10D3A00081452285EFB0EFD11545E945EF404FAA01
:10D3B0001375F5FCB7050980A8D51244B240416148
:10D3C000828061113725F87F93058580054506C267
:10D3D0002382050A238D050EEFB0CFEE9240210186
:10D3E0006FF0FFFA130181FD3705F87F06D226CED4
:10D3F0004ACC4ECA52C856C65AC422C21309455214
:10D4000003457900058909ED13050005A5451306B7
:10D41000800C2308A900A308B900A307C9002DA008
:10D420000345F90009E51305800CA307A90003458E
:10D43000090109E5130500052308A90003451901A1
:10D4400001E52545A308A9003725F87F93048580C9
:10D4500009451544A38CA40E9305D00C2285EF40FA
:10D460002F9F6D99B709098023AAA9329305F00C63
:10D470002285EF40EF9D1365050123AEA932930588
:10D4800060022285EF40CF9C136505089305A00F2D
:10D4900023ACA90823A8B9349305000F2285EF40D7
:10D4A0002F9B41895DE99305E00C2285EF404F9A5F
:10D4B0001375F5FD23ACA9329305500F0345F90010
:10D4C000330A85022285EF40AF985295130AF03F48
:10D4D0006375AA001305F00F29A80305F900930549
:10D4E000500FB30A85022285EF408F96569513752B
:10D4F000F50F23ACA91C930570072285EF404F95CB
:10D500008345F900937AC5FF338B85029305500F4D
:10D510002285EF40EF935A956374AA000D4529A820
:10D520000345F9009305500F330985022285EF402A
:10D530002F924A9521810D89336555019305000885
:10D5400023AEA91C23A0B90415459305E00CEF40B8
:10D550002F901365050223ACA932054593050040C1
:10D56000EFB07FBD1305403D23A8A40E1244224B0B
:10D57000B24A424AD2496249F244925013018102AE
:10D5800082807D7106C622C201442285EFF0BFD29F
:10D590002285EFF0BFD63725F87F13048580032559
:10D5A000840A89452324B40A6306B5003725F87F29
:10D5B000A30805940145EF903FE837050980232231
:10D5C000040C2326053E1244B240416182807D71E5
:10D5D00006C622C22A841545E945EF406F8709C86F
:10D5E0001375F5FC13650502B7050980A8D535A0AC
:10D5F00013750503C1456302B5021545E945EF40C2
:10D600002F851375F5FC13650501B70509803726CD
:10D61000F87FC946A8D52324D68E1244B240416172
:10D62000828061111545E94506C2EF406F8213758E
:10D630000503930500026314B50005451DA01545BB
:10D64000E945EF40EF8013750503C1456317B50049
:10D650003725F87F0325858E01C51305F00F11A02E
:10D660000145620592406185210182807D711545E9
:10D67000F54506C622C2EF30BFFD0D898D45054434
:10D680006303B5021545F545EF309FFC3189B1457F
:10D69000630BB5001545F545EF309FFB0D898945B6
:10D6A0006318B500014422851244B2404161828072
:10D6B0001545F545EF30DFF93189A1456314B50013
:10D6C0000145DDB77D55CDB77D7115459305F00258
:10D6D00006C622C2EF30DFF7137505F8B7050980DB
:10D6E00023AEA50AEFF0BFCA3725F87F1304858063
:10D6F0000325840AD145136505016307B504034575
:10D70000640A9375E50F01452303B40AEF90DFD255
:10D710000545EFB02FBB0345640A058901E90145C2
:10D72000EFF07FB90325840A914539A00545EFF054
:10D730009FB80325840ACD452324B40A6306B500A7
:10D740003725F87FA30805941244B24041618280D6
:10D750007D7106C622C2EFF01FC13725F87F130482
:10D7600085800345640A9375150099C9154593058D
:10D77000000FEF30FFED1375050809E90345640A52
:10D78000058905E10325840A954521A00325840A1E
:10D79000E1452324B40A6306B5003725F87FA308C2
:10D7A00005941244B240416182807D7106C622C256
:10D7B000EF909FC81544E9452285EF307FE93D8908
:10D7C00063048500094511A03D45B725F87F938581
:10D7D000858003A6850A23A4A50A6306A60037252B
:10D7E000F87FA30805941244B240416182807971A8
:10D7F00006D64ECEB729F87F03C569A052CC094A98
:10D8000026D24AD056CA5AC85EC662C422C2630F24
:10D81000450D054B630865136363A016EF901FB1B8
:10D8200015449305D00F2285EF309FE29344F5FF16
:10D830009305C00F2285EF30BFE1658D0DC51544FE
:10D840009304E00C2285A685EF309FE01365450028
:10D8500037090980232CA9322285A685EF305FDFA6
:10D860006D99232CA9323725F87F930A858003C54B
:10D870008A0A91456305B510930560026301B510EE
:10D880003705F87F0345A5520989636AA00EEF901A
:10D890009F9F1544AA849305000F2285EF305FDB1C
:10D8A0001375050809C503C56A0A05896DE5EFF01A
:10D8B0009F999305800933BBA50003C56A0A0589B2
:10D8C0006369A0126367901213451B006363A01283
:10D8D00015459305B00FEF30BFD72A89EF909F8A87
:10D8E0006304A90E03855A0A0505C5A015449305CE
:10D8F000F0022285EF30DFD53726F87F137505F863
:10D90000B70509809304868023AEA50A2382040A02
:10D91000EFF03FABEF90AFC69305000F2285EF30DD
:10D920003FD31375050821E50145EF90FFB003A52E
:10D93000840A23A4440B630F45033725F87FA3080B
:10D9400005940DA83725F87F130485800325C40BA3
:10D950000DC5EFF05F8F9305700963E2A5020385A3
:10D9600069A005052383A9A0232E040A09A801455F
:10D97000EFF0BFE3238309A019A0238349A1124438
:10D98000224CB24B424BD24A624AF249025992545B
:10D99000B2504561828003C54A0A631B6501154583
:10D9A000F545EF30FFCA0D89E30945F103C54A0A81
:10D9B0006310450F1545F545EF309FC93189134573
:10D9C0008500133B1500D5BD01459375F50F130672
:10D9D0005006A382AA0A63EDC500EF90BF8EEF90B8
:10D9E0006FFA3335A000337BAB00A3820A0A11A083
:10D9F000054BEF902FF98DE03335A00033756501AD
:10DA000001ED3725F87F834575A085C1E145A30366
:10DA100005A023A0BA0CA5B7394585453726F87F60
:10DA200023A0AA0CA303B6A099BF03A50A0C21F951
:10DA300013099009054BF544A14B228C1375FC0F7B
:10DA400031C903C56A0A7D1C058909E9EFF0AFFFFA
:10DA5000E36625FFEF900FF375D115B703C54A0AAA
:10DA6000631B65012285A685EF309FBE0D89E30803
:10DA700045F103C54A0A631945012285A685EF30A1
:10DA80003FBD3189E30D75EFEF900F9B45D9C5BDC3
:10DA9000014B25B50565EF60CF8403A58A0A23A451
:10DAA0000A0A09C53725F87FA3080594038569A0EC
:10DAB00005052383A9A0E1B5130181FD3725F87F72
:10DAC00006D256C6930AA59903851A02B725F87F90
:10DAD00052C8138A85808345AA1011814ACC1379D4
:10DAE000750026CE4ECA5AC422C299CD03C50A0279
:10DAF000B33520011376F5010545EFA05FD8630A21
:10DB0000A01E0545EFA09FD06305201B03851A02C8
:10DB100003467A0F935515009D896318B60003C616
:10DB20000A02B5467D8A631AD632A30BBA0E634C3D
:10DB3000051C03C50A029375F5016306201F3D46C7
:10DB40006384C5228944638795220D466380C52A74
:10DB50001146638FC52A85496399352F83258A0A23
:10DB60002546636CB62EB395B90093F5053B630665
:10DB7000B02E19816318350583459A0F6374B50477
:10DB800005451544A30CAA0E9305E0022285EF304B
:10DB90003FAC83459A0F6599638495009394150073
:10DBA000458DB704098023ACA40A9305400F228554
:10DBB000EF301FAA83459A0F1375F5FC92054D8D22
:10DBC00023A8A43C09449305100F2285EF305FA8D9
:10DBD000137505088144630395004E89370BF87F60
:10DBE0003705F87F1316290023082B2913892A02E9
:10DBF0009309D52A4E85CA85A686EF408FCC03456A
:10DC00000B297146931525003385B9000D8EA68525
:10DC1000A686EF406FD003C539009375B50F154543
:10DC2000A381B9009305000FEF309FA2137505087B
:10DC30000DC103C55A02098909C505459145EFC0C3
:10DC40004F8F03C50A021375050201E50545EFF084
:10DC50008FE68549930500104E85EFC08F8D4A856C
:10DC6000EFC0CFA03705F87F0345B55205896301A2
:10DC7000A020EFA09F8DEFA0CFFD630BA01E372546
:10DC8000F87F034545A0937525004E856383950075
:10DC90002285B715F87F3726F87FA1463727F87F0A
:10DCA000A38EA57E23288A0A2320D6A0A308379511
:10DCB0006DA215459305000FEF309F991375050868
:10DCC000E306A0E403258A0AF545E311B5E403C59C
:10DCD0000A0285457D8975151375F50FE3E8A5E200
:10DCE00013055002B725F87F2324AA0AA3880594B8
:10DCF000ADA203258A0A9D45631AB5041305600287
:10DD00002324AA0A91A803459A0F89456317B514DD
:10DD100003C50A02FD457D89631DB5121305D002B6
:10DD2000EF30DF913DA21385F5FFBD4563EAA50005
:10DD3000B74501000A05938585012E9508410285A6
:10DD400003459A0F89456306B51035A19305500226
:10DD50002324BA0A6306B5003725F87FA308059483
:10DD60000545EFA0BFAAD5A803459A0F89456302D0
:10DD7000B50EE5A085456315B91403466A0A058A00
:10DD80006300C01419816318B50403469A0F6374C5
:10DD9000C5041544A30CBA0E9305E0022285EF30AA
:10DDA0003F8B03469A0F894565996304B600931526
:10DDB00016004D8DB704098023ACA40A9305400FCB
:10DDC0002285EF30FF8883459A0F1375F5FC920585
:10DDD0004D8D23A8A43C3705F87F0345B55205892E
:10DDE00061ED03258A0A9305700225A603C55A0230
:10DDF000930500081375050F630AB50A930500051E
:10DE0000631DB504370509809D452320B514B1A0D5
:10DE10000545C145EFB0FFF113852A02EFC00F851C
:10DE200003C55A02098909C505459145EFB07FF040
:10DE300003258A0AF9456312B50203456A0A81453A
:10DE400005896306B518754571BD03459A0F6314BE
:10DE500095320545C145EFB08FE71244224BB24AD7
:10DE6000424AD2496249F2449250130181028280AF
:10DE70000945B725F87F13069002B726F87F0547B6
:10DE80002328AA0A23A0C5A0A388E694F9B71545BC
:10DE90009305000FEF30CFFB9375050803258A0A21
:10DEA000636CB0109945E31AB5FA15A20545B7257C
:10DEB000F87FA302AA141DBDEFA0DF826303A01E9A
:10DEC00005459145EFB0AFE003258A0AF54591A4D9
:10DED00003258A0AFD45630AB51C930550026305B4
:10DEE000B50CF1AA03258A0A95456314B50E2145A0
:10DEF000B725F87F2324AA0AA38805943DAA1545CF
:10DF00009305000FEF30CFF413750508E30AA0E284
:10DF100003456A0A058909E93705F87F0345253273
:10DF200013750502E30EA0E00545EFB02FF1E346BF
:10DF300005F203456A0A05890DD103258A0AE545DC
:10DF4000C9AA03456A0A05890DC13705F87F03454B
:10DF500055301375050211E915459305000FEF3093
:10DF60002FEF137505086368A0200545EFB01F83E8
:10DF7000EDB515459305000FEF308FED13750508CE
:10DF8000E300A0DC03456A0A05896361A01A37052E
:10DF9000F87F0345253279AA05442285EFA09FB278
:10DFA0008D452285EFB0AFD2EFF08FFA7DB5032516
:10DFB0008A0A9305F002B1AA99456305B516FD4595
:10DFC000E31DB5E803456A0A0589E36EA0E621452D
:10DFD00011BB03456A0A05892DE115449305C00F5D
:10DFE0002285EF30EFE61365050137090980232804
:10DFF000A93E9305D00F2285EF308FE541891DE1C1
:10E0000015449304E00C2285A685EF306FE4136578
:10E010004500232CA9322285A685EF306FE36D9948
:10E02000232CA93203258A0AA1452324BA0A6306B0
:10E03000B5003725F87FA30805943705F87F13044A
:10E0400045520345240193040005330595026549B3
:10E05000B3552503B7090980154513F6F50F930548
:10E06000300723A4C91CEF30AFDE8345240171992A
:10E07000B3859502B3D52503A1818D894D8D23A646
:10E08000A91C3725F87F834545A013F6250009E62E
:10E0900093E525002302B5A093E505022302B5A070
:10E0A0006DBB03258A0AE945ADA015459305000F10
:10E0B000EF300FDA1375050871E103258A0A9945D7
:10E0C000E31DB5D815459305200FEF306FD815C95E
:10E0D00015449305200F2285EF308FD7B705F87FC1
:10E0E000938445522389A4009305300F2285EF3095
:10E0F0002FD6B7050980A389A40023A4053C238952
:10E100000400054593050004EFB0BFC203258A0A49
:10E110009D452324BA0AE302B5D43725F87FA30826
:10E12000059425BB2145EFA0FF8E05BB3705F87F81
:10E13000034555300989E305A0C009459305100F33
:10E14000EF300FD1137505041DE505458D45EFB082
:10E150000FB8E34405D0854421442685A285EFB05D
:10E160005FBD03456A0A014993752500638C250547
:10E170001375D50F91A805459145F1B90545EF30C7
:10E18000EFCB03456A0A014493752500638585003A
:10E190001375D50F19A0136525002303AA0A05815D
:10E1A0000589EFF04F9103456A0A058963048500EC
:10E1B000754511A0214583258A0A2324AA0AE38EE6
:10E1C000A5C8A1BF136525002303AA0A05810589F7
:10E1D000EFF06F8E91652685EFA0FFF503456A0A83
:10E1E000058963032501754403258A0A23248A0AC5
:10E1F000E30585C61DB73725F87F1305A59F834521
:10E2000015003726F87F93F5750F23040690A300B9
:10E21000B500828021111545F54506CA26C64AC4B7
:10E2200022C2EF30EFC20544937535008944228540
:10E23000638C95001545F545EF308FC19375C5008A
:10E2400021462685639FC508B725F87F938485807E
:10E250002382A40A2285EFF06F8A2285EFF0AF8532
:10E2600003C9440A1545E545EF308FBE631C89009C
:10E270007999B7050980E8D11545E545EF304FBDDF
:10E28000799921A813651500B7050980E8D11545CE
:10E29000E545EF30EFBB13651500B705098037265C
:10E2A000F87FE8D11305A69F83451500394693F5FD
:10E2B000750FA300B5002380041023A0C40C85456E
:10E2C00003C5440A6315B5001305004021A0056588
:10E2D00013050580EF50FF801165EF509F800145C9
:10E2E00031A03725F87F2306058A054512442249C7
:10E2F000B244D24061018280211106CA26C64AC4B6
:10E300004EC222C0EFE03FF4930590096361B50669
:10E310001545F545EF30CFB3854493753500268517
:10E3200081E91545F545EF30AFB2318929C109457D
:10E33000B725F87F1389858001442302A90A228525
:10E34000EFE0DFFB2285EFE01FF78349490A15451F
:10E35000E545EF30EFAF639E99007999B7050980E5
:10E36000E8D11545E545EF30AFAE799931A80544C0
:10E37000B9A813651500B7050980E8D11545E5452D
:10E38000EF300FAD13651500B70509803726F87F0C
:10E39000E8D11305A69F83451500854493F5750FB5
:10E3A000A300B500A145268523000910EFB07F9892
:10E3B00039452320A90C0345490A63159500130527
:10E3C000004021A0056513050580EF508FF12285DF
:10E3D000024492492249B244D240610182803D7197
:10E3E00006CE22C22A841545F54526CA4AC84EC61D
:10E3F00052C4EF30EFA53D8911C53725F87FB945E7
:10E400002324B58C3725F87F9309858003A5090C53
:10E410003DC91544F5452285EF308FA33D891DE99F
:10E42000514A954475491375FA0F19C92685CA854D
:10E430007D1AEF30EFA13D897DD51375FA0F19E9EB
:10E440003705F87F03055552130585071375F50F3A
:10E4500023AAA90A03A5490B15E9EFE0DFDE93051E
:10E4600090096365B502EFE0FFF7EFF0FFE819ED03
:10E4700003A5890A23A4890A630A85003725F87F42
:10E48000A308059421A02285EFF02FB21244224A5E
:10E49000B2494249D244F240056182803D7137253C
:10E4A000F87F06CE26CA4AC84EC652C456C222C0FB
:10E4B0009309858003A5490C11C915459305000FE3
:10E4C000EF300F99098915C123A2090C03C5490A28
:10E4D00009C5EFF0CFB1EF909FD383A5C90B03C55A
:10E4E000091089CD8545630BB5000244924A224A42
:10E4F000B2494249D244F240056182800544631F1B
:10E50000850603C5490A3DC93725F87F1309A59F2C
:10E51000034519002380091093758500B1E911891D
:10E5200031CD3725F87FB705098089441305A59BB0
:10E530009385850C7946A686EF30BFB815459305BF
:10E540001003EF30EF901D8965C515459305100345
:10E55000EF300F909375750005456396A50E8345C2
:10E560001900A380A91093F5B50FA300B90039A035
:10E570001375750FA300A900EFF00F9503AA890A80
:10E580009305D0021305EAFFE3EDA548B745010066
:10E590000A05938585052E950C4103A5C90A828538
:10E5A00089456303B5063725F87F834545A0238257
:10E5B000090A93F5E50F2302B5A0EFE0FFBDEF9048
:10E5C0009FEB01442285EFE07FD32285EFE0BFCEB1
:10E5D000238D090EEFE0BFDB15449305F002228581
:10E5E000EF300F87137505F8B705098023AEA50A2C
:10E5F0009305000F2285EF30AF851375050809C517
:10E600001305800223AAA90A15459305000FEF30D0
:10E610002F841375050801C91545F545EF304F8363
:10E620003D89E301A00E03A5890A8D456F00703E68
:10E6300003451900A38009101375B50FA300A900A5
:10E64000EFF08FC725BF154593051003EF304F80BE
:10E65000834519001D8993F5B50FA300B900E31F89
:10E6600095F0A380991019BF8D456307B502154534
:10E670009305000FEF20DFFD1375050819C9370555
:10E68000F87F03055552130585071375F50F23AA67
:10E69000A90A394523A0A90C15459305000FEF20C1
:10E6A0003FFB13750508636AA0761544F54522857E
:10E6B000EF201FFA3D8905E5D14A9544754913F5C8
:10E6C000FA0F19C92685CA85FD1AEF207FF83D8902
:10E6D0007DD513F5FA0F01E5394523A0A90C03A553
:10E6E000090CE360A034EFE01FB693059009E36ADC
:10E6F000B532EFE03FCFEFF03FC0E364A0326F00F0
:10E70000F00391456309B5760544A1452285EFB034
:10E710004FE21305A0282381091023A8A90A8945DF
:10E7200003C5A90F636FB572154535AF9545E30A6B
:10E73000B52E83C5690A3729F87F1396250003058E
:10E7400049A0218A8589D18D1365150093E525009F
:10E75000B70A098095442302A9A023ACBA0A9305FD
:10E76000F0022685EF20DFEE1365150223AEAA0A1C
:10E77000EF909FA505442285EFA04F891305F00F68
:10E78000A38BA90EF1452685EF209FEC13650501AB
:10E7900023A8AA0603C5A90F630EA0768944E3E661
:10E7A000A40205651305853861AB9945E30BB526D1
:10E7B00005442285238D090EEFA04F8581440D4627
:10E7C0002285A685EFA08F8711462285A685F1AE0A
:10E7D0009D45E308B52405442285EFA02F8381459C
:10E7E00019462285EFA08F851305401F91AB83C585
:10E7F00059140544E3878522B714F87F83C5D47F75
:10E800006304B07A0945639AA5003725F87F83052C
:10E8100045A093E585002302B5A0EF901FA637051C
:10E82000F87FB705F87F1305952C9385D52A714697
:10E830008146EF301F8903A5890A93059002A38EB4
:10E84000047E6F00101DA545E30DB51C05448565CC
:10E850002285EFA05F8E9D452285EFA05FC74DAB5F
:10E86000BD456309B502EFE0DFB515459305F0023C
:10E87000EF201FDE137505F8B7050980054423AEA8
:10E88000A50A2285EFE09FA72285EFE0DFA2794568
:10E8900023AAA90A1545F545EF209FDB0D8985457B
:10E8A000631AB5001545F545EF209FDA318991458A
:10E8B0006302B5021545F545EF209FD90D8909443E
:10E8C000630A85001545F545EF209FD83189A1459C
:10E8D000631FB56403A5890AC1456F009013C14544
:10E8E000630FB500394523A0A90C3705F87F030550
:10E8F0005552130585071375F50F23AAA90A154567
:10E90000F545EF20FFD40D890544631A85001545B0
:10E91000F545EF20FFD3318991456302B5021545D6
:10E92000F545EF20FFD20D898945630AB5001545ED
:10E93000F545EF20FFD13189A1456315B500394573
:10E9400023A0A90C03A5090C630FA04E3725F87F5F
:10E950009304659503C914021545F545EF205FCF73
:10E960003D89630325033705F87F83055552154517
:10E970009385850713F6F50FF54523AAC90AEF20FD
:10E980003FCD3D89A380A40203A5490B09C503C55A
:10E99000F90FE308A0081545F545EF207FCB0D8959
:10E9A00001E91545F545EF20BFCA31896308A07C10
:10E9B0001545F545EF20DFC90D89631385521545CF
:10E9C000F545EF20FFC831899145631BB5500944D7
:10E9D0006F00E07AC545630CB5003705F87F030585
:10E9E0005552130585071375F50F23AAA90A372574
:10E9F000F87F034465971545F545EF207FC58945A8
:10EA00000D896310B44285456314B5021545F5457B
:10EA1000EF201FC431899145631CB5003705F87F8D
:10EA200003055552130585071375F50F23AAA90A87
:10EA300003A5490B6367A07EFDAECD456303B57E9C
:10EA40003705F87F03457552930530023D893385BC
:10EA5000A540B725F87F514639A8D1456303B57C59
:10EA6000EFA07F9C01C50545EFA0EFB9130560310C
:10EA7000B725F87F5546B726F87F054723A8A90A8A
:10EA800023A0C5A0A388E6946F00A079D545630AAA
:10EA9000B57895449305F0022685EF207FBB13756A
:10EAA00005F8370909800544232EA90A2285EFA01D
:10EAB0006F81F1452685A38D090EEF207FB913657F
:10EAC00005012328A906EFA01F966300A0480D4565
:10EAD000B5A9D9456307B57403C5690A03C6990F7B
:10EAE0009315250005490947A189CA866303E600F5
:10EAF000B2860589139616004D8D518DB70A09808F
:10EB000015449304F00223ACAA0A2285A685EF20BF
:10EB10003FB41365150223AEAA0A2285A685EF200D
:10EB20003FB313652500930560093726F87FDD465E
:10EB30003727F87F23AEAA0A23A8B90A2320D6A034
:10EB4000A3082795F9AD15459305F002EF205FB0B6
:10EB5000137505F8B705098023AEA50A0545EF90A2
:10EB60007FF603A5890AE1456DA5E145630DB5482A
:10EB70008544930500102685EFB08F9D6305A0485E
:10EB800005651305853823A8A90A894503C5A90F7A
:10EB90006361B5463D4585A1E5456304B5682285B9
:10EBA000EF90DFC609462285A285EF903FC941AAB2
:10EBB000E9456308B56605448D452285EFA03F9180
:10EBC00063410566930500042285EFB08F963705F3
:10EBD000F87F0345855295451D893305B502930598
:10EBE00030023385A540B725F87F6D4651A6ED4527
:10EBF0006315B524EFE02FE5B705F87F83C56553AE
:10EC00001306F005B385C5026546B3D5C50263FAA0
:10EC1000A56003A5890AF145EDAB05459945EFA02F
:10EC20001F8B2A8463450422054593050002EFB03B
:10EC30004F9003A5890AF545E9AB03C55914630252
:10EC4000855E03C5990F89456318B502054593058F
:10EC50000008EFB0CF9511E9396505449305050229
:10EC60002285EFB0EF8E630AA0640145EFE03F9686
:10EC7000EFE03F9B6367A05A054593050002EFB0A4
:10EC80002F8D6308A0440544C1452285EFB04F8C09
:10EC90006300A046054593050002EFA0CFC951A32C
:10ECA000F9456300B5580544A1442285A685EFA027
:10ECB0001F826358A056930500022285EFA0AFC7BC
:10ECC000714523A8A90A814503C5690A058963031B
:10ECD000B500F5443725F87FB725F87F232095A0A8
:10ECE000A38885943DABFD45630DB55203C509105E
:10ECF000630D85FE0545A545EFA06FFD63430552F5
:10ED0000054491652285EFA00FC303C5690AF1454B
:10ED1000058923A8B90A6360A0423725F87FA14579
:10ED200031A993055002630EB54E05442285EF903C
:10ED30007FD9B5452285EFA08FF96344052471453D
:10ED4000B725F87F1306600225A493056002630AC5
:10ED5000B54C0385A90F0505238DA90EEF804FE75C
:10ED6000EFE09F967DA993057002630CB54A594563
:10ED7000B725F87F6946EDAA930580026303B54A7B
:10ED80005945B725F87F13069002DDA2930590023E
:10ED90006309B5480545EFA0FFAD6354A048B7250A
:10EDA000F87F03C545A03716F87F9376F50D2382CB
:10EDB000D5A0B705F87F1305967F9385B533114627
:10EDC0008146EF300FB003A5890A994599A19305B3
:10EDD000E0026308B54403C5690A05896364A00EAF
:10EDE0002145B725F87F23A4A90AA388059415A96E
:10EDF0009305F0026307B54203C5690A058909C98D
:10EE000015459305000FEF20BF841375050861E5D4
:10EE10007145B725F87F2146A1AA0545EFF02FDC03
:10EE200009A1631AB5001545F545EF207F823189A8
:10EE3000A1456308B53E054501A81305201CB7256B
:10EE4000F87F714635A20145EFE03F96D9AEEFA0BD
:10EE50008FDD01C50545EF901FFB79556303A43C89
:10EE600075A613056002B725F87F3726F87F23A023
:10EE7000A5A0A3088694EFE00FBD9305800963E584
:10EE8000A50203C529100DE105459305B04F3726AE
:10EE9000F87F89463727F87F2381A91023A8B90A6C
:10EEA0002320D6A0A308A794EFE0EFB9930590091B
:10EEB0006369B53603C529106305A03603A5890A21
:10EEC000954581AE15459305000FEF206FF813753A
:10EED00005086308A0347145B725F87F754649A831
:10EEE0001545F545EF20CFF60D8909496312251D1B
:10EEF0001545F545EF20CFF53189A145631AB51ABF
:10EF00000D44B5AC03A5490B636DA0300545EF80FA
:10EF1000AFD2EDAC3705F87F034585529305C0F9B4
:10EF20000D810D893305B5021305251C11BD03A5FF
:10EF3000490B6368A02E0145EF800FD003A5890A15
:10EF400023A4890A630F852CC9AC0945EF90BFEB58
:10EF50002285EF909FBC3705F87F03056552F94580
:10EF600011810D893305B5025105B725F87F594642
:10EF7000B726F87F23A8A90A23A0C5A0A388869452
:10EF80004DA43725F87F1305A59F8345150003A6DB
:10EF9000890A93F5750F93066002A300B50023A4B8
:10EFA000D90A6300D62895ACA1456304B500EF806B
:10EFB0006FD9B724F87F03C544A093751500636F1C
:10EFC000B01203A5890A8945A9A405449305001038
:10EFD0002285EFA0FFD7630AA016056513058538C3
:10EFE000B725F87F3726F87F23A8A90A23A095A084
:10EFF00091AA13056002B725F87F3726F87F23A072
:10F00000A5A0A308969403C5B90F9305500463EA1D
:10F01000A52003C5690A03C6990F93152500094960
:10F02000A189A28663032601B2860589139616007C
:10F030004D8D518DB704098023ACA40A1545930565
:10F04000F002EF20EFE01365150223AEA40A22853B
:10F05000EFA0CFDE6344050423AE090AE54503A50E
:10F06000890A23A4B90A6306B5003725F87FA308E7
:10F070000594054593050010239D090EEFA07FCB55
:10F0800003C5990F631F25191545E945EF204FDC8E
:10F090001375F5FC13650501A8D461A20385B90FAA
:10F0A000930560090505A38DA90E23AEB90A95AA9B
:10F0B0001545F545EF20CFD90D89630A2501154582
:10F0C000F545EF20EFD83189A145631AB50A1144FF
:10F0D0007DA005459165EFA0BFC749C50545914590
:10F0E000EFA01FC76307A01E03A5890AFD4515A24F
:10F0F00003A5C90DB725F87F79469DBD9375050118
:10F10000636AB01811896369A01C15459305000F47
:10F11000EF200FD41375050811C505459165EFA0C3
:10F120003FC34DFD05458565EFA09FC205CD03A5F5
:10F13000890AA545F9A83725F87FF5453726F87FD0
:10F140002320B5A0A3088694E9A8EF90EFB9EF902B
:10F15000CF92EF802FBF030549A01365250023023E
:10F16000A9A0C1A08565054593850580EFA05FBE78
:10F170004DC903A5890A9305E00261A8014415451C
:10F180009305B00F23808402EF208FCC2A84EF7088
:10F190007FFF6304A400EF80EF9203C504020946D9
:10F1A0009305E5FF63F6C50003A5890AC54595A04B
:10F1B0009145631DB504EFE0EFA2EFE0CF8883C572
:10F1C00049141386050283C5F90F637AA60C636A96
:10F1D000B016EFE04F87930510026360B516EFE0BD
:10F1E0008F869305700963EAA5141545F145EF2054
:10F1F0002FC613654500B705098005469306200311
:10F20000A8D9A38FC90E23AAD90A25AA03A5890ABA
:10F21000BD4523A4B90A6306B5003725F87FA308C6
:10F22000059403C5490A23A6490B05CD3725F87F68
:10F23000130505950346150083A5090B21C66366D2
:10F24000B0AAB725F87F83A505A003A6890AA30065
:10F25000050023A4B90A630AB6A8A30005006FF04D
:10F26000CFA803A5090B09C53725F87F232005A0E2
:10F2700003A5090B630BA0A63725F87FA308059407
:10F280006FF0AFA66303B0A63725F87F232005A053
:10F290006FF0AFA503A5890A930550029DBFBDC1BC
:10F2A000A38F090E3705F87F03055552130585070F
:10F2B0001375F50F23AAA90AADB7EFE08FB6E30DDA
:10F2C000859A03A5490EE369A09A0545EFE02FB0A2
:10F2D00065B205459165D1B2EF902FA703C544A053
:10F2E00089451375350F3726F87F93069002372727
:10F2F000F87F2382A4A023A8B90A2320D6A0A308BC
:10F30000879405B71544F1442285A685EF204FB4B4
:10F310006D99370909802328A9062285A685EF2043
:10F320002FB3136505012328A906EFE0BFEEE36ABA
:10F33000A0EE03A5890AD545E9BD03C5F90FE3028F
:10F34000A0EE03A5490BE36EA0EC15459305000F55
:10F35000EF200FB009810D89930580023305B502B6
:10F360002382A9147DBD00003D7106CE26CA4AC87D
:10F370004EC652C422C2EF202FB3630BA016054421
:10F38000370A0F80A145228523208A1423220A14DC
:10F39000EF200FAC2549AA842285CA85EF204FAB08
:10F3A00093D514001375050C93F5F5034D8DAD44FD
:10F3B000930970052320AA162685CE85EF204FA934
:10F3C00013658500232EAA142685CE85EF204FA82D
:10F3D000719913652500232EAA142285CA85EF2072
:10F3E0002FA713758503C1456317B5006545B7059C
:10F3F0000F8023AEA5122D449305C0052285EF2072
:10F400002FA5136515002328AA169305B00522859C
:10F41000EF200FA479992326AA16EF20EFA809441C
:10F4200063148502AD449305C0052685EF204FA2E5
:10F43000136515002328AA169305B0052685EF202D
:10F440002FA179992326AA16EF200FA6AD442A8969
:10F450009305B0052685EF20AF9F6305890011490C
:10F46000A28519A01949CA854D8D9305C00523268B
:10F47000AA162685EF20CF9D336525012328AA16DD
:10F480000545EF20AF9BB7090680930480099305DB
:10F490003007228523A4991CEF208F9B71991309B3
:10F4A000000223A6A91C93055007228523A8291D25
:10F4B000EF200F9A719923AAA91CEF20EF9E6319E0
:10F4C00085021544B709098093053007228523A4D6
:10F4D000991CEF20EF97719923A6A91C930550075B
:10F4E000228523A8291DEF20AF96719923AAA91C74
:10F4F0001244224AB2494249D244F2400561828014
:10F5000021119307400A3305F502B727F87F938747
:10F51000878006CA4AC43389A7000345290926C63D
:10F520004EC222C025E503453909160713770702A5
:10F5300013750504598D1365A5012318C906A30881
:10F5400009082308D908A309A9083725F87F130457
:10F5500085A0814469462285A68693092909EF2062
:10F560005FB6834539091305490713F6F501A285EE
:10F57000A686EF201FB503550907A1651375F51F72
:10F580004D8D85452319A9062380B900024492496F
:10F590002249B244D240610182803D7106CE22C22E
:10F5A0002E848358060026CA254793D5B800BD8906
:10F5B0009304F00F4AC84EC652C46369B71E63076E
:10F5C000D01E9307400A3727F87F3308F502130748
:10F5D00087803A9893F2084013090807A308B808EF
:10F5E0006361500613F8F81FE942B3585802330517
:10F5F000F502B309A70003C5390993841500937771
:10F60000F507138A3909A389F90823100901639DB5
:10F610001405338758023307E84039EF13650508AE
:10F620002300AA00B9E9139726003725F87F1305B0
:10F6300085A08146B2853A86EF20BFA82388890835
:10F64000B1A803560900E946B352D60263F2550841
:10F65000B305F5023306B70083053609819993E5B2
:10F66000A501A309B60875A863E8150103053709C4
:10F6700013650508A309A708DDD5130580063385A2
:10F68000A502B7050780938585F92E959305260079
:10F690001396260079168546EF20BFA203050A00BF
:10F6A000634F050421669395B40013060640137555
:10F6B000050ED18D1365250085442399B906239A3B
:10F6C000090623888908231009002300AA00E9A855
:10F6D000B306F5023303D7008306330993E806F82F
:10F6E00093063309A30913096399B2029952B385AA
:10F6F0005502B295FD8913F608FED18D0DA0B725F0
:10F70000F87F8144138549079385A5A06946A6869D
:10F7100023890908EF20FF9A51A893F5080E23804A
:10F72000B6003305F502FD89B309A700A9C113840A
:10F730002907814579462285AE8693041809138AE4
:10F740003909EF207F9D83C50400138549078DC5C6
:10F7500013068006B385C5023706078083460A0074
:10F76000130686F9B29513F6F601894639A81305F2
:10F77000E00F2389A9081DA883450A00B726F87F52
:10F7800013F6F501938586A08146EF209F930355DC
:10F790000900838504001375F51FAE054D8DA16525
:10F7A0004D8D85442310A400238999081395840165
:10F7B0001244224AB2494249D244F240618505616D
:10F7C0008280000061114145894506C2EF105FE863
:10F7D0007D898D456367B500294581451306000F76
:10F7E00029A02945814513060003EF20CFDFEF1044
:10F7F000BFEB19CD3705F87F03451527A1453D8996
:10F800006318B5002945814513060003EF20AFDDDD
:10F81000924021018280B725F87F03A645A2B70652
:10F820001480136606403797148023A2C5A288C6A9
:10F830002324A78082803725F87F034595A2828004
:10F840003725F87F0345A5A282803725F87F034539
:10F8500085A282803725F87FA30405A28280372500
:10F86000F87F230505A282803725F87F230405A2AF
:10F8700082803725F87F8345B5A205456396A500AC
:10F88000B725F87F2384A5A28280611106C237259F
:10F89000F87F8325C5A281C5FD152326B5A237258E
:10F8A000F87F834575C181C5FD15A30BB5C037250C
:10F8B000F87F834565C181C5FD15230BB5C037258C
:10F8C000F87F832505A381C5FD152328B5A237251B
:10F8D000F87F832545A381C5FD15232AB5A20545DB
:10F8E0009305A015EF10DFD6137605083725F87FAE
:10F8F000834585A301E691C9FD1531A013063006A5
:10F900006365B6008505230CB5A292402101828073
:10F9100011C53705A4802328050082803705A480FF
:10F920009305F002370605809306000C0947B727B8
:10F9300014800CC92328D65823A0E78082803D710B
:10F9400006CE26CA22C62944930480085000228588
:10F95000A6854AC8EF209F811245A68513660540FB
:10F960002285EF204FC81309400830002285CA8540
:10F97000EF20CFFF2245B70500013366B500228591
:10F98000CA85EF204FC62245B70500FFFD15337627
:10F99000B5002285CA85EF200FC51245A6851376CE
:10F9A000F5BF2285EF202FC432444249D244F240B1
:10F9B000056182803705A48085452CD18280211184
:10F9C00006CA26C622C21304000AF1442285A6856F
:10F9D0004AC4EF10FFC7136525003709A480232808
:10F9E000A9062285A685EF10BFC675992328A9060A
:10F9F00012442249B244D24061018280211106CAD8
:10FA000022C0214405659305C5F0228526C64AC457
:10FA10004EC2EF10FFC31379F501056581499304C8
:10FA200025F031A02285A685EF109FC2850913F528
:10FA3000F90FE36925FF024492492249B244D240BA
:10FA4000610182803D7106CE26CA4AC84EC652C4A4
:10FA500022C28144254937440C809149194A11A892
:10FA6000232834FFEF10DF82232844FFEF105F824A
:10FA7000850413F5F40FE375A9FE21452328A4FEA0
:10FA8000EF101F81232804FE1244224AB249424942
:10FA9000D244F24005616FF07FF661110565930570
:10FAA000E531214506C2EF10BFBA1375050793056E
:10FAB00000036314B500EFF0FFF89240210182804B
:10FAC00037050C80BD452322B52E2322052E372570
:10FAD000F87F832545A241767D16F18D2322B5A2BC
:10FAE000828037050C80BD452322B52E2322052EAA
:10FAF0003725F87F832545A241767D16F18D37069F
:10FB00003480930690056547B7270C802322B5A261
:10FB10002320D6502320E65023A0E78082807D71E9
:10FB200006C622C23725F87F0144130595A36D460A
:10FB3000A285A286EF204FDE3725F87FA285A28618
:10FB40001244B240130545A5514641616F20CFDCF8
:10FB5000370584809305F00F13068003B7060C80E9
:10FB60001147B7070580130800026CD110C5F8CE05
:10FB700023AC07558280B71514803786148023A0E4
:10FB8000A58008C6828037450C8093054007130680
:10FB9000000585462328B5C0232A05C0232CC5C0EF
:10FBA000232605C22324D5C22322D5C22320D5C0B3
:10FBB0008280B7450C801306000A23A8C5C023AA7B
:10FBC00005C023A605C223A4A5C2828037460C80A7
:10FBD0009306000A05472328D6C0232A06C02326F9
:10FBE00006C22324A6C2232CB6C02322E6C22320A9
:10FBF000E6C0828061113725F87F06C2B725F87FFD
:10FC00003726F87F230405A63725F87F8546372752
:10FC1000F87FD1473728F87FA38405A6230506A6D9
:10FC20001305D5A6814513060008A305D7A623060C
:10FC3000F8A6EF30F03637450C809305000A4146B0
:10FC40002328B5C0232A05C0232605C22324C5C204
:10FC5000924021016FF09FDA130181FD85652145F6
:10FC60009385D5F006D226CE4ACC4ECA52C856C687
:10FC70005AC422C2EF10DF9D13750502014435E11D
:10FC8000856521459385C5F0EF109F9C7D8941498D
:10FC9000631925050565930425F03725F87F81490B
:10FCA0002144372AF87F930AD5A6372BF87F15A071
:10FCB0002285A685EF10DF9983458AA603069BA6B9
:10FCC0009205D695CE952A962380A500A304CBA6AF
:10FCD0008509E39F29FD03058AA60544050523043C
:10FCE000AAA622851244224BB24A424AD24962490C
:10FCF000F24492501301810282803725F87F130568
:10FD0000D5A68345750303466503A205D18D034639
:10FD1000A503856713174600938707F0131886001D
:10FD20007D8F3378F8004297034895033D8A034E50
:10FD3000D5032206336707013366060113184E0008
:10FD4000220E3378F800B377FE008342E503C297B2
:10FD50000348C503834885038343F5030345B5037F
:10FD600033065640B3E70701B726F87F4697B72812
:10FD7000F87F3723F87F372EF87F33067640372811
:10FD8000F87F3E95B727F87F23A8B6AE23AAE8AE42
:10FD9000230C53AEA30C7EAE232EC8AE23A0A7B077
:10FDA0008280130181FC06DA3725F87F034595A68A
:10FDB00026D64AD44ED252D056CE5ACC5ECA62C84B
:10FDC00066C66AC46EC222C005C5054B1375FB0F1B
:10FDD0000244924D224DB24C424CD24B624BF24AFD
:10FDE000025A92592259B254D2501301810382808F
:10FDF0003725F87F8345A5A60545638BA502A9E1B4
:10FE00003725F87F1305D5A68345E5070D4663E33F
:10FE1000C500B2853726F87F0305F507B726F87FBA
:10FE2000A305B6A62382A6B0EFF03FED014B79BF44
:10FE3000B725F87F8385C5AE3726F87FA302B6B015
:10FE4000B725F87F9385D5A603C62500814685632F
:10FE50009147130700043728F87F9308000E894262
:10FE60003723F87F130E0006994E314F8D4FB72080
:10FE7000F87F1304400C9304D0051309800D938977
:10FE80004300138A4308368B93FAF70FE3F0CAF462
:10FE9000B38B550183CA0B0013FC0A0E630FEC02EF
:10FEA00063001C05631FCC0B032C43A293FCEA01E7
:10FEB000136B4C00232263A363E2DC0503CD2B000C
:10FEC00083CD3B0083CC1B006364B0056312ED055A
:10FED0006390FC0583CB7B00ADA8A303F8B051A0D1
:10FEE00083CB1B00138CABFF636D5C00C91B636A83
:10FEF0007507832B43A2B3EB7B0001A8238300B0DB
:10FF000085A0832B43A293EB0B04232273A391A818
:10FF10002A8B63988D042A8B63159D042A8B639228
:10FF20002C05838C6B00336B3C01232263A363D4C9
:10FF3000DC00336B4C0113FC8C0063C40C006308C1
:10FF400080016304DC00136B0B10232263A383CBBB
:10FF50005B0003CC60B02A8B63757C01238370B196
:10FF60002A8B93FAFA01D697850793FAF70FE37D68
:10FF700056F1A9BD7D7106C63725F87F832545A2B8
:10FF800022C2214513F4052093051008EF104FEC11
:10FF900009EC7999B7050C8023A2A520214593058A
:10FFA0003003EF10EFEA6D9931A813651500B7051E
:10FFB0000C8023A2A520214593053003EF104FE9C3
:10FFC00013654500B7050C8023A6A50C1244B2406A
:10FFD000416182803D7106CE52C40D6A26CA22C09C
:10FFE0001304CA27A1442685A2854AC84EC656C214
:10FFF000EF100FE6137535F8B7DA0C8023A8AA9E28
:020000040001F9
:100000002685A285EF10CFE4930900022A89268570
:10001000CE85EF10EFE30A0541053365250123A8DE
:10002000AA9E2685CE85EF10AFE209C92145A2859B
:10003000EF100FE21365050423A8AA9E93050A2773
:100040002145EF10EFE01365C50023A0AA9C0244F0
:10005000924A224AB2494249D244F2400561828022
:100060003D7106CE26CA9304000222C02A8493055D
:10007000401126854AC84EC652C456C2EF104FDD05
:1000800013190501930580112685EF106FDC2205F9
:100090002A999305C0112685EF108FDBB729F87FC9
:1000A00083D549A20566130A0681B3F545014A9531
:1000B00091C98945630AB4008545631BB4000A05EC
:1000C000954529A0058129A006058D453355B50222
:1000D0009375F50F135685004181B70A2480137676
:1000E000F60F1375F50F9304000223A0BA2A23A874
:1000F000CA2823A0AA28930580122685EF104FD581
:1001000023A8AA2C930540122685EF106FD423A0B4
:10011000AA2C930500122685EF108FD31309C0096E
:1001200023A8AA2A2685CA85EF108FD21365050455
:1001300023A8AA262685CA85EF108FD11365050846
:1001400023A8AA2603D549A2337545011DC105C0C0
:10015000B7050C80054523A0050893054016EF1050
:100160002FCF13651500B705058023A8A558EF000C
:1001700060010244924A224AB2494249D244F240C2
:10018000056182807D7106C622C03724F87F034551
:1001900064B026C29544330595029305600A6362F4
:1001A000B502EF00800C93055015636CB500EF00AD
:1001B000C00B834564B0B385950263F4A500EF00DE
:1001C000E00002449244B240416182807D7106C6E3
:1001D0003725F87F034585B09305000226C222C06B
:1001E000630DB50011E50545B7050C8023A0A51CDE
:1001F0000545B7050C8023AAA51A0544B7040C8051
:100200009305F015228523A2841AEF106FC413659D
:100210000501B705058023AEA556A0C43725F87F94
:10022000832545A21166D18D2322B5A202449244B2
:10023000B240416182803725F87F034585B011E5E2
:100240000545B7050C8023A0A51C37050C80854506
:10025000232AB51A2322B51A3725F87F832545A20C
:100260002166D18D2322B5A282807D7106C622C26D
:10027000EF10801A2A84214593050002EF104FBD2C
:100280000D898945630BB5008545631DB50015458E
:100290003305A4021354250031A00D453305A402F3
:1002A0001354150022851244B240416182807D7151
:1002B00006C622C2130400029305802E2285EF1089
:1002C0002FB91375050FC145630AB50093050003E7
:1002D0006309B50063098500014431A013040004DB
:1002E00019A01304000622851244B24041618280A5
:1002F0006111130500029305C00806C2EF104FB547
:100300001375050419E91305000293058008EF1021
:100310002FB412051375050619A0EFF05FF9B72584
:10032000F87F2384A5B09240210182802111B70576
:100330000C8006CA26C64AC422C2054523A0051C55
:1003400023AA051A23A2051A23A405049305F01570
:10035000EF100FB03D99B70505809304000223AE5E
:10036000A5562145A685EF10AFAE0D692A849305E9
:1003700019054145EF10CFAD05890DE99305290514
:100380004145EF10EFAC05890DE53725F87F0345B2
:1003900085B00D8863029502930500066318B502C7
:1003A0003725F87F832545A2096639A8EFF01FE2BB
:1003B00091A0EFF05FE83DA811C83725F87F8325AD
:1003C00045A2056613060680D18D29A8EFF0FFE946
:1003D00093059025636EB5003725F87F832545A2E8
:1003E00093E505012322B5A22285EFF07FC719A06E
:1003F000EFF05FD912442249B244D24061018280B9
:10040000130181FD130500029305001306D226CEC9
:100410004ACC4ECA52C856C65AC45EC222C0EF1059
:100420002FA31189B7090C809304200823A09940B9
:1004300049E109453544854423A2A9401385094172
:1004400081452286A68623A48940EF10FFCC37255C
:10045000F87F034585B023A8A94013050002930542
:10046000C008EF10EF9E1375050469E5214593055B
:100470004010EF10EF9D6301A01E130500029305CD
:100480008008EF10EF9C2189636FA0169305000C84
:100490001305000223AAB94093058008EF104F9B73
:1004A0004189630BA01A4145B7050C8023ACA540D8
:1004B00065A2130500029305801AEF106F9993054A
:1004C000C004631FB5089304000293050044268509
:1004D000EF100F9823A2A940930540442685EF1002
:1004E0002F97214423A4A940930510102285EF10D3
:1004F0002F962A89930520102285EF106F952A8464
:10050000330589001379F40F130A2508814A138BE8
:10051000094121A8931B250093858B442685EF1064
:100520002F93B3856B0188C1850A13F5FA0FE36336
:1005300025FF45A8130500029305802EEF104F916B
:100540002A89214593054010137AF900EF104F9046
:100550005DC163E5440D13156A0013050504C9A8C0
:1005600009493544130500029305004423A229419B
:1005700023A48940EF10CF8D63109504130500026A
:1005800093054044EF10CF8C631825030149130AEB
:100590001009930A400393040002138B094111A828
:1005A0009305C9442685EF10AF8AB305690188C158
:1005B0001109E31759FF35A00149130A1009930ADD
:1005C000400393040002138B094111A893050944C9
:1005D0002685EF10EF87B305690188C11109E3177C
:1005E00059FFEF0080193725F87F034595B055C1B5
:1005F00023AE094079A819456310AA061305000C1B
:1006000093050006B1A01305000293058008EF10C2
:100610002F84418901ED1305000419A81545636C69
:10062000450113154900130A05FE39A813050008F2
:1006300023AAA94015A01375E90099456316B500D2
:1006400013154900130A05FF1305000C9375FA0FE3
:1006500023AAA94023ACB940EF002012130A1009C5
:100660000DC9B725F87F83C595B095C10D45636B5E
:10067000B500214593055010EF009FFD13658502DD
:1006800023AAA94023AE0940EF00E03019A023AE11
:10069000A9403725F87F032545A2A165E98DB9ED6D
:1006A00099656D8D3DCDA144130940102685CA85FD
:1006B000EF001FFA1375F50923A8A9402685CA85FE
:1006C000EF001FF91365050623A8A9409305101034
:1006D0002685EF00FFF78D4563E5A50421459305C9
:1006E0001010EF00FFF693055A00338AA54011451C
:1006F000B94523A2A94023A4B94025A0A1441309C8
:1007000040102685CA85EF00BFF41375F50923A8AC
:10071000A9402685CA85EF00BFF31365050223A80B
:10072000A9409374F40F0149214409A89305491085
:100730002285EF00FFF12A9A0509FD14E5F81375EB
:10074000FA0F3305A0408D6523A6A94093850527A0
:100750002145EF00FFEF13650503B7D50C8023A0FB
:10076000A59C0244924B224BB24A424AD24962496A
:10077000F2449250130181028280130181FD06D25E
:1007800026CE4ACC4ECA52C856C65AC45EC222C0F1
:10079000EF009048930900022A89930580054E8551
:1007A000EF001FEB131485009305C0054E85EF0085
:1007B0003FEA93040006330AA4004E85A685EF00A5
:1007C0003FE913044006931A85004E85A285EF0089
:1007D0003FE8AA9A930500084E85EF007FE7131BB8
:1007E0008500930540084E85EF009FE62A9B930500
:1007F00080064E85EF00DFE5931B85009305C0065C
:100800004E85EF00FFE49305803E3306B902335670
:100810004603856693860687B305B602B3D565039E
:100820003386AB003725F87FA30405B06319D602E1
:100830000566130606F0638DCA0405666399CA123D
:10084000938695FE05476362D7089305564B63610F
:10085000BA089145A304B5B01304200611AA1305E4
:1008600000286398AA001305001E6314A60005441F
:1008700001A21305002D639DAA029306001E6319B1
:10088000D602138575FC1335450013141500CDA051
:10089000938695FE05466360D60485659385554B22
:1008A000636EBA028D45A304B5B01304D005C9A088
:1008B00093060050639ADA026318A602138515FDA9
:1008C00011466378C5064D4465A06545639EA50243
:1008D0001304300671A8E5466394D5048945A30442
:1008E000B5B01304E00569A01305007801446391D5
:1008F000AA0813058043631DA606138515FD11463E
:10090000637CC5047D44ADA0138635FE0945636153
:10091000A6061386F5FC6378A6041304500689A87E
:10092000938635FE636ED600A304C5B01304F005AC
:1009300081A0138575FC13354500131425000DA8FF
:100940001386F5FC094526846364A602938555FC4D
:1009500063EDA502014531A8138575FC13354500EB
:100960001314450031A0938555FC63E3A5020144AF
:1009700022850244924B224BB24A424AD2496249F2
:10098000F244925013018102828013051006D5B7FC
:1009900013046006F1BF130181FD0D6506D222C26A
:1009A0001304C5282145A28526CE4ACC4ECA52C87A
:1009B00056C65AC4EF00DFC9719937D90C80B70900
:1009C0000C8093051008930400020546154A8D46D5
:1009D00031472328A9A223A0B9589305802A268548
:1009E00023A2C95823A4495923A8D95823AAE958AE
:1009F00023AC0958EF00DFC53D8911C99145630457
:100A0000B5021345350013351500160539A8EFF06A
:100A1000DFD63725F87F834595B0B5C523AE995805
:100A2000034595B039A0130500039305000423AED8
:100A3000B958930A7008014BA14423A0A95A19A8D8
:100A400093054B162685EF00BFC05695050B937A8C
:100A5000F50F7D1AE36640FFB3055041214523A6FB
:100A6000B958A285EF00DFBE136535002328A9A27F
:100A70001244224BB24A424AD2496249F24492504D
:100A8000130181028280014523AE09585DB76111CF
:100A9000130500029305C00806C2EF007FBB137563
:100AA000050409E91305000293058008EF005FBA09
:100AB000158101A8130500029305C02EEF005FB950
:100AC0001D899375F50F01456384A5001385F5FF16
:100AD000B7050C8023A0A508924021018280130154
:100AE00081FD06D226CE4ACC22C037090C80930461
:100AF0004008054429454ECA52C856C65AC45EC26B
:100B00002326994423288944232AA9441305000253
:100B100093050026EF00DFB3631C95001305000268
:100B200093054026EF00DFB2631485000D4511A048
:100B300001450A05814A93690526130AF008130B3B
:100B4000800213040002A144D68B2DA0B385590165
:100B50002285EF00FFAF9385CA4533E625019385D3
:100B60007B1108C22685EF00BFAE5295850B137A24
:100B7000F50F910AE39C6AFD330540418D65232CF6
:100B8000A944938515272145EF009FAC13653500D7
:100B9000B7D50C8023A2A59C0244924B224BB24AAB
:100BA000424AD2496249F244925013018102828042
:100BB000130181FD06D24ECAB7090C8013057008D7
:100BC00026CE4ACC52C856C65AC422C223A2A9482D
:100BD000130500029305C01AEF009FA79305C004F8
:100BE0006318B50613040002930540302285EF0018
:100BF0003FA623A4A948930580302285EF005FA576
:100C0000A14423A6A948930520122685EF005FA4DE
:100C10002A89930530122685EF009FA3B305A9000A
:100C20009374F50F13897508014A938A494921A8DD
:100C3000131B25009305CB302285EF007FA1B30560
:100C40005B0188C1050A1375FA0FE36395FE25A8B9
:100C50000545E944014A1309200A930A8006130452
:100C60000002138B494923A4A94823A6994811A837
:100C700093054A302285EF00BF9DB3056A0188C104
:100C8000110AE3175AFF014A214401A8930555129E
:100C90002285EF00FF9B2A99050A1375FA0FE36777
:100CA00095FE1375F90F3305A0408D6523A8A9485B
:100CB000938505272145EF00BF991365050CB7D52E
:100CC0000C8023A0A59C1244224BB24A424AD2492E
:100CD0006249F2449250130181028280611106C27E
:100CE0003725F87FB725F87F3726F87FB726F87FB6
:100CF0003727F87FB727F87F3728F87FB728F87F9E
:100D0000B722F87F3723F87FB723F87F372EF87F95
:100D1000B72EF87F372FF87FB72FF87FB720F87FEF
:100D2000232205A2238505B0230406A6238406A258
:100D3000A30507B0238607B0A30608B0238308B035
:100D4000238702B0A30503A2238403B023020EB0BD
:100D5000A3820EB023280FAEA3870FB0A38300B0E9
:100D6000EF200052924021016FE07FDB37050580C4
:100D7000C1456146930600081307000693079007D4
:100D8000130800099308F00F930230021303600266
:100D900093036003232E0562232005642322056448
:100DA000232405642326B5642328C564232A056407
:100DB000232CB564232EC564232005662322B56643
:100DC0002324C5662326D5662328D566232AE5660F
:100DD000232CF566232E0567232015692322F56849
:100DE00023240569232615692328F568232A056924
:100DF000232C1569232E55682320656A2322756AE2
:100E00002324056A2326056A2328056A232A556AAE
:100E1000232C556A232E556A82803705F87F930567
:100E2000455203C5750183C58501931665001317E7
:100E300075009D6793F606707D8FD98E1397850098
:100E40009397D500316813770710B3F7070113980C
:100E50001501B7083000337818015D8FB708F87FA7
:100E6000B742CFFF657313763500336707018147BB
:100E700013080002938808479382F2EF1303F38F5D
:100E800081A01DC1B383F80003AE430083AE4302CB
:100E9000137ECEFFB3FE6E00336ECE00B3EED601EE
:100EA00023A2C30123A2D30399C9B383F80003AEDD
:100EB0004304337E5E00336EC70123A2C305A1073E
:100EC000E39107FD8280611141459305002706C229
:100ED000EF000FF811810D8993055005B305B50298
:100EE0001A051365350137063480B706A480370725
:100EF00005802320B61A23A0A60C232E0754924067
:100F00002101828061110545A54506C2EF004FF41D
:100F100013758503C145631EB5043725F87F034566
:100F2000E5B0E5456306B502A945630EB500D145B8
:100F3000630BB50099456315B502294593058005F6
:100F400037C68A3D1DA037F5913D130605B029A08F
:100F500037C53B3D1306053029459305800531A073
:100F600029459305800537D6AD3DEF00DFE7EFE07B
:100F70001F9D3725F87F0345E5B0D145630DB500CA
:100F8000A945630FB50099456311B5023705F87F90
:100F90009305053539A83705F87F9305054111A854
:100FA0003705F87F9305053B29A03705F87F9305A2
:100FB000054729453146EF102F9892402101828044
:100FC0007D7106C626C2C14493050010268522C045
:100FD000EF000FE82A84930500272685EF004FE7EE
:100FE000137505081DE13726F87F832646A23725AD
:100FF000F87F0347E5B09375F40FDD9A2322D6A25C
:101000006308B706230785B095A03725F87F032628
:1010100045A28545B726F87FA385B6A293768600BC
:10102000B725F87F99C683C6E5B01377F40F6381BF
:10103000E604936686001376F40F79472322D5A23F
:10104000238785B06305E60051456319A600EFF0DC
:101050009FE73705F87F9305054F29A03705F87FEF
:101060009305054D29451146EF100F8DEFF09FE9CF
:1010700002449244B24041618280211106CA22C2D8
:10108000414493054020228526C64AC4EF004FDC28
:10109000AA84930520102285EF008FDB3D899305FC
:1010A000E5FF094663E9C50259C99D456305B502D7
:1010B000054463198514B724F87F03C514C1058955
:1010C0006362A014EFF0DFEF370505802328055891
:1010D000A38884C005AA13F514001DED13050003B1
:1010E00093050032EF00CFD66189630DA010414512
:1010F00093054020EF00CFD505896365A010371513
:1011000034809305F00F2320B5C8EFE05F8B3725BF
:10111000F87FA30805C0FDA03725F87F834515C1DA
:101120008989EDE1B71534801306F00F23A0C5C8F7
:10113000830515C193E52500A308B5C0E1A013F50B
:10114000140069E1B724F87F03C514C121895DE962
:10115000EFE0FF862145A388A4C013050003930593
:101160000032EF00EFCE418951CD37153480232076
:1011700085C8EF006FD30DED1304000A93044004FB
:101180002285A685EF00CFCC79993709A480232842
:10119000A9102285A685EF00AFCB13651500232883
:1011A000A9102285A685EF00AFCA79992328A91036
:1011B0003725F87F854537260C809306900A370738
:1011C0003480E5472305B5A22328D6802320F75095
:1011D0002320F680EFE0FF90370505809305000C93
:1011E0002328B5583725F87F0345F5B001CD0945CB
:1011F0009305900FEF00CFC5058909C50545AA8560
:10120000EF201FD112442249B244D24061018280B2
:10121000211106CA3725F87F0345B5B0A54526C676
:101220004AC44EC222C0636DB50605449305601BD7
:101230002285EF00EFC1418925C537050580C145ED
:10124000232AB56C3725F87F832545A24166D18DC9
:101250002322B5A2EF004FC521C5EF00EFC40DED6D
:101260009304000A130940042685CA85EF004FBE87
:101270007999B709A48023A8A9102685CA85EF000B
:101280002FBD1365150023A8A9102685CA85EF0078
:101290002FBC799923A8A9103725F87F230585A2AB
:1012A000024492492249B244D240610182806111D4
:1012B00041459305001006C2EF008FB99945630EB2
:1012C000B500E545630EB500D145630EB500A945EF
:1012D000631EB5001305E01021A81305200A09A814
:1012E0001305302A31A01305C02119A01305A0321F
:1012F000924021018280211106CA26C64AC44EC2EC
:1013000022C0EFF0DFFA2A84A14405659305F5E2D7
:101310002685EF00EFB31319050105659305E5E296
:101320002685EF00EFB222052A9905659305D5E2DF
:101330002685EF00EFB12A990565930525E32685FB
:10134000EF000FB1931905010565930515E3268597
:10135000EF000FB02205AA990565930505E32685E0
:10136000EF000FAFB30524031306803E4E95B385FF
:10137000C502B3D5A50237D50C801306D0032324AC
:10138000059CA58163E5C5009305000311A0E14517
:1013900041462326B59C2328C59C024492492249F4
:1013A000B244D240610182807D7106C622C013041E
:1013B000000293058014228526C2EF006FA92189BF
:1013C00001C937052480A1452320B552EFF0BFF2B3
:1013D00021459305200CEF00AFA71375050205C941
:1013E000B7040C8023A48430130000001300000015
:1013F00021459305200CEF00AFA51375050201C927
:101400000545B7050C8023A0A42623A00526024489
:101410009244B24041618280211106CA26C64AC464
:101420004EC222C0EFF0BFE8930400022A84930565
:1014300040112685EF00CFA11319050193058011F6
:101440002685EF00EFA022052A999305C011268575
:10145000EF000FA02A99930500122685EF004F9FF9
:1014600093190501930540122685EF006F9E220512
:10147000AA99930580122685EF008F9D4E95B3059E
:101480008902024492492249B244D24033D5A5028E
:1014900061018280211106CA22C23724F87F4AC422
:1014A000130944A20345190026C6098955C1EFE076
:1014B000DFDB832544A219666D8E19C679767D1609
:1014C000F18D05812322B4A2B7040C809305501539
:1014D00023A404166360B5023705058089450546D7
:1014E0008D463727F87F2326B56C23A8C414230F15
:1014F000D7C02DA89305400A33B5A500B7050580D0
:1015000023A6A56C03451900058911E93725F87F45
:10151000B7050C80230F05C023A8051401A80545B5
:10152000B725F87F238FA5C023A8A414032544A2C0
:10153000136525002322A4A2EF1090541305000286
:101540009305C012EF00CF900981058923AAA40852
:1015500012442249B244D24061018280372524805E
:101560008945232005B02328B5B0232005B22328C0
:10157000B5B282800945B725F87FA385A5B08280E2
:10158000211106CA4AC40D6926C622C01304C92700
:10159000A1442685A2854EC2EF008F8B13651500EE
:1015A000B7D90C8023A8A99E2685A285EF004F8A73
:1015B000759937040C8023A8A99E930530032685CE
:1015C0002328041423240416EF008F8879992326F6
:1015D000A40C930509272685EF008F87137535F036
:1015E00023A0A99C9305C9282685EF006F867199D1
:1015F000B715148037262480894623A8A9A223A8DA
:101600000530232006B02328D6B0232006B2232895
:10161000D6B2EFE0CFD0130500029305C009EF006A
:101620002F831375F5F3370424802328A426B724C9
:10163000F87F03A544A2C5759385F57E6D8D23A221
:10164000A4A2054593054016EF008F807999B70550
:10165000058023A8A55823200434B725F87F03A5C7
:1016600044A2A38505B00244759923A2A4A292497D
:101670002249B244D24061018280611106C2EFF07A
:101680003FF037250C809305900A37060C80BD4645
:101690002328B5802322D62E2322062EB725F87FB5
:1016A00003A645A2C176FD16758E9306700A23A285
:1016B000C5A22328D58092402101828061111305A3
:1016C00000029305C01306C2EFF09EF8218901C9FC
:1016D00037052480A1452328B54EEFE07FD2924004
:1016E000210182806111130500029305C01306C217
:1016F000EFF01EF6058901C93705248085452328AA
:10170000B54EEFF0CFBD924021018280AA860145FF
:101710000547AA8713F8F70F637EC800931848009F
:10172000B6982E9883A80800034808008507E3832D
:1017300008FF3A8582803D7106CE26CA93040002D6
:101740009305C01326854AC84EC652C422C2EFF084
:101750003EF013750502014421C537052480B725E5
:10176000F87F2328954E938445A5371524801305CB
:1017700005AA5146A685EFF07FF91DC11309802AFD
:101780000544130A802F9309000209A84E85CA85D3
:10179000EFF01EEC2380A40011098504E31849FF33
:1017A00022851244224AB2494249D244F24005619C
:1017B00082806111130500029305001406C2EFF048
:1017C0003EE919819240058921018280211113058A
:1017D00000029305C01306CA26C64AC44EC222C0E0
:1017E000EFF01EE71375050839C53705248093050A
:1017F00000082328B54E3725F87F130495A3371525
:101800002480130505C16D46A285EFF03FF005C5A4
:1018100093044030930900371309000209A84A8550
:10182000A685EFF0FEE22300A40091040504E398EE
:1018300034FFEFF0EFB7024492492249B244D2405C
:1018400061018280370505809305F00F37163480DB
:10185000930600043707848091472328B56C23281A
:10186000D6922320B6C8232AF71082803D7106CE77
:101870004EC68D6926CA22C037151480B7851480DC
:101880009384C92721444AC852C456C237C614801B
:101890002320058023A405002285A6852322061483
:1018A00023240614EFF0DEDA1365150037D90C8017
:1018B0002328A99E2285A685EFF09ED97599370A1F
:1018C0000C802328A99E93053003228523280A141F
:1018D00023240A16EFF0DED779999384092723266B
:1018E000AA0C2285A685EFF0BED6137535F023200D
:1018F000A99C9385C9282285EFF09ED57199B725BB
:101900002480894A2328A9A223A005B023A855B181
:1019100023A005B223A855B3D9452285EFF05ED3A5
:1019200013651500232CAA042285A685EFF05ED24C
:1019300079992320A99C938519272285EFF05ED100
:101940007199B7250C801306900AB7043480E546D8
:101950003707A4809307F002370805809308000C2E
:10196000B72214802322A99C23A8C58023A0D45089
:1019700023A0D5801CCB2328185923A05281EFF037
:10198000EFB5EFF07ED205E9130400039305800262
:101990002285EFF0FECB4D991365450023A0A40AE4
:1019A000930580262285EFF0BECA13650508B7159A
:1019B000348023A0A59A3726F87F8546A304D6A2B3
:1019C00081450244924A224AB2494249D244F240F5
:1019D00029452E8605616F000FC1211106CA3725E2
:1019E000F87F034585A39305B00526C64AC44EC2B9
:1019F00022C0636EB5023725F87F8345B5A209463C
:101A0000638AC5066365B022B725F87F83C515874D
:101A100005468589A305C5A2630BB0203725F87F4D
:101A2000832545A293E505402322B5A209A4A54537
:101A300063EFA51E3729F87F0345B9A289496307DB
:101A4000350985456315B51E414593050027EFF01F
:101A50003EC013750508636CA01C3725F87FB725B9
:101A60000C801306900AA30539A3230805B023A808
:101A7000C58075AA85453726F87FB7260C80A30553
:101A8000B5A2230A06C023A806803725F87F0345A0
:101A9000B5B0636EA01805659305E5312145EFF0FB
:101AA0003EBB137505076364A018414593054020AC
:101AB000EFF01EBA0589636CA0163725F87FB725AD
:101AC000F87F230505B0A38605B095A23724F87FDB
:101AD000034504B18544630F9500630735078D45C1
:101AE000630CB50C91456317B50EA30509A2EFF081
:101AF000FFD735AA3729F87F032549A36369A012C8
:101B0000EFD0DFEF37050C809305F00F37460C80E0
:101B10009306000A1307F007232CB530232EB530A7
:101B20002328D6C0232A06C0232606C2232496C211
:101B3000232CE6C0232296C2232096C0A945030584
:101B400004B1232AB9A2CDA021459305600CEFF082
:101B50003EB0137505082DC921459305700CEFF0B3
:101B60003EAF137505044DED3725F87F85650349B4
:101B700045B02145938525F0EFF09EAD6312250B0E
:101B8000EFD0DFE73725F87F0345B5A645C93745D0
:101B90000C809305000A1306F00F2328B5C0232AF2
:101BA00005C0232605C2232495C2232CC5C02322A9
:101BB00095C2232095C0BDA021459305600CEFF090
:101BC0003EA91375050811ED3725F87F032545A3B8
:101BD00039EDB9A0A9453726F87F0505232AB6A215
:101BE000A9A021459305700CEFF09EA6137505047E
:101BF00015E93725F87F8565034955B0214593855B
:101C000025F0EFF0FEA4631D250113050019B7258B
:101C1000F87F230894B023AAA5A2EFD03FDE01A845
:101C2000114521A0030504B105052308A4B0024411
:101C300092492249B244D2406101828013050019C1
:101C4000B725F87F23AAA5A2230894B0CDB75D716C
:101C50003745010086C69305C519A6C2CAC05ED61F
:101C600090453400D841CC450325C519B7070580F8
:101C70001308F00FB71834809302000437038480F0
:101C8000914B3709A4809303F002130E000CB72E7A
:101C9000148089444EDE52DC56DA5AD862D466D2B9
:101CA0006AD06ECE22CC90C6D8C22ECA2AC423A82F
:101CB000076D23A8589223A008C9232A731123284B
:101CC000790023A8C75923A09E80EFF02F8A0D45E5
:101CD000B70924801304000237DA0C80B70514809A
:101CE000514C554B13061008B79C148093063008CE
:101CF000854A2D479307000F7948371D14809308B4
:101D000020029302900B930D70031303500393036F
:101D100010032320A90C23A0894023220A9C23A27C
:101D2000850123AA6501D0CD23AECC8084D123AA1E
:101D3000050223AA0C8294DD23ACDC8223A00524B7
:101D400023A8550123A85C8123A4750323A47C83C5
:101D500023A0E52023A2F52023A4952023A6052176
:101D600023A0051823200D4023221D4123245D407C
:101D70002326BD4123286D40232A7D40EF00EFA597
:101D80006319550113050003232CAD4023A28C8158
:101D900031A8EF008FA463159500232CBD4139A015
:101DA00013058003B715148023ACA5401305A00BC1
:101DB000D94537C61480A9442322AD4223246D435C
:101DC0002326BD42232056012C0009462685EF001C
:101DD000AFB6814526852E86EF00EF80B7043480AC
:101DE00037252480B7050C801306D00FB7160C805A
:101DF00041479307900F69489308B00A9302100B6C
:101E00003D4323A804182320853A23A6052623282A
:101E1000C53A23AAE6C02328F5222320052123283A
:101E2000152123205522232065309305C0092285E2
:101E3000EFF01E8213654500B7550C801306A0060F
:101E40009306B0091307800523A8A92623A0C5D0AF
:101E50002322DAA22320590123A8E40AEFE01FE895
:101E60003725F87FB725F87F230C05A223A805A204
:101E7000EFF09E8311ED15459305200CEFF04EFD1C
:101E8000137575FC13650503B705098023A4A530F8
:101E90006244F24D025D925C225CB25B425BD25ABC
:101EA000625AF25906499644B640616182807D715A
:101EB00006C63725F87F832545A23726F87F0346D7
:101EC000B6A226C293F5F5BF854422C02322B5A24F
:101ED00063179604EFF04EFD05E913040003930524
:101EE00080022285EFF0CEF64D99B705348023A00D
:101EF000A50A930580262285EFF08EF51375F5F778
:101F0000B715348023A0A59A3725F87FB705A4809C
:101F1000230495A2A4D1EFF0AFE6EFD09FBC02441A
:101F20009244B24041618280611113050002930521
:101F3000C00F06C2EFF0CEF11D8979158D4563EA19
:101F4000A500B74501000A059385C51A2E950841DD
:101F500011A00145B7050C8023AAA52492402101B8
:101F60008280211106CA22C22A8413F5F50FA181AD
:101F700037C7148093F5F50F9377F60F218226C6A5
:101F80004AC41376F60F2328A714232AB71413057F
:101F900000029305C008232CF714232EC714232016
:101FA000D71623220716EFF0AEEA1375050409E9E8
:101FB0001305000293058008EFF08EE9158101A852
:101FC000130500029305C02EEFF08EE81D89B7259A
:101FD000F87F83A545A20566130606816D8E09CE9E
:101FE0001375F50F8D456300B50289456311B50280
:101FF00013152400954511A819656D8D3335A00082
:102000003354A40029A0131514003354B50293557A
:1020100084001375F40F3709248093F5F50F1356D8
:102020000401130400029304C0091376F60F93060B
:1020300000082320A92A2328B9282285A685232041
:10204000C9282328092C2320D92C2328092AEFF07A
:102050002EE0136505042328A9262285A685EFF026
:102060002EDF13650508B715148005462328A92619
:1020700023A8C53012442249B244D2406101828073
:102080000146B726F87F3725F87F138716B18545B7
:10209000930700083288A30705B063E50503B28201
:1020A000B28839A0330357000303030085029A98CE
:1020B000E39AF2FE93F8F80F050813070708E30EFA
:1020C00010FD61AA3726F87F032806AF3566130690
:1020D000D6286360C806B727F87F83A747AF85680F
:1020E00005479388F8EFA307E5B063E6F80489682D
:1020F0009388087133081803B352F8023728F87F21
:10210000032808B01303D008B3D2020363E56206C4
:10211000B387070313088007B3870703B3D71703F1
:10212000138816B193D88700230BF802A30B18036A
:1021300099A00147B5A08568938808F7330818036C
:10214000B357F802138816B1930800079302000FE3
:1021500013030002414E93D38700230BF802A30B15
:102160007802A30C1803230D5802230C0802230F36
:102170006802A30FC80301489308F007938716B1BC
:10218000C28209A8338307010303030005089A925A
:1021900093F2F20FE31818FF33085040A38F07079C
:1021A000B727F87F83C777B0CDCB938616B19388D6
:1021B0000708B697938717080148B6989302000658
:1021C0001303F00529A8B383070103CE0300636757
:1021D0005E002E8723806300A307B5B0050883C384
:1021E000080093F3F301E36078FE83852608938566
:1021F00005F893F5F50FB69583C7150003C80500DC
:10220000A207B3E7070163E4C7020146494711A8E3
:10221000B387C600838767033388C5002300F800AF
:102220000506E317E6FE8545A307B5B021A01375A3
:10223000170005C501459305F0072A8609A83387CD
:10224000A6000307070805053A961376F60FE3186C
:10225000B5FE3305C040A38FA60E82807D7106C6F1
:1022600022C23724F87F0346D4B089456308B602FA
:1022700005456307A60471E2B725F87F37460C8051
:102280009306000A2147238405A62328D6C0232AC3
:1022900006C0232606C22324E6C271A8856521450F
:1022A0009385D5F0EFF0CEBA137505023DED1545D7
:1022B000B725F87F054623A6A5A2A306C4B0B5A8F6
:1022C0003726F87F8326C6A2ADEA3727F87F8347F3
:1022D000B7A6B726F87F03C786A69207C107637B18
:1022E000F704B728F87F13183700B7470C80938896
:1022F00018B123AC07C146988148A14201A8330315
:1023000018010343030023A267C08508E39958FE20
:102310007948050723A2B7C223A0A7C0232606A396
:102320002384E6A6A306B4B009A83725F87F0325C1
:10233000C5A201E50D45A306A4B01244B240416117
:1023400082803D7106CE52C4130A000293058005B7
:10235000528526CA4AC84EC656C222C0EFF04EAFBA
:10236000131485009305C0055285EFF06EAEB30AD5
:10237000A400930500065285EFF08EAD13044006CD
:10238000AA845285A285EFF0AEAC2A899305000598
:102390005285EFF0EEABAA89930540055285EFF028
:1023A0002EABB725F87F03A645A205679376F6FD09
:1023B000130707F723A2D5A26393EA069396840036
:1023C0000567CA96130707F0639BE6042167939697
:1023D0008900130707F0F98E3695C1466311D504BD
:1023E000136506023726F87F032606AF23A2A5A2AF
:1023F0009314F600EFE0BFEB33D5A4023726F87F45
:10240000B726F87FB725F87F0326C6AF83C696AFF9
:1024100083A545AF369633558502EFF09FB402444D
:10242000924A224AB2494249D244F240056182802E
:10243000211106CA22C03724F87F0345D4B04AC40C
:102440000D4926C64EC2630025038544630A9508DC
:102450008945630CB50A6364A012EFD0AFF9030598
:10246000D4B005059DA83729F87FB729F87F8344A4
:10247000A9A603C5B9A663629504054563619502E3
:10248000B725F87F13957400938515B12E95B72560
:10249000F87F9385D5A613060008EF106028EFD0CB
:1024A0005F90850413F5E40F0581B7450C80230583
:1024B00099A623AAA5C003C5B9A693F5F40F637323
:1024C000B5063725F87F832545A213F6450009E6B2
:1024D00093F5F5DF2322B5A21145A306A4B045A0CC
:1024E000B725F87F3725F87F83C5A5A6034585A6C0
:1024F0001396350032951316450037450C80232C72
:10250000C5C063EDB402A6851DA8EFD0EFF429C5C0
:102510003725F87F034585A69D4563F0A506A306EC
:1025200024B1B1A83725F87FB725F87F05462304E5
:1025300005A6A38405A6A306C4B091A0914579463B
:10254000B726F87F09472322B5C2232095C023A6CA
:10255000C6A2A306E4B025A03725F87F0325C5A2AF
:1025600019ED3725F87F8345C5A6BDD5FD15230692
:10257000B5A6EFD02FCDEFE0BED1A30694B00244B4
:1025800092492249B244D24061018280797106D6D3
:102590005EC6930B0002930580055E8526D24AD065
:1025A0004ECE52CC56CA5AC862C466C222C0EFF0A0
:1025B0002E8A2A849305C0055E85EFF06E892A89EC
:1025C000930500065E85EFF0AE88AA849305400669
:1025D0005E85EFF0EE87AA89930580045E85EFF0B3
:1025E0002E872A8A9305C0045E85EFF06E86AA8A3C
:1025F000930500055E85EFF0AE852A8B93054005B7
:102600005E85EFF0EE84B725F87F83C545A293F58C
:102610000502EDE193158400B38B250193158A0023
:102620002166AE9A93158B00130606F0F18D33895F
:10263000A50013958400B3853B413385A540B309BC
:102640005541338B2A4193D419001305C002135A04
:102650001900636065091304000293054011228587
:10266000EFE01EFF131C0501930580112285EFE0AA
:102670003EFE22052A9C9305C0112285EFE05EFDF7
:102680002A9C930500122285EFE09EFC931C050115
:10269000930540122285EFE0BEFB2205AA9C93051C
:1026A00080122285EFE0DEFA93858B07B3856541C2
:1026B0001396F5003356760366959376E9FF330655
:1026C00086033355A60213868A0733066641EFF068
:1026D0005F8913559900B72524801376FA0F93D696
:1026E000990023A0A5B013F5F40F23A8C5B023A02B
:1026F000D5B21DA037252480B725F87F232005B04B
:1027000083C595AF85812328B5B0232005B2372531
:10271000F87F034585AF0581B725248013040002A7
:1027200023A8A5B2930500052285EFE07EF2A1441F
:1027300013094009137A05082685CA85EFE05EF182
:10274000814963053A011365250011A07599370A7F
:102750000C80930580072328AA242285EFE05EEFF2
:10276000137405082685CA85EFE09EEE63053401E3
:102770001365150011A079992328AA240244924CCC
:10278000224CB24B424BD24A624AF249025992540D
:10279000B25045618280211106CA26C64AC44EC283
:1027A00022C0EFF00F8111C53725F87FA30505B0D2
:1027B00091A83724F87F0345B4B08D446364950431
:1027C000EFE07FF701CD130500029305C008EFE0AD
:1027D0003EE81375050415E1EFE0EF9B0345B4B047
:1027E000A5456361B5021305000693050004EFE0FB
:1027F0003EE6118919ED3D4521A0EFE07FD809455E
:10280000A305A4B0024492492249B244D2406101D6
:1028100082800345B4B0B945631AB50021459305DC
:10282000200CEFE0FEE21375050849ED13050002E8
:1028300093050014EFE0DEE1137505080DC53705BB
:102840002480930500082320B55013050003930549
:10285000C014EFE0FEDF930590066366B500EFE07D
:10286000DFE1A30594B0214593053060EFE05EDE23
:102870009305E00F6311B5023725F87F834585C1C5
:10288000294663EAC500B7250C801306B00A23A8C1
:10289000C580230C05C00345B4B0AD45E364B5F66F
:1028A000414593051020EFE0BEDA11891DE537257B
:1028B000F87F832545A241666D8E29D641767D1627
:1028C000F18D71A037050C80930500082324B530E5
:1028D000EFE0BFDAA30594B035B705449305601B5C
:1028E0002285EFE0FED6137605013725F87F832594
:1028F00045A221EE4166B3F6C50089F6D18D2322AB
:10290000B5A2EFE07EDA0DED9304000A130940044E
:102910002685CA85EFE0DED37999B709A48023A87C
:10292000A9102685CA85EFE0BED21365150023A83D
:10293000A9102685CA85EFE0BED1799923A8A910F0
:102940003725F87F230585A275BD4166D18D2322E9
:10295000B5A24DBD3D7106CE26CA4AC84EC652C468
:1029600022C2EFF05FE3B729F87F03C5B9B0B545E0
:10297000791563EFA508B74501000A059385051190
:102980002E9508410285130500029305C008EFE06B
:102990003ECC137505046306A032130500029305AF
:1029A000C013EFE0FECA137505026301A032EFE029
:1029B0009FD8EFD05FFE31A6EFE06F8DEFD05F9331
:1029C000EFD0DF963725F87F032505AFB5659385F2
:1029D000D528636BB50009459305900FEFE05EC7FE
:1029E000058919C1EFF0FF95EFF05FBA0545A545E0
:1029F000EFE01EC613758503C1456314B52C15455C
:102A0000B725F87F194623A6A5A2A385C9B07DAC3A
:102A10001305000293050014EFE09EC3137505042F
:102A20006306A02A1305000293050014EFE05EC2BE
:102A3000137585086304A02A370524809305800850
:102A40002320B55061A43724F87F0325C4A2636F07
:102A5000A026054593054016EFE09EBF13650504CB
:102A6000B705058023A8A55891450385B9B023264D
:102A7000B4A291AC3725F87F0325C5A26368A024D2
:102A8000054593054016EFE0BEBC1375F5FBB70591
:102A900005809304000A1304000223A8A558268584
:102AA000A285EFE0FEBA13658500370AA4802320D3
:102AB000AA082685A285EFE0BEB95D997149232059
:102AC000AA082685CA85EFE0BEB8136585002328CD
:102AD000AA062685CA85EFE0BEB75D992328AA0617
:102AE0003725F87F032545A281451375050263004C
:102AF000B51C130400041305200865AA130500067D
:102B000093050004EFE0DEB411896301A01C3705D2
:102B10000C80930500082324B530EF30EF8C8385BB
:102B2000B9B029453726F87F85052326A6A2A385B7
:102B3000B9B069AA3725F87F8325C5A26368B018A4
:102B40009305401F37240C809304900A2326B5A2D6
:102B500015459305700F23289480EFE07EAF137521
:102B6000050F9305000F631EB514130500039305AD
:102B7000001423289480EFE0BEAD13650502B7056D
:102B8000348023A0A550214593050060EFE05EACA2
:102B9000136505022320A4802DA23725F87F032585
:102BA000C5A26365A012EFC05FEF21AAEFD05F85D9
:102BB000EFD04FC2EFE01F8E3725F87F034545A2C7
:102BC00013750508630FA00E13050005B725F87FE0
:102BD00023A6A5A2FDA03724F87F0325C4A27DE586
:102BE0003725F87F0345E5C18D456317B5000545D9
:102BF000B7050C8023A4A516214593053003EFE00B
:102C00003EA513651500B7050C801306400623A6E4
